:020000040800F2
:1000000000800020792D0008B11A0008B31A0008FA
:10001000B51A0008B71A0008B91A00080000000055
:10002000000000000000000000000000BB1A0008F3
:10003000BD1A000800000000BF1A0008C11A00081D
:10004000C92D0008C92D0008C51A0008C92D0008CF
:10005000C92D0008C92D0008D11A0008D71A0008B8
:10006000C92D0008C92D0008C92D0008C92D000898
:10007000C92D0008C92D0008C92D0008DD1A000887
:10008000C92D0008C92D0008C92D0008C92D000878
:10009000C92D0008C92D0008E91A0008C92D00085B
:1000A000C92D0008C92D0008C92D0008C92D000858
:1000B000C92D0008C92D0008C92D0008C92D000848
:1000C000C92D0008C92D0008C92D0008C92D000838
:1000D000C92D0008F11A0008C92D0008C92D000813
:1000E000C92D0008C92D0008FD1A0008C92D0008F7
:1000F000C92D0008C92D0008C92D0008C92D000808
:10010000C92D0008C92D0008091B0008C92D0008C9
:10011000C92D0008C92D0008C92D0008C92D0008E7
:10012000C92D0008C92D0008C92D0008C92D0008D7
:08013000C92D0008C92D0008CB
:1001380010B5054C237833B9044B13B10448AFF319
:1001480000800123237010BD08010020000000007A
:1001580030F4000808B5034B1BB103490348AFF35B
:10016800008008BD000000000C01002030F40008E9
:10017800034613F8012B002AFBD1181A01387047DF
:1001880081F0004102E000BF83F0004330B54FEA40
:1001980041044FEA430594EA050F08BF90EA020FAD
:1001A8001FBF54EA000C55EA020C7FEA645C7FEA40
:1001B800655C00F0E2804FEA5454D4EB5555B8BF63
:1001C8006D420CDD2C4480EA020281EA030382EAD4
:1001D800000083EA010180EA020281EA0303362D66
:1001E80088BF30BD11F0004F4FEA01314FF4801C39
:1001F8004CEA113102D0404261EB410113F0004F4B
:100208004FEA03334CEA133302D0524263EB430301
:1002180094EA050F00F0A780A4F10104D5F1200E9F
:100228000DDB02FA0EFC22FA05F2801841F10001FA
:1002380003FA0EF2801843FA05F359410EE0A5F1CE
:1002480020050EF1200E012A03FA0EFC28BF4CF0FF
:10025800020C43FA05F3C01851EBE37101F00045B5
:1002680007D54FF0000EDCF1000C7EEB00006EEBC2
:100278000101B1F5801F1BD3B1F5001F0CD349084C
:100288005FEA30004FEA3C0C04F101044FEA4452A3
:1002980012F5800F80F09A80BCF1004F08BF5FEA2A
:1002A800500C50F1000041EB045141EA050130BD0A
:1002B8005FEA4C0C404141EB0101013C28BFB1F51C
:1002C800801FE9D291F0000F04BF01460020B1FA67
:1002D80081F308BF2033A3F10B03B3F120020CDA3A
:1002E8000C3208DD02F1140CC2F10C0201FA0CF018
:1002F80021FA02F10CE002F11402D8BFC2F1200C7D
:1003080001FA02F120FA0CFCDCBF41EA0C01904032
:10031800E41AA2BF01EB0451294330BD6FEA04047B
:100328001F3C1CDA0C340EDC04F11404C4F1200266
:1003380020FA04F001FA02F340EA030021FA04F378
:1003480045EA030130BDC4F10C04C4F1200220FACF
:1003580002F001FA04F340EA0300294630BD21FA0D
:1003680004F0294630BD94F0000F83F4801306BFD3
:1003780081F480110134013D4EE77FEA645C18BFC7
:100388007FEA655C29D094EA050F08BF90EA020F5E
:1003980005D054EA000C04BF1946104630BD91EA56
:1003A800030F1EBF0021002030BD5FEA545C05D159
:1003B8004000494128BF41F0004130BD14F5800498
:1003C8003CBF01F5801130BD01F0004545F0FE410C
:1003D80041F470014FF0000030BD7FEA645C1ABF41
:1003E800194610467FEA655C1CBF0B46024650EA78
:1003F800013406BF52EA033591EA030F41F40021A4
:1004080030BD00BF90F0000F04BF0021704730B529
:100418004FF4806404F132044FF000054FF00001FE
:1004280050E700BF90F0000F04BF0021704730B5BF
:100438004FF4806404F1320410F0004548BF404294
:100448004FF000013EE700BF42004FEAE2014FEAE9
:1004580031014FEA02701FBF12F07F4393F07F4FC4
:1004680081F06051704732F07F4208BF704793F0C7
:100478007F4F04BF41F40021704730B54FF46074DA
:1004880001F0004521F000411CE700BF50EA0102DD
:1004980008BF704730B54FF000050AE050EA010286
:1004A80008BF704730B511F0004502D5404261EBF6
:1004B80041014FF4806404F132045FEA915C3FF437
:1004C800D8AE4FF003025FEADC0C18BF03325FEAD4
:1004D800DC0C18BF033202EBDC02C2F1200300FA85
:1004E80003FC20FA02F001FA03FE40EA0E0021FAAA
:1004F80002F11444BDE600BF70B54FF0FF0C4CF498
:10050800E06C1CEA11541DBF1CEA135594EA0C0F49
:1005180095EA0C0F00F0DEF82C4481EA030621EA84
:100528004C5123EA4C5350EA013518BF52EA0335BF
:1005380041F4801143F4801338D0A0FB02CE4FF071
:100548000005E1FB02E506F00042E0FB03E54FF0A1
:100558000006E1FB03569CF0000F18BF4EF0010E99
:10056800A4F1FF04B6F5007F64F5407404D25FEA95
:100578004E0E6D4146EB060642EAC62141EA555148
:100588004FEAC52040EA5E504FEACE2EB4F1FD0C8A
:1005980088BFBCF5E06F1ED8BEF1004F08BF5FEA08
:1005A800500E50F1000041EB045170BD06F00046BA
:1005B80046EA010140EA020081EA0301B4EB5C0467
:1005C800C2BFD4EB0C0541EA045170BD41F480115F
:1005D8004FF0000E013C00F3AB8014F1360FDEBF84
:1005E800002001F0004170BDC4F10004203C35DA60
:1005F8000C341BDC04F11404C4F1200500FA05F3E3
:1006080020FA04F001FA05F240EA020001F0004283
:1006180021F0004110EBD37021FA04F642EB0601F9
:100628005EEA430E08BF20EAD37070BDC4F10C0423
:10063800C4F1200500FA04F320FA05F001FA04F2E7
:1006480040EA020001F0004110EBD37041F10001D3
:100658005EEA430E08BF20EAD37070BDC4F12005DE
:1006680000FA05F24EEA020E20FA04F301FA05F246
:1006780043EA020321FA04F001F0004121FA04F2EE
:1006880020EA020000EBD3705EEA430E08BF20EABE
:10069800D37070BD94F0000F0FD101F000464000F8
:1006A80041EB010111F4801F08BF013CF7D041EA7A
:1006B800060195F0000F18BF704703F0004652007E
:1006C80043EB030313F4801F08BF013DF7D043EA4F
:1006D8000603704794EA0C0F0CEA135518BF95EA05
:1006E8000C0F0CD050EA410618BF52EA4306D1D18C
:1006F80081EA030101F000414FF0000070BD50EAAB
:10070800410606BF1046194652EA430619D094EA34
:100718000C0F02D150EA013613D195EA0C0F05D11E
:1007280052EA03361CBF104619460AD181EA030172
:1007380001F0004141F0FE4141F470014FF000002A
:1007480070BD41F0FE4141F4780170BD70B54FF0C5
:10075800FF0C4CF4E06C1CEA11541DBF1CEA135545
:1007680094EA0C0F95EA0C0F00F0A7F8A4EB050427
:1007780081EA030E52EA03354FEA013100F088801E
:100788004FEA03334FF0805545EA131343EA1263E7
:100798004FEA022245EA111545EA10654FEA00269C
:1007A8000EF000419D4208BF964244F1FD0404F555
:1007B800407402D25B084FEA3202B61A65EB0305B1
:1007C8005B084FEA32024FF480104FF4002CB6EB6E
:1007D800020E75EB030E22BFB61A754640EA0C00EE
:1007E8005B084FEA3202B6EB020E75EB030E22BF2E
:1007F800B61A754640EA5C005B084FEA3202B6EB6F
:10080800020E75EB030E22BFB61A754640EA9C002D
:100818005B084FEA3202B6EB020E75EB030E22BFFD
:10082800B61A754640EADC0055EA060E18D04FEABB
:10083800051545EA16754FEA06164FEAC30343EA5B
:1008480052734FEAC2025FEA1C1CC0D111F4801F28
:100858000BD141EA00014FF000004FF0004CB6E721
:1008680011F4801F04BF01430020B4F1FD0C88BFC0
:10087800BCF5E06F3FF6AFAEB5EB030C04BFB6EBCB
:10088800020C5FEA500C50F1000041EB045170BDBE
:100898000EF0004E4EEA113114EB5C04C2BFD4EBEB
:1008A8000C0541EA045170BD41F480114FF0000E6F
:1008B800013C90E645EA060E8DE60CEA135594EAEB
:1008C8000C0F08BF95EA0C0F3FF43BAF94EA0C0FEE
:1008D8000AD150EA01347FF434AF95EA0C0F7FF463
:1008E80025AF104619462CE795EA0C0F06D152EAB7
:1008F80003353FF4FDAE1046194622E750EA41069B
:1009080018BF52EA43067FF4C5AE50EA41047FF4AB
:100918000DAF52EA43057FF4EBAE12E74FF0FF3C10
:1009280006E000BF4FF0010C02E000BF4FF0010CE1
:100938004DF804CD4FEA410C7FEA6C5C4FEA430C5A
:1009480018BF7FEA6C5C1BD001B050EA410C0CBFA9
:1009580052EA430C91EA030F02BF90EA020F00200B
:10096800704710F1000F91EA030F58BF994208BF72
:1009780090422CBFD8176FEAE37040F0010070472F
:100988004FEA410C7FEA6C5C02D150EA013C07D186
:100998004FEA430C7FEA6C5CD6D152EA033CD3D0D1
:1009A8005DF8040B704700BF8446104662468C46CB
:1009B8001946634600E000BF01B5FFF7B7FF0028FE
:1009C80048BF10F1000F01BD4DF808EDFFF7F4FF27
:1009D8000CBF012000205DF808FB00BF4DF808EDB2
:1009E800FFF7EAFF34BF012000205DF808FB00BFD5
:1009F8004DF808EDFFF7E0FF94BF012000205DF8F7
:100A080008FB00BF4DF808EDFFF7CEFF94BF0120AB
:100A180000205DF808FB00BF4DF808EDFFF7C4FFA4
:100A280034BF012000205DF808FB00BF4FEA4102F7
:100A380012F5001215D211D56FF47873B3EB625228
:100A480012D94FEAC12343F0004343EA505311F04F
:100A5800004F23FA02F018BF404270474FF00000E1
:100A6800704750EA013005D111F0004008BF6FF01F
:100A7800004070474FF00000704700BF80F0004012
:100A880002E000BF81F0004142001FBF5FEA41035E
:100A980092EA030F7FEA226C7FEA236C6AD04FEA5E
:100AA8001262D2EB1363C1BFD218414048404140A3
:100AB800B8BF5B42192B88BF704710F0004F40F455
:100AC800000020F07F4018BF404211F0004F41F471
:100AD800000121F07F4118BF494292EA030F3FD03D
:100AE800A2F1010241FA03FC10EB0C00C3F1200350
:100AF80001FA03F100F0004302D5494260EB4000DF
:100B0800B0F5000F13D3B0F1807F06D340084FEA49
:100B1800310102F10102FE2A51D2B1F1004F40EB3E
:100B2800C25008BF20F0010040EA030070474900A6
:100B380040EB0000013A28BFB0F5000FEDD2B0FA43
:100B480080FCACF1080CB2EB0C0200FA0CF0AABF66
:100B580000EBC25052421843BCBFD0401843704704
:100B680092F0000F81F4000106BF80F4000001320A
:100B7800013BB5E74FEA41037FEA226C18BF7FEAE1
:100B8800236C21D092EA030F04D092F0000F08BF23
:100B98000846704790EA010F1CBF0020704712F00A
:100BA8007F4F04D1400028BF40F00040704712F149
:100BB80000723CBF00F50000704700F0004343F0AE
:100BC800FE4040F4000070477FEA226216BF0846E4
:100BD8007FEA23630146420206BF5FEA412390EAA7
:100BE800010F40F4800070474FF0000304E000BF9D
:100BF80010F0004348BF40425FEA000C08BF70474E
:100C080043F0964301464FF000001CE050EA010211
:100C180008BF70474FF000030AE000BF50EA010226
:100C280008BF704711F0004302D5404261EB410113
:100C38005FEA010C02BF84460146002043F0B64338
:100C480008BFA3F18053A3F50003BCFA8CF2083A5D
:100C5800A3EBC25310DB01FA02FC634400FA02FC66
:100C6800C2F12002BCF1004F20FA02F243EB02006D
:100C780008BF20F00100704702F1200201FA02FCCF
:100C8800C2F1200250EA4C0021FA02F243EB0200C2
:100C980008BF20EADC7070474FF0FF0C1CEAD05206
:100CA8001EBF1CEAD15392EA0C0F93EA0C0F6FD0C7
:100CB8001A4480EA010C400218BF5FEA41211ED0A5
:100CC8004FF0006343EA501043EA5111A0FB013191
:100CD8000CF00040B1F5000F3EBF490041EAD37166
:100CE8005B0040EA010062F17F02FD2A1DD8B3F1E2
:100CF800004F40EBC25008BF20F00100704790F051
:100D0800000F0CF0004C08BF49024CEA502040EAA2
:100D180051207F3AC2BFD2F1FF0340EAC250704768
:100D280040F400004FF00003013A5DDC12F1190FA6
:100D3800DCBF00F000407047C2F10002410021FA18
:100D480002F1C2F1200200FA02FC5FEA310040F130
:100D5800000053EA4C0308BF20EADC70704792F0A9
:100D6800000F00F0004C02BF400010F4000F013AE1
:100D7800F9D040EA0C0093F0000F01F0004C02BFDC
:100D8800490011F4000F013BF9D041EA0C018FE74B
:100D98000CEAD15392EA0C0F18BF93EA0C0F0AD051
:100DA80030F0004C18BF31F0004CD8D180EA010077
:100DB80000F00040704790F0000F17BF90F0004F10
:100DC800084691F0000F91F0004F14D092EA0C0FF2
:100DD80001D142020FD193EA0C0F03D14B0218BF85
:100DE800084608D180EA010000F0004040F0FE40CB
:100DF80040F40000704740F0FE4040F44000704767
:100E08004FF0FF0C1CEAD0521EBF1CEAD15392EAE5
:100E18000C0F93EA0C0F69D0A2EB030280EA010CD5
:100E280049024FEA402037D04FF0805343EA11116E
:100E380043EA10130CF000408B4238BF5B0042F1CC
:100E48007D024FF4000C8B4224BF5B1A40EA0C0071
:100E5800B3EB510F24BFA3EB510340EA5C00B3EBA3
:100E6800910F24BFA3EB910340EA9C00B3EBD10F91
:100E780024BFA3EBD10340EADC001B0118BF5FEAE3
:100E88001C1CE0D1FD2A3FF650AF8B4240EBC2500C
:100E980008BF20F0010070470CF0004C4CEA5020CD
:100EA8007F32C2BFD2F1FF0340EAC250704740F41C
:100EB80000004FF00003013A37E792F0000F00F00E
:100EC800004C02BF400010F4000F013AF9D040EA8C
:100ED8000C0093F0000F01F0004C02BF490011F420
:100EE800000F013BF9D041EA0C0195E70CEAD15318
:100EF80092EA0C0F08D142027FF47DAF93EA0C0FFF
:100F08007FF470AF084676E793EA0C0F04D14B02E2
:100F18003FF44CAF08466EE730F0004C18BF31F094
:100F2800004CCAD130F000427FF45CAF31F000438E
:100F38007FF43CAF5FE700BF4FEA4002B2F1FE4FDB
:100F48000FD34FF09E03B3EB12620DD94FEA002383
:100F580043F0004310F0004F23FA02F018BF40425C
:100F680070474FF00000704712F1610F01D1420243
:100F780005D110F0004008BF6FF0004070474FF0F7
:100F88000000704742000ED2B2F1FE4F0BD34FF073
:100F98009E03B3EB126209D44FEA002343F00043E7
:100FA80023FA02F070474FF00000704712F1610F0A
:100FB80001D1420202D14FF0FF3070474FF00000DC
:100FC800704700BF53B94AB9002908BF00281CBFA1
:100FD8004FF0FF314FF0FF3000F06AB9ADF1080C67
:100FE8006DE904CE00F006F8DDF804E0DDE902233F
:100FF80004B070472DE9F047089D0C46002B4ED1F0
:1010080094468C458646B2FA82F262D94AB1C2F158
:101018002003914020FA03F30CFA02FC194300FA6A
:1010280002FE4FEA1C471FFA8CF6B1FBF7F44FEAB1
:101038001E4307FB141143EA014304FB06F19942DE
:101048000AD91CEB030304F1FF3080F012819942A6
:1010580040F20F81023C6344591A1FFA8EF3B1FB28
:10106800F7F007FB101143EA014300FB06F69E4226
:101078000AD91CEB030300F1FF3180F0FC809E428B
:1010880040F2F980634402389B1B40EA0440002187
:101098001DB1D3400022C5E90032BDE8F0878B427C
:1010A80005D90DB1C5E9000100210846F5E7B3FAF5
:1010B80083F1002946D1A34202D39042C0F0F080C8
:1010C800861A64EB03030120002DE6D0C5E900630E
:1010D800E3E7002A40F09080A1EB0C044FEA1C489B
:1010E8001FFA8CF70121B4FBF8F64FEA1E4308FB00
:1010F800164443EA044307FB06F0984208D91CEB60
:10110800030306F1FF3402D2984200F2CD8026464E
:101118001C1A1FFA8EF3B4FBF8F008FB104443EADC
:10112800044300FB07F79F4208D91CEB030300F1B7
:10113800FF3402D29F4200F2B0802046DB1B40EA17
:101148000640A5E7C1F120068B4022FA06F71F43A7
:1011580020FA06FC04FA01F343EA0C03F44000FA0F
:1011680001F8380C4FEA1349B4FBF0FE1FFA87FC6C
:1011780000FB1E4449EA04440EFB0CF9A14502FA9F
:1011880001F20AD93C190EF1FF3A80F08480A1459A
:1011980040F28180AEF1020E3C44A4EB09041FFA30
:1011A80083F9B4FBF0F300FB134449EA044403FB5E
:1011B8000CFCA44507D93C1903F1FF3067D2A445BC
:1011C80065D9023B3C4443EA0E40A0FB0293A4EBE2
:1011D8000C049C42CE469C4651D34ED055B1B8EB38
:1011E8000E0364EB0C0404FA06F6CB401E43CC4015
:1011F800C5E90064002150E7C2F1200320FA03F199
:101208000CFA02FC24FA03F394400C434FEA1C48FE
:1012180000FA02FE1FFA8CF7B3FBF8F008FB103156
:10122800230C43EA014300FB07F1994208D91CEB60
:10123800030300F1FF362CD299422AD902386344BD
:101248005B1AA4B2B3FBF8F108FB113344EA034478
:1012580001FB07F3A34208D91CEB040401F1FF3694
:1012680013D2A34211D902396444E41A41EA004175
:1012780039E70446F0E6084606E7C845AED2B9EBBA
:10128800020E63EB070C0138A8E73146EDE7034689
:1012980099E73046D4E7D6467FE7634402384DE7FE
:1012A8000646234608460FE7023E634430E700BF80
:1012B800704700BF1348144A08B54FF00043C0E90F
:1012C80000230422426101220023C2614FF48051AD
:1012D8000722C0E90233C0E90933C0E90C120361EF
:1012E8000383837680F8203080F82C30826380F87E
:1012F8003C30C36401F038FE18B1BDE8084000F086
:1013080035BB08BD24010020002401400268084BB9
:101318009A4282B00AD14FF0B0431A6E42F400727A
:101328001A661B6E03F400730193019B02B07047A9
:10133800002401400268054B9A4201BF4FF0B042B9
:10134800136E23F400731366704700BF0024014036
:1013580030B585B000240546CDE901440394FFF774
:10136800A9FF144802F094F908B100F0FFFA1148F7
:10137800039401A9CDE9015401F054FF08B100F02C
:10138800F5FA0C4802F0AEF808B100F0EFFA4FF0A9
:10139800FF31084801F0E8FE064802F05BF905480D
:1013A80001F03CFF0446034802F0FEF8204605B071
:1013B80030BD00BF24010020014B024A1A6070476B
:1013C800240100200024014008B50948FFF7C0FFA8
:1013D80068B1084BB3F8AA304FF6FF72934216BFB4
:1013E80040F6E442044B5343B3FBF0F398B208BD14
:1013F800002000B40075FF1FD8084C0013B5002367
:10140800ADF80630FFF7E0FF04461948FFF7A0FFE4
:10141800184BB3F8C820B3F8A8108A4204FB00F0B0
:1014280018D040F6E443B0FBF3F364205B1A43435F
:10143800521A93FBF2F31E331BB2ADF80630BDF817
:1014480006305BB21B02ADF80630BDF8060000B2EC
:1014580002B010BD4FF47A7240F6FF73B0FBF3F39D
:101468005343A3F53923A3F50C6340F6C412E0E710
:10147800001000B00075FF1F4FF0B04307B59A6C1D
:1014880042F004029A649A6C02F004020192019AF2
:101498009A6C42F001029A649B6C03F0010300937A
:1014A800002202210F20009B02F090F90F2003B0C8
:1014B8005DF804EB02F0BCB908B502F00DFC10B100
:1014C8006FF0040008BD064B9A6942F040429A61E9
:1014D8004CF2FA321A6102F011FC0028F2D0EFE760
:1014E80000400058F0B585B000230D46009306462D
:1014F800A8B3FFF7E1FF044670BB02F0EDFB88BB21
:101508001A481B4A02230193D0F8E01506F17843E4
:1015180002EA8121B3FBF1F701FB1733DB0A0293DF
:10152800D0F8E00505F178410139314402EA80221A
:10153800B1FBF2F002FB1011C3EBD1230133694672
:1015480001A8039302F05AFC20B1022814BF6FF0DF
:101558000104012402F0D2FB204605B0F0BD6FF073
:101568000504F9E76FF00404F6E700BF0070FF1FF9
:1015780000FCFF03014B1860002070478801002021
:101588002DE9F04FB0F1006F89B006460F4690463E
:10159800C0F0C080DFF89091644DD9F8E03505EAD5
:1015A800832303F10063013B984200F2B3800029D2
:1015B80000F0B38040EA02035B0740F0AE80FFF71B
:1015C8007BFF044690BB02F087FB002840F0A88010
:1015D800D9F8E015009705EA812106F17842B2FBB7
:1015E800F1F301FB132208F17843013B3344B3FBC9
:1015F800F1F001FB1033DB0A01334FEAD22AA3EBE7
:10160800D222012A039388BFC6F30A050AF5803758
:10161800C6F108038CBFC5F500654546FF02B34611
:101628000693039B9A4505D302F068FB204609B050
:10163800BDE8F08FA6F10803069A1A4495421CD813
:10164800009B04950193CDF814B04FF00009059B59
:1016580009EB0301049B99453DD3009BAB442B4404
:10166800A8EB0505B5F5006F009328BF4FF400659A
:101678000AF1010A07F50067D3E753F8081F5A680B
:10168800B2F1FF3F08BFB1F1FF3FD5D0284B186832
:1016980010B96FF00504C7E727B14FF40062394667
:1016A8000DF0EAF9DFF888900099D9F80030CBF30B
:1016B8000A001844AAB20DF0DFF94FF40061384669
:1016C800FFF710FF00BBD9F8003001934FF4006317
:1016D80005970493B9E7019B07914B4402930120B6
:1016E800D3E9002302F044FB88B90799019BD1E9AB
:1016F800000259F80310029B5B689A4208BF8842AF
:1017080005D109F10809A2E76FF001048CE76FF031
:10171800030489E74FF0FF3488E76FF0050485E795
:101728006FF0040482E700BF0070FF1F00FCFF0396
:1017380088010020B1F1006F70B510D30B4BD3F8BE
:10174800E0650B4B03EA862303F10063013B9942F2
:1017580005D838B192B20DF08FF9002070BD4FF066
:10176800FF30FBE76FF00500F8E700BF0070FF1FD0
:1017780000FCFF03B0F1006F10B40DD3084BD3F891
:10178800E045084B03EA842303F10063013B9842D8
:1017980002D810BCFFF7A6BE4FF0FF3010BC704750
:1017A8000070FF1F00FCFF034FF0B04382B0DA6CFB
:1017B8000243DA64DB6C03400193019B02B070477B
:1017C8002DE9F04387B01422002101A80DF080FD17
:1017D8000220FFF7E9FF364F0420FFF7E5FF01205D
:1017E800FFF7E2FF4FF43A410022384602F07AFC54
:1017F80001254FF40A430024CDE9013501A902234C
:1018080038460326CDE903434FF4041902F044FB9C
:1018180001A94FF09040CDE90169039502F03CFB26
:101828004FF4405301A93846CDE901354FF040083F
:10183800CDE9034602F030FB01A91E480395202795
:10184800CDE9018902F028FB01A94FF09040CDE9CC
:101858000175CDE9035602F01FFB01A94FF0904036
:10186800CDE90184CDE9035602F016FB224639463C
:101878004FF0904002F036FC22462146062001F047
:10188800A5FF062001F0D4FF22462146072001F0DB
:101898009DFF072001F0CCFF22462146162001F0CB
:1018A80095FF162001F0C4FF07B0BDE8F08300BF24
:1018B800000400480008004800B59BB048220021F9
:1018C80008A80DF005FD1C22002101A80DF000FD5F
:1018D80002F022FC4FF0B0420120D2F8903023F001
:1018E8001803C2F89030D2F8003423F4C06343F4EC
:1018F8000073C2F80034D2F8003403F4C0630093D4
:10190800009B2423089381230B930023CDE9100324
:10191800B02208A8CDE9122302F076FD08B172B60C
:10192800FEE74F23CDE90130CDE90300059007908C
:10193800022101A803F002F808B172B6FEE71BB055
:101948005DF804FB08B501F0BDFAFFF7B5FFFFF736
:1019580037FF00F0B5FD0022034B114602200CF0C2
:1019680085FF00F0B4FDFCE7B1F4000872B6FEE7AD
:1019780000B58DB02C22002101A80DF0A9FC174854
:10198800174B03601F2383604FF080420023C0E998
:101998000433C0E9072383614FF48073436203F083
:1019A8008DFA08B1FFF7E2FF0C4803F0B3FB08B16A
:1019B800FFF7DCFF4FF00053002207930748089217
:1019C8004FF4807301A9029206920B9303F0D6FAA2
:1019D80008B1FFF7CBFF0DB05DF804FB8C010020C8
:1019E8000028004010B5044690B03822002102A813
:1019F8000DF06EFC2268194B9A422CD14FF48033BB
:101A0800029302A84FF480730F9303F0D5F808B13E
:101A1800FFF7ACFF4FF0B0430220D3F8902042F418
:101A28000042C3F890209A6D42F480629A659B6DDB
:101A3800002203F4806311460193019B01F0C6FE66
:101A4800022001F0F5FE00222A20114601F0BEFE18
:101A58002A2001F0EDFE10B010BD00BF00280040A4
:101A68007047000008B501F043FA044B0120C3F8A1
:101A78008800BDE8084002F0A7BB00BF000400587A
:101A880001F03DBA08B501F03AFABDE8084000F0A7
:101A9800D7BC08B501F02CFABDE8084001210020A8
:101AA80002F042BB70477047FEE7FEE7FEE7FEE73D
:101AB800FEE770477047704770470000014803F021
:101AC8004FBB00BF8C010020012002F019BB02208F
:101AD80002F016BB014802F081B800BFEC010020FB
:101AE800402002F00DBB0000014803F0FBBE00BF20
:101AF8004C020020014803F067B900BF8C010020A8
:101B0800014803F056BD00BFD4010020F0B587B0EE
:101B180000244FF0B0430594DA6C42F00102DA6415
:101B2800DB6C03F00103012500932026032701A99C
:101B38004FF09040009B0395CDE90165049702F0B2
:101B4800ABF9402301A94FF09040CDE90134CDE92C
:101B5800035702F0A1F9224631464FF0904002F0B7
:101B6800C1FA07B0F0BD00000D4B0E4A1B68B3FB6D
:101B7800F2F3DBB258434FF0E023002258619A6138
:101B88001A6942F001021A611A6902F00112012A67
:101B9800FAD01A6922F001021A6100229A6170478C
:101BA8007400002000127A00012238B540214FF05D
:101BB800904002F097FA0120FFF7D6FF202100227B
:101BC8004FF0904002F08EFA40214FF0904002F022
:101BD80083FA0128F8D018240025012220214FF08B
:101BE800904002F07FFA0120FFF7BEFF202100227B
:101BF8004FF0904002F076FA40214FF0904002F00A
:101C08006BFA6D00012804F1FF344FF0010008BFA2
:101C18000135FFF7A9FF14F0FF04DED101222021CE
:101C28004FF0904002F05EFA0120FFF79DFF20215F
:101C380022464FF0904002F055FA85F4000038BD76
:101C480007B5FFF7B1FF064B18601B680093002229
:101C5800044B114602200CF009FE03B05DF804FBAA
:101C6800CC010020E4F4000808B5FFF74FFFFFF7A8
:101C7800E7FF4FF4FA7000F061F9BDE80840FFF79C
:101C8800DFBF00000000000007B5FFF78DFF124B13
:101C98001860124B1A68904215D91B68C01AFEF7D3
:101CA800A7FFFEF7D1FB0AA3D3E90023FEF74EFDF9
:101CB800FEF7BCFE0A4B0022186011460090094B43
:101CC80002200CF0D3FD03B05DF804FBAFF30080F5
:101CD8009A99999999398C40D0010020CC0100201B
:101CE800C80100200BF5000837B5114D0446FFF771
:101CF800CBFF2B68009300220E4B114602200CF0FC
:101D0800B5FD0D4A2B68236013601268D21A642A45
:101D18000BD9642B09DDFFF793FF642000F00EF95F
:101D280003B0BDE83040FFF78BBF03B030BD00BF44
:101D3800C801002029F50008C4010020054808B59D
:101D48000823036003F052FA18B1BDE80840FFF712
:101D58000DBE08BDD40100204FF0B04307B55A6E40
:101D680042F001025A665B6E002203F00103019300
:101D780011463220019B01F029FD322003B05DF8A5
:101D880004EB01F055BD00000CB407B5054A05ABDE
:101D9800102101930DF07AF903B05DF804EB02B05D
:101DA800704700BF3FF5000830B585B0044602A86B
:101DB8000D460CF097FFBDF90C30064A0093102130
:101DC800029B2046FFF7E0FF2046FEF7D1F9288066
:101DD80005B030BD3FF500084FF0B04210B593682C
:101DE80023F4004393600DF005F80F4B01241C7099
:101DF80000F0AAF80CF0D0FC0C480CF0E7FC0C4BF7
:101E08004FF400421A6102200CF0E6FCFFF7D4FA06
:101E180000F000F9FFF728FF0CF0D8FD2146204616
:101E2800BDE810400CF0F2BDE0010020B11D000833
:101E3800004000580CF000BE08B5FFF7C5FA40F6A0
:101E4800B83398420CD8B0F5E16F0BD3FE23A0F558
:101E5800E16058434FF49663B0FBF3F0C0B208BD9D
:101E6800FE20FCE70020FAE77FB5684600F0B6F8E8
:101E78000198FFF761F800B207B05DF804FB0000B5
:101E8800194A38B5D2F88035591C044619D101F0E1
:101E98003DF8054601F046F8054401F03DF82B0EE3
:101EA800E3712B0CA3712B0A6371030EE370C0F36B
:101EB8000742C0F307232571C0B2A2706370207077
:101EC80038BD190AC3718171190C1B0E4171037158
:101ED800D2F88435C370D2F88405C0F30722C0F362
:101EE8000743000EE9E700BF0070FF1F38B5094B34
:101EF800D3F8803503600133054609D101F006F8AF
:101F0800044601F009F8444001F00CF844402C6004
:101F180038BD00BF0070FF1F012102200CF060BD1A
:101F2800002102200CF05CBD00207047024B18789D
:101F380008B100F0A7B87047E001002082B0019016
:101F4800019802B000F03AB9F0B5224A224CD2F812
:101F5800903043F4804389B0C2F8903000F0E8FF35
:101F680000F0EEFF00F0F4FF01230493032306932F
:101F780000254FF0B04305950795DA6C42F0020250
:101F8800DA64DA6C02F002020292029ADA6C42F027
:101F98000202DA64DB6C03F0020301934FF480570A
:101FA80003A92046019B03974FF4005601F074FFE4
:101FB80003A92046039601F06FFF2A4639462046BA
:101FC80002F090F82A463146204602F08BF809B014
:101FD800F0BD00BF000800580004004810B50446D2
:101FE800FFF70CFA074BA36040F30F20FEF700FE43
:101FF800054B064A2360064B6060C4E903230020B2
:1020080010BD00BF0000484200007A440D093E00A0
:10201800AB03050000207047014B1868704700BFEC
:10202800E40100200320704708B501464FF47A7296
:1020380000238002890DFEF7C5FF08BD4FF47A73AF
:10204800A0FB0303800A40EA83507047034B98685B
:102058009A689042FBD1C043704700BF00280040F7
:1020680008B5FFF7F3FF014B186008BDE401002035
:1020780008B5FFF7EBFF024B1B68C01A08BD00BF8D
:10208800E4010020024B187808B1FFF7DFBF704762
:10209800E801002010B5074B074C0122DA654FF420
:1020A8008071204602F056FE4FF0FF332363002074
:1020B80010BD00BF002800408C010020024600210E
:1020C800014803F05EB800BF8C01002002460121E0
:1020D800014803F056B800BF8C01002010B58CB041
:1020E8002C220021044601A80DF0F2F8FFF7D2FFD8
:1020F8000C4B0D481B681C440023089306934FF0B3
:102108000053E443079301224FF4807301A902941A
:102118000B9302F033FF08B1FFF728FC00200CB046
:1021280010BD00BFE40100208C01002038B5054631
:10213800FFF78CFF02210446074803F029F8C4F38F
:1021480009024FF47A71A2FB0121920AA30A2A809C
:1021580043EA805038BD00BF8C01002001480021AF
:1021680003F016B88C0100200148012103F010B8D3
:102178008C010020F8B50F4D2E78CEB90E4C4FF0DB
:10218800FF372763FFF7F4FBFFF784FF4FF48071F5
:10219800204602F0DFFD2046276302F09DFF32460D
:1021A8002046022102F0EDFFFFF75AFF01232B70B2
:1021B8000020F8BDE80100208C010020014610B580
:1021C8004FF47A7200238002890DFEF7FBFE014668
:1021D800FFF73CFF0446FFF739FF031B8B4200D390
:1021E80010BD00BFF7E70CF00DBF000010B5064C9E
:1021F8000221204602F0CCFF0221421C2046BDE805
:10220800104002F0BEBF00BF8C0100201648174ADC
:1022180008B54FF4E133C0E9002300230C22C0E9DC
:102228000233C0E90523C0E90733C0E90933036174
:1022380004F03DF908B1FFF799FB0B48002104F0C1
:10224800AEFA08B1FFF792FB0748002104F0C7FA7D
:1022580008B1FFF78BFB044804F081FA18B1BDE818
:102268000840FFF783BB08BD4C0200200044004033
:1022780070B596B006461422002103A80DF028F880
:102288003822002108A80DF023F832682B4B9A4217
:1022980051D10223089308A8294B0A9302F08CFC19
:1022A80008B1FFF763FB4FF0B04300259A6D254C4A
:1022B80042F400329A659A6D02F400320292029A50
:1022C800DA6C42F00102DA64DB6C03F0010301937B
:1022D800019B0C220223CDE903230323CDE90553F7
:1022E80003A907234FF09040079301F0D5FD164945
:1022F80025621423C4E900131023C4E902352046DB
:102308008023C4E90435C4E9065501F0F1FA08B19F
:10231800FFF72CFB0B48102101F0B6FC08B1FFF7C2
:1023280025FB2520F46700220221A66201F04EFA5F
:10233800252001F07DFA16B070BD00BF00440040B2
:1023480004000C00EC0100205800024002680C4B0D
:102358009A4210B5044612D14FF0B0420C21936D49
:1023680023F4003393654FF0904001F041FEE06F95
:1023780001F030FBBDE81040252001F067BA10BD20
:102388000044004008B50A460146024803F00EFA28
:10239800002008BD4C02002013B5114B114C1860E9
:1023A8004FF40013009302AB13E90600204604F033
:1023B8007AF92368DA69D103FCD4DA695202FCD5C8
:1023C8009A68084842F480029A6004F0B2F9064913
:1023D8000448012204F020F9002002B010BD00BF1B
:1023E800E00200204C020020E802002008B5074B5C
:1023F8001860FFF741F8FFF709FF054AD2F8803067
:1024080043F00063C2F88030002008BDE4020020D9
:102418000008005808B54FF0B04308489A6B42F4DA
:1024280000329A639A6B22F400329A63FFF78EFFA8
:102438000F2001F00BFA002008BD00BF4C0200205D
:1024480008B5074804F033F808B1FFF78FFA0548D4
:1024580001F04EFA18B1BDE80840FFF787BA08BD89
:102468004C020020EC0100200268044B9A4203D180
:10247800034B00201B681847704700BF004400400A
:10248800E402002002680B4B9A4210B504460FD1B3
:10249800094B1B682BB1D0F8902012B907480121CD
:1024A800984720460549BDE81040012204F0B4B819
:1024B80010BD00BF00440040E0020020E8020020F8
:1024C80008B5FFF789FCBDE8084000F057BB4FF09E
:1024D800FF300CF015BB7047014BD870704700BF38
:1024E8000C000020014B1874704700BF0C0000203E
:1024F80007B5064B00221B5C00931146044B0220D3
:102508000CF0B4F903B05DF804FB00BFB2F50008A5
:1025180098F5000808B5022000210CF0B9FABDE8CA
:10252800084001480CF01CBD400400200021012097
:102538000CF0AEBA10B542F21073084C002818BF60
:102548000346074823600CF0BDFC216804480CF0E2
:1025580041FDBDE8104002480CF002BD0800002013
:102568004004002037B5044638B390F9065035BB0F
:1025780014480CF0A7FC14482A464FF4006101F0F7
:10258800B1FD124B2A46294602200CF06FF9E37977
:10259800012B0CBF0E4B0F4B0022114602200CF0F2
:1025A80065F994F90530019394F9043000930022F9
:1025B800094B114603200CF059F903B030BD074B05
:1025C800EAE700BFEC02002000040048B6F5000866
:1025D800CBF50008E8F500081EF6000805F6000827
:1025E80008B50E4B1B78022B03D1002108200CF0F4
:1025F8004FFA0B4800224FF4004101F073FD0848E0
:1026080000224FF4007101F06DFDBDE80840044858
:1026180000224FF4006101F065BD00BF700000208A
:1026280000040048024800224FF4004101F05ABD5E
:1026380000040048024800224FF4007101F052BD26
:10264800000400480A460149FFF774B800F003087F
:1026580070B51F4801224FF4004101F043FD1C48AA
:1026680001224FF4007101F03DFD01224FF4006199
:10267800174801F037FD17480CF024FC04F010FD52
:10268800044650B10022144B114602200CF0EEF81B
:10269800BDE8704011480CF063BC114D114B024667
:1026A800014602200CF0E2F801260F4B2E7022465C
:1026B800214602200CF0DAF80C4804F085FB287853
:1026C800314604F0D9F803480CF04AFCE0E700BFB3
:1026D800000400484004002047F6000828040020B1
:1026E8007000002065F6000879F600080C0000204C
:1026F8002DE9F04391B0FFF79FFB044604F0B6F9CB
:10270800054600287CD103A8FFF768FC09A8FFF755
:10271800EBFA099B00930122594B294602200CF041
:10272800A5F8584B00940122294602200CF09EF887
:102738000498554CFEF700FC00B20122534B009060
:10274800294602200CF092F802230598237050497C
:10275800FEF7A2FAFEF716FC86B20498FEF7ECFB29
:102768004C4907B20398FEF797FA4949FEF748FB28
:10277800FEF708FC484A636812781A706368C0F369
:1027880007225A70636898706368DF706368320A5A
:102798001A7163685E71414E3378082B01D0012BA2
:1027A80040D86268002393716268D37162681372BB
:1027B80053720A23099A6168120ACA54626809990D
:1027C8001A44023351706370354C637A63B104F074
:1027D80039F9012808D120460CF074FB3148002251
:1027E8004FF4006101F07EFCF1782748002204F0E4
:1027F80053F9014688BB01222B4B10460CF036F8E2
:1028080000242A480CF05EFB294B28481968A1428D
:1028180038BF21460CF0DEFB24480CF0A1FB11B0B8
:10282800BDE8F083DDE90687D4F80490FFF704FBE0
:1028380089F8060063684FEA2842DA7163684FEA4C
:1028480028221A723A149A723A1283F80980DA72B4
:102858001F735D739D730F23ACE70631D0D104F06D
:10286800EBF804460028CBD001224FF47A730021FC
:10287800B0FBF3F3104600930E4B0BF0F7FFC0E7E5
:1028880098F60008ABF6000800000020B6F600082D
:10289800000020410000C842340300200C00002042
:1028A800EC02002000040048C1F6000840040020A3
:1028B80008000020D0F6000802484FF4006101F03B
:1028C80016BC00BF0004004800B503468DB00028C0
:1028D8002CD0407802280AD003282AD0164B002290
:1028E800114602200DB05DF804EB0BF0BFBF1A7F54
:1028F8000B92DA7E0A929A7E09925A7E08921A7E82
:102908000792DA7D06929A7D05925A680492DA68EF
:10291800039293F914200292B3F9122001921B7CBE
:1029280000930022054B11460BF0A0FF0DB05DF897
:1029380004FB034BD3E700BFEEF6000805F70008D9
:1029480077F7000801284FF000020CBF024B034B39
:10295800114602200BF08ABF96F70008A8F7000876
:1029680008B504F0A6FB80B904F06CF801280CD176
:10297800BFF34F8F0549064BCA6802F4E062134360
:10298800CB60BFF34F8F00BFFDE708BD00ED00E04F
:102998000400FA051FB50446002837D00378002B39
:1029A80034D001224FF400711E4801F09BFB1E48F1
:1029B8000CF0D6FA002211461C4B02200BF056FFF1
:1029C80094F91830039394F90A300293237C019305
:1029D800E368009300221146154B03200BF046FFD5
:1029E8000022144B114603200BF040FF237A012BE1
:1029F8000ED1617A104A114B002918BF13460022E4
:102A0800009311460E4B03200BF030FF04B010BDAD
:102A180000220C4B1146032004B0BDE810400BF017
:102A280025BF00BF000400481C030020C1F70008B0
:102A3800F2F7000823F80008BDF70008BCF7000803
:102A480030F8000841F80008F0B5054687B00C4694
:102A5800002937D02C4801224FF4004101F042FBF5
:102A68002A480CF07DFA26789EB1002D4AD06B6872
:102A78002E7873B1022E27D0032E0AD16A78012A44
:102A880007D11878012802D0022800D008B904F02C
:102A9800CDF8237C052B15D894F90A20059294F9D2
:102AA800092004921A4A52F82330039394F9083003
:102AB800CDE901630022E36800931146154B03201A
:102AC8000BF0D4FE07B0F0BD6F78012FE1D11D786F
:102AD800114B05F001051D7065B92A460F4B2946B3
:102AE80003200BF0C3FE2A4607484FF4006101F0AB
:102AF800F9FACEE700221146094B03200BF0B6FE87
:102B08003A46F1E72E46C4E70004004804030020D3
:102B180090F9000862F80008340300204FF8000814
:102B280059F8000838B504460D4607484FF40061C7
:102B3800FEF720FE30B92A4621460348BDE8384052
:102B4800FEF71EBD38BD00BF00F0030810B504F045
:102B580045FB10F1080F07D1064B0022BDE81040D5
:102B6800114602200BF082BE013001D1024BF4E77E
:102B780010BD00BFA9F80008BFF80008F0B587B07D
:102B88000024012603274F4B029422462146CDE913
:102B980000670220022505940BF068FE0523CDE9A5
:102BA80000532246484B0294214628460BF05EFE0D
:102BB800464B009622462146CDE9017428460BF083
:102BC80055FE05A9204604F059FA059BC3F30722D0
:102BD8000292C3F307421B0E0192009322463C4B1C
:102BE800214628460BF042FE05A9304604F046FA75
:102BF800059BDAB20392C3F307220292C3F307429A
:102C08001B0E019200932246324B214628460BF0B8
:102C18002DFE314B3148009422464FF4FA710CF0E6
:102C2800F3F82F4B2F48009422464FF4FA710CF01A
:102C3800EBF82D4B2D48009432464FF4FA710CF006
:102C4800E3F82046FEF796FC08B1FEF78FFE284B06
:102C5800009400224FF4FA6126480CF0D5F8264A71
:102C6800002101200BF0D0FF244A002102200BF0A4
:102C7800CBFF234A002104200BF0C6FF214A002184
:102C880008200BF0C1FF00F059F81F491F4804F055
:102C9800ABF91F4804F098F814480CF061F91D4B83
:102CA8000021187803F0E8FD1B4900941B4B0968C4
:102CB8001B4800220CF0A8F819480CF051F907B08D
:102CC800F0BD00BFD7F80008F8F8000819F90008A7
:102CD8003AF900085BF900083D2600081C030020AB
:102CE8002D26000804030020C1280008EC0200205B
:102CF800E925000828040020D56B0008F9260008FB
:102D0800552B000859260008000003012400002064
:102D18000C00002070000020080000201D2500087D
:102D280040040020022804D0402806D100210420B5
:102D380001E0002108200BF0ABBE7047034B0022D6
:102D4800C3E902220122C3E9002270475804002087
:102D5800004870475804002000F034B800F072B8FA
:102D680000F0A4B800F0A4B800F0A4B800F0A4B82B
:102D78000D48854600F0A5F80C480D490D4A00237A
:102D880002E0D458C4500433C4188C42F9D30A4A18
:102D98000A4C002301E013600432A242FBD30CF07A
:102DA8009FFAFEF7CFFDFEE700800020000000201C
:102DB80008010020A0030108080100204016002097
:102DC800FEE700002DE9F04186B000244FF0B04343
:102DD8000594DA6C1A4D42F00402DA64DB6C039451
:102DE80003F004030093009B10270123CDE901732E
:102DF80001A90323284604934FF0200801F04CF85A
:102E080001A928460826CDF8048001F045F801A953
:102E18002846019601F040F822464146284601F02E
:102E280061F922463946284601F05CF928462246CF
:102E3800314601F057F9204606B0BDE8F08100BFE1
:102E48000008004808B5032812D8DFE800F002138C
:102E58001A2600221448082101F044F900221248D9
:102E6800102101F03FF900220F48202101F03AF922
:102E7800002008BD01220C48082101F033F9012285
:102E8800EDE701220848082101F02CF90122064843
:102E9800102101F027F90122E6E701220248082162
:102EA80001F020F90022F2E70008004800207047EE
:102EB8000120704701207047002814BF16200F20FA
:102EC8007047704710B5032000F06EFC01F08CFAD3
:102ED800064B18600F20FFF727F8044618B9FEF7CD
:102EE800E2FD204610BD0124FBE700BF740000206E
:102EF8004FF0E022136923F00203136170474FF08B
:102F0800E022136943F0020313617047014BD3F8C1
:102F1800900570470070FF1F014BD3F89405704768
:102F28000070FF1F014BD3F8980570470070FF1F12
:102F3800024A536843F0010353607047002004E0DD
:102F4800024A536843F0020353607047002004E0CC
:102F5800024A536843F0040353607047002004E0BA
:102F68008068C0F380007047F7B5002301930446DA
:102F7800002800F0E980856D25B9FEF7C7F9E565F9
:102F880084F8545023689A68D00040F1A1809A6868
:102F9800D10000F1B480A26D42F01002A265E26D8A
:102FA80042F00102E26501251846FFF7D9FFA26D3C
:102FB80002F01002024340F0C980A26D206922F499
:102FC800817242F00202A2659A68D2075DD4226B30
:102FD800A67E94F82CC0003A18BF01221703D4E942
:102FE80002120A43217E42EA8132617E42EAC132FC
:102FF80042EA4632002842EA4C02B4BF20F00041BF
:103008004FF400113A430A4394F82010012903D1E0
:10301800002E76D142F48032616A21B1A66A01F4A9
:10302800E07131430A43D968E66C21F4FE3121F49A
:10303800FF711143D96094F83C206168012A01F0BE
:10304800404C4CEA060609D1D4E910273A433243EA
:10305800A66C324342EA0C0242F001061F693E4A5E
:103068003A4032431A6121F00042B2F1804F0CD04D
:10307800B1F1004F09D0394ED6F8082701F4701184
:1030880022F470120A43C6F808275A69666BA16BC6
:1030980022F0070232435A615A6922F0700242EA6A
:1030A80001125A61002835D19A6A62F00F029A62B9
:1030B8005B6903F007039E423CD10023E365A36DDF
:1030C80023F0030343F00103A365284603B0F0BDD2
:1030D8009A68234922F0104222F0170242F08052E7
:1030E8009A60204A1268B2FBF1F201325200019252
:1030F800019A002A3FF44BAF019A013AF7E70025FD
:1031080052E7A16D41F02001A165E16D41F0010197
:10311800E16581E7B0F5001FCAD19A6AE269013A10
:1031280092006FF00F0102F01C0201FA02F2216E08
:103138000A43BCE7A36D23F0120343F01003A36511
:10314800E36D43F00103E3650125BEE7A36D43F09A
:103158001003A365F8E700BF02FCFF1F0020014031
:10316800400D030074000020F8B54569082D044699
:103178000E460AD00368DB68D80705D5A36D43F06F
:103188002003A3650120F8BD0425FEF7CFFE0746FE
:1031980023681A682A4220D0A26D42F40072A26500
:1031A800DA6812F4406F14D1A27E92B91A68120735
:1031B8000FD51846FFF7D4FE20BB5A6822F00C0240
:1031C8005A60A26D22F4807222F0010242F00102DC
:1031D800A265227EFAB10020D5E7711CD9D0FEF78E
:1031E800A5FEC01BB04201D8002ED1D123681B68B0
:1031F8002B40CDD1A26D84F8543042F00402A26570
:103208000320C0E7A26D42F02002A265E26D42F001
:103218000102E265DDE70C221A60DCE70368186C3E
:1032280070470000F7B50023019390F85430012B44
:10323800044600F0C08005680269012380F8543014
:103248002846FFF78DFE002840F0AF80D1E9003016
:10325800022822F004027ED0B2F1004FC3F3110E0F
:1032680035D1AA6A42EA0E02AA628A68686902EA45
:10327800032222F07C4222F0FF0220EA03210A43C3
:10328800002B6A611DDA4D4A4D4DD2F80817AB4242
:1032980001F0E07043D10D0213D4D2F8083723F0BF
:1032A800E073034343F40003C2F80837454B1A6838
:1032B800454BB2FBF3F20C2302FB03330193019B52
:1032C80053BB0020002384F8543003B0F0BD226EB5
:1032D80000F01F074FF00F0C0CFA07FC6FEA0C0602
:1032E80022EA0C0CBEF1000F11D1C3F38462BA407C
:1032F80042EA0C0222668008E26901309042B4D8A2
:10330800A86AC3F38362BA4006403243ACE793FA33
:10331800A3F2B2FA82F2EAE7019B013BCEE72B4D1A
:10332800AB420BD1C901CCD4D2F8083723F0E073F3
:10333800034343F08073C2F80837C2E7244DAB4219
:10334800BFD14B02BDD4D2F8083723F0E073034352
:1033580043F48003EFE7B2F1004F01BFAA6AC3F359
:1033680011018A43AA62002BABDA1548134983423C
:10337800D1F8082709D1D1F8083702F0A07223F054
:10338800E0731A43C1F808279BE71048834204D129
:10339800D1F8083702F44002F1E70D48834290D192
:1033A800D1F8083702F0C072E9E7A26D42F02002B6
:1033B800A265184686E7022087E700BF0020014083
:1033C800001000B074000020400D0300004000B859
:1033D800002000B4026838B504461046FFF7C0FD67
:1033E80008B9002038BD9368990707D4936823F07B
:1033F800004323F0170343F010039360FEF796FD94
:10340800054623689B685B07EBD5FEF78FFD401BDD
:103418000228F6D923689B685A07F2D5A36D43F0B2
:103428001003A365E36D43F00103E3650120D9E7C9
:1034380073B50023026801939368DD07044602D53B
:10344800002002B070BD9168214B194209D0A36DCC
:1034580043F01003A365E36D43F00103E365012026
:10346800EFE7936823F0004323F0170343F00103C9
:103478009360184BD3F8083718021CD4637E012BCD
:10348800DED0FEF753FD144E054622681368DB07AD
:10349800D6D49368D9075FBF9368334043F00103DC
:1034A8009360FEF743FD401B0228EED923681B6892
:1034B800DA07EAD4CBE7094B094A1B68B3FBF2F3F6
:1034C80001330193019B002BD8D0019B013BF8E706
:1034D8001700008000200140E8FFFF7F74000020F3
:1034E800400D030038B504460068FFF739FD05466E
:1034F80020BB94F85430012B20D0012384F8543099
:103508002046FFF795FFB0B9A36D226823F47063D6
:1035180023F0010343F48073A3651C23E065136063
:1035280084F85400936823F0004323F0170343F012
:103538000403936038BD84F85450FBE70220F9E790
:10354800026838B5936891680446C80701D400201A
:1035580038BD9907FBD4936803F00503012B19D1F3
:10356800936823F0004323F0170343F002039360AA
:1035780003231360FEF7DAFC054623689B68DB0724
:10358800E5D5FEF7D3FC401B0228F6D923689B68D3
:10359800DA07F2D5A36D43F01003A365E36D43F09A
:1035A8000103E3650120D3E770B5044600284BD03A
:1035B800836D43F002038365FFF70CFF054668B986
:1035C8002046FFF7BDFF054608B90123A365226819
:1035D800936823F0104323F01703936023685A6815
:1035E80022F4677222F003025A6040F29F321A6096
:1035F800D968164A0A40DA601A6922F040421A610C
:103608005A6922F007025A611A6A02F0F0221A6215
:103618005A6A02F0F0225A62DA6A02F0F022DA629A
:103628009A6A0B4A00269E62D2F8083723F0FE7386
:10363800C2F808372046FDF77DFEE6652666A665D2
:1036480084F85460284670BD0125FBE700023E83DC
:103658000020014010B590F85430012B044615D0D5
:10366800012380F85430FFF7B5FE58B92046FFF71C
:1036780067FF38B9A36D23F4807323F0010343F087
:103688000103A365002384F8543010BD0220FCE731
:10369800F7B50023019390F85430012B04467FD0EE
:1036A800012380F85430FFF74BFF23689A6812F023
:1036B8000102054607D0A36D43F01003A36500235C
:1036C80084F854302DE0A16D364F21F4817141F01A
:1036D8000201A165DE68D96826F4FF4626F07C065B
:1036E80021F40041360421F00301360CD96008208A
:1036F8009968394041F0004199609968002913DAC6
:103708000199013101910199B1F52E3FF5D3A36DCE
:1037180023F0120343F01003A365002384F8543008
:103728000125284603B0F0BDD3F8B410013801F0E4
:103738007F010A44DCD199681A48014041F001012F
:103748009960D3F8B41021F07F0141EAD202C3F89E
:10375800B4209A68024042F002029A60FEF7E6FB43
:10376800074623689A68D20708D4DA683243DA60D1
:10377800A36D23F0030343F001039FE7FEF7D6FB95
:10378800C01B0228EDD923689B68D907E9D5A36D2A
:1037980043F01003A365E36D43F00103E365BFE75E
:1037A8000225BEE7E8FFFF7F0749CA6822F4E06206
:1037B8000302120403F4E063120C134343F0BF63E3
:1037C80043F40033CB60704700ED00E0164B30B592
:1037D800DC68C4F30224C4F10703251D042B28BFA9
:1037E8000423062D4FF0FF358CBF033C002405FA57
:1037F80003F321EA0303A54022EA0502A3400028B7
:1038080043EA0203ACBF00F16040084A4FEA0313E1
:10381800B8BF00F00F00DBB2AABF00F56140135437
:1038280080F8003330BD00BF00ED00E014ED00E08B
:10383800002807DB044A4109012300F01F008340E8
:1038480042F82130704700BF00E100E000280CDB9F
:103858004309064900F01F0020330122824041F845
:103868002320BFF34F8FBFF36F8F704700E100E055
:1038780070B5D0E913456560446D14B1D0E91645BB
:103888006560D0E9105404F01C060124B4406C6053
:10389800046863608368102B0BBFA260A160E160BD
:1038A800E26070BD0268416CD3B210B5083B1424C5
:1038B800B3FBF4F30B4CA24288BF0B4A21F003017F
:1038C80099BF01F1804202F502325218073382642F
:1038D800064AC26403F01F03012202FA03F30365D8
:1038E80010BD00BF070402401C08024080080240C7
:1038F80038B500285CD002682E4B9A424FF014016C
:103908004AD82D4B1344B3FBF1F32C499B00C0E973
:103918001013022380F825301368056923F4FF4348
:1039280023F070031360D0E9024323432B43456916
:1039380011682B4385692B43C5692B43056A2B43C3
:103948000B431360FFF7AEFFB4F5804F04BF0023AD
:1039580043604368816C03F07F020A60D0E9131466
:10396800013B032B4C601ED8154B16498165134447
:103978009B000121013A01FA02F200214365C26568
:103988001960114B5A6400230122C36380F8243064
:1039980080F82520184638BD0C4B1344B3FBF1F3CF
:1039A8000B499B00B3E70023C0E91533C365EAE779
:1039B8000120F0E707040240F8FFFDBF00000240C5
:1039C8003F8200104009024000090240F8FBFDBF99
:1039D8000004024038B5002841D00268136823F07B
:1039E800010313601F4B9A424FF0140130D81E4B4D
:1039F8001344B3FBF1F31D499B00C0E910130124E4
:103A080003F01C0304FA03F3002515604B60FFF76D
:103A180049FF836C41681D60D0E913325A604A1E21
:103A2800032A06D8124B0B449B0094401D60114B8F
:103A38005C640023C363C0E91533C0E90B33C0E9F4
:103A48000D33C36580F8253080F82430184638BD1A
:103A5800094B1344B3FBF1F308499B00CDE7012060
:103A6800F5E700BF07040240F8FFFDBF0000024071
:103A78003F82001000090240F8FBFDBF000402402D
:103A880070B590F82450012D04463BD090F825607D
:103A98000125AE4280F824504FF000062CD10225B3
:103AA80080F825500568C6632E6826F001062E604A
:103AB800FFF7DEFE036BBBB12B6843F00E032B60F0
:103AC800A36C1A68D20342BF1A6842F480721A6063
:103AD800636D1BB11A6842F480721A602B6843F058
:103AE80001032B60002070BD2B6823F004032B60BA
:103AF8002B6843F00A03E2E78023C36380F824605D
:103B08002846F0E70220EEE7034640B190F825206A
:103B1800022A06D00422C263002280F82420012051
:103B280070470268806C116821F00E01116001680D
:103B380021F480710160116821F001011160D3E95D
:103B4800100202F01C0101228A404260D3E91321CD
:103B580051605A6D32B1116821F480711160D3E956
:103B6800162151600122002083F8252083F82400C3
:103B7800704708B590F82530022B03D00423C3639F
:103B8800012008BD03681A6822F00E021A601A683C
:103B980022F001021A60826C136823F480731360A8
:103BA800D0E9101303F01C02012393404B60D0E9C5
:103BB80013325A60436D33B11A6822F480721A6066
:103BC800D0E916325A60012380F82530002380F8A6
:103BD8002430836B03B198470020D2E770B4426C5D
:103BE800046C036826681D6802F01C0204219140D9
:103BF80031420FD015F0040F0CD01A6892065EBF40
:103C08001A6822F004021A60036B6160002B33D03B
:103C180070BC184702219140314217D015F0020FAD
:103C280014D01A68940606D41A6822F00A021A6098
:103C3800012280F82520114A93428CBF104B114B6A
:103C48005960002380F82430C36ADFE708219140D7
:103C5800314211D029070FD5196821F00E011960DA
:103C6800012303FA02F26260C36380F8253000235F
:103C780080F82430436BC9E770BC7047800002406D
:103C8800000402400000024060B10268C8061368E0
:103C980005D5C9024CBF43F4801323F48013136085
:103CA80000207047012070470A4A536943F4802373
:103CB80030B55361EFF3108472B60023CD58C55068
:103CC8000433B3F5807FF9D11369DB03FCD484F3A3
:103CD800108830BD00400058064B5A69002ABFBF03
:103CE800054A9A6002F188329A60BABF5869C00FD3
:103CF800002070470040005823016745044B5A696B
:103D080042F000425A615869C043C00F704700BF73
:103D18000040005870B50546FEF708F9124E0446F3
:103D28003369D90313D43369DA0744BF01223261F6
:103D38004CF2FA32134011D10B4E306910F4802046
:103D48000BD0FEF7F3F8001BA842F6D304E0FEF709
:103D5800EDF8001BA842E3D3032070BD024A1361AB
:103D6800024A01205360F8E7004000586804002028
:103D78002DE9F041184D98462B78012B06460C4644
:103D8800174626D001232B704FF47A7000236B60FE
:103D9800FFF7C0FFA0B9012E16D1104A536943F0AE
:103DA800010353612760BFF36F8FC4F804804FF499
:103DB8007A70FFF7AFFF094A536923EA0603536194
:103DC80000232B70BDE8F08139462046FFF76CFFD1
:103DD800EDE70220F6E700BF680400200040005825
:103DE800054A536923F47E7343EAC00040F48030E7
:103DF80040F0020050617047004000582DE9F04142
:103E0800234F3B78012B054688463FD001233B7062
:103E18004FF47A7000237B60FFF77CFF044688B973
:103E28002B68042B13D11B4A536943F4803343F0A6
:103E3800040353614FF47A70FFF76CFF0446154B87
:103E48001A681B6800233B702046BDE8F0814FF0DC
:103E5800FF33C8F800306E68D5E901321344B34225
:103E68000AD93046FFF7BCFF4FF47A70FFF752FFCC
:103E780050B1C8F800600446064A536923F47E73BB
:103E880023F002035361DAE70136E5E70224DBE7B2
:103E980068040020004000582DE9F04F524C0023E0
:103EA8004FF00F090A6832FA03F501D1BDE8F08F27
:103EB800012505FA03F818EA020200F08E804E6820
:103EC800032706F003054FEA430E07FA0EFC6F1EA0
:103ED800012F6FEA0C0C32D8876807EA0C0ACF6802
:103EE80007FA0EF747EA0A078760476827EA0808CB
:103EF800C6F300179F4047EA08074760C76807EA04
:103F08000C088F6807FA0EF747EA0807022DC76002
:103F180017D14FEAD30800EB880803F0070AD8F84E
:103F280020704FEA8A0A09FA0AFB27EA0B0B0F6985
:103F380007FA0AF747EA0B07C8F8207001E0032DD3
:103F4800DCD1076805FA0EF507EA0C073D4316F4BD
:103F5800403F056041D023F0030707F1804707F58C
:103F6800803703F0030CBD684FEA8C0C4FF0070E46
:103F78000EFA0CFEB0F1904F25EA0E0E2FD01B4D15
:103F8800A8422ED005F58065A84214BF0725022552
:103F980005FA0CF545EA0E05BD602568D74316F409
:103FA800801F0CBF3D4015432560656816F4001F4F
:103FB8000CBF3D4015436560D4F8805016F4803F2F
:103FC8000CBF3D401543C4F88050D4F88450B60364
:103FD80054BF3D401543C4F88450013362E70025BF
:103FE800D6E70125D4E700BF0008005800040048C0
:103FF800374A2DE9F04F00234FF0010A4FF0070B25
:104008004FF00F0931FA03F401D1BDE8F08F0AFA35
:1040180003FC1CEA010654D023F0030404F1804495
:1040280004F5803403F00307A568BF000BFA07F80E
:10403800B0F1904F08EA050E45D0264DA84244D06D
:1040480005F58065A8420CBF02250725BD407545CA
:1040580017D1D2F8805025EA0605C2F88050D2F868
:10406800845025EA0605C2F88450156825EA060535
:104078001560556825EA06055560A56825EA08050E
:10408800A560056803265C0006FA04F423FA06F620
:10409800254300EB8606056003F00705376AAD0087
:1040A80009FA05F527EA05073762856825EA040550
:1040B8008560456825EA0C054560C56825EA04045D
:1040C800C46001339EE70025C0E70125BEE700BFB5
:1040D80000080058000400480369194214BF012071
:1040E800002070470AB18161704781627047436957
:1040F80001EA030221EA030141EA024181617047B2
:10410800044AD168014208B502D0D060FEF70AFE21
:1041180008BD00BF00080058024A136843F48073C2
:1041280013607047000400580D4B10B55B690C46CE
:1041380028B99A0507D500F027F820B110BD9B05CE
:1041480001D400F019F8074A1369012C23F004037D
:10415800136101D130BFF1E740BF20BF20BFEDE7B9
:104168000004005800ED00E0024B186800F4C0603D
:10417800704700BF00040058024A136843F48043A4
:1041880013607047000400580C4A136823F48043F6
:1041980013600B4B1B6832214B430A49B3FBF1F305
:1041A8005169890500D533B9536913F4007F14BFE9
:1041B800032000207047013BF2E700BF00040058CD
:1041C8007400002040420F000B4A136823F00703D5
:1041D80043F002031360094B1A69012842F00402F4
:1041E8001A6105D130BF1A6922F004021A617047BA
:1041F80040BF20BF20BFF6E70004005800ED00E0F4
:104208004FF0B0431868C0F3404070474FF0B043D8
:104218001868C0F3400070474FF0B042536823F469
:104228007F4343EA0023536070474FF0B043186858
:10423800C0F34060704700007FB54FF0B0432C4A90
:10424800D3F80831C0F3031003F00F0352F82040ED
:10425800284A52F82330B4FBF3F4FFF785FF264BC6
:10426800054693E80700B5F5007F04AB03E90700AE
:1042780010D0224B9C4218D303F5B70303F67F53A3
:104288009C4229D903F5741303F510639C4225D881
:1042980002230BE01A4B9C4207D91A4B9C421BD9AC
:1042A80003F5370303F5D853F0E7002304AA02EB1C
:1042B800830353F80C4C144D2B6823F00703234356
:1042C8002B60FDF733FE06462B6803F007039C427C
:1042D80006D1002004B070BD0123E7E70024EAE717
:1042E800FDF724FE801B0228EED90320F2E700BF69
:1042F800A8F9000808FA000848F40008C0CF6A00C6
:10430800BFEA21013F933402004000584FF0B04308
:1043180010B59A68D96812F00C0205D00C2A4AD157
:1043280001F00303012B51D14FF0B0412B480B682A
:1043380013F0080306D00B6813F0080337D1D1F83F
:10434800941007E00C68240756BFD1F89430096828
:10435800C3F3032350F82330002A0CBF184600206B
:104368004FF0B0418A6802F00C020C2A1ED1CA68CC
:1043780002F00302022A2ED0032A06D10B68184A3B
:1043880013F4801F174B18BF13464FF0B042D06884
:10439800D168D268C0F306205843C1F30213013331
:1043A800B0FBF3F0530F0133B0FBF3F010BD0B6813
:1043B800C3F30313CEE7042A05D0082A06D11B68E5
:1043C80013F4801305D006480023C9E700231846D4
:1043D800C6E70448C4E7024BD7E700BFA8F90008BE
:1043E8000024F4000048E80108B5FFF78FFF4FF0FC
:1043F800B043044A9B68C3F3031352F82330B0FB5D
:10440800F3F008BD08FA00082DE9F0410446002839
:1044180053D04FF0B0439D68DE6803689B0605F0F3
:104428000C0506F0030668D5026A1DB10C2D46D1AD
:10443800012E44D1002A40D04FF0B043A16A1A6837
:10444800170756BFD3F894301B681B0903F0F00315
:1044580099421FD90846FFF7EFFE00282DD14FF0EB
:10446800B042136843F0080313601368A16A23F08D
:10447800F0030B431360606AFFF7CEFEFFF7B4FF4B
:10448800AB4B1860AB4B1868FDF74EFD002834D0D5
:10449800BDE8F0814FF0B042136843F008031360A1
:1044A800136823F0F0030B431360606AFFF7B4FE50
:1044B8000846FFF7C1FE0028E0D00120E8E74FF0EA
:1044C800B043002A54D01A6842F001021A60FDF77E
:1044D8002DFD0746FFF79AFE002842D04FF0B04264
:1044E800136843F0080313601368A16A23F0F0030C
:1044F8000B431360606AFFF78FFE2368D80748D420
:104508002368990700F18C8023681E0740F1FA8020
:10451800A3694FF0B046002B00F0E180D6F8943044
:10452800E16903F01002914200F0C48003F0030235
:10453800022AC2D0D80740F1B380D6F8943023F0CD
:104548000103C6F89430FDF7F1FC0746D6F894301D
:10455800990740F1A580FDF7E9FCC31B112BF5D99C
:1045680004E0FDF7E3FCC01B0228B3D903208FE762
:104578001A6822F001021A60FDF7D8FC0746FFF717
:1045880045FE0028B9D0FDF7D1FCC01B0228F6D99A
:10459800ECE7082D03D00C2D05D1032E03D1636859
:1045A800002BADD189E74FF0B043A1681A6822F417
:1045B80080120A431A606268B2F5803F10D11A6807
:1045C80042F480321A60FDF7B1FC0746FFF718FE87
:1045D800002895D1FDF7AAFCC01B6428F6D9C5E7C9
:1045E800B2F5041F04D11A6842F400121A60E6E713
:1045F800196821F480311960196821F400111960D3
:10460800002AE0D1FDF792FC0746FFF7F9FD0028E4
:104618003FF476AFFDF78AFCC01B6428F5D9A5E7FF
:10462800042D236903D00C2D0ED1022E0CD1002BA2
:104638003FF443AF4FF0B0426169536823F0FE4343
:1046480043EA016353605FE74FF0B046BBB133689C
:1046580043F480733360FDF769FC074633685A05F5
:1046680005D4FDF763FCC31B022BF7D97EE77368FB
:10467800626923F0FE4343EA0263736044E73368E8
:1046880023F480733360FDF751FC074633685B05FC
:104698007FF53AAFFDF74AFCC31B022BF6D965E755
:1046A8004FF0B042E169D2F8943023F010030B4385
:1046B800C2F894304FF0B047D7F8943043F0010374
:1046C800C7F89430FDF732FC0646D7F894309A07BD
:1046D80018D4FDF72BFC831B112BF6D946E7D6F827
:1046E800943023F00103C6F89430FDF71FFC074609
:1046F800D6F894309B0705D5FDF718FCC31B112B82
:10470800F6D933E72368580754D50B4F3B68D905CA
:1047180014D4FFF701FDFDF709FC06463B68DA05EE
:104728000CD4FDF703FC831B022BF7D91EE700BF4F
:10473800740000207800002000040058E3684FF05F
:10474800B046002B58D023F08003052B02BFD6F8C3
:10475800903043F00403C6F890304FF0B046FDF7B0
:10476800E5FBD6F8903043F001030746C6F89030D1
:1047780041F28838D6F890309B0705D4FDF7D6FB70
:10478800C31B4345F6D9F1E6E36823F00403812B04
:104798001BD1FDF7CBFBD6F8903043F08003C6F869
:1047A800903007464FF0B04641F28838D6F890303E
:1047B800180504D5E36A002B4AD1002068E6FDF706
:1047C800B5FBC01B4045F1D9D0E6FDF7AFFBD6F8E5
:1047D800903023F08003C6F8903007464FF0B0467B
:1047E80041F28838D6F890301905E3D5FDF79EFBDD
:1047F800C01B4045F6D9B9E6FDF798FBD6F89030CE
:1048080023F080030746C6F8903041F28838D6F87E
:1048180090301A0516D4FDF789FBD6F8903023F0AE
:104828000103C6F8903007464FF0B04841F2883689
:10483800D8F890309B07BDD5FDF778FBC31BB34272
:10484800F6D993E6FDF772FBC01B4045DFD98DE62C
:104858000C2D4ED0022B4FF0B0431A6822F0807214
:104868001A6033D1FDF762FB0546FFF7DEFC38BB63
:10487800D4E90C314FF0B0420B43D0682D490140C8
:104888000B43E16B0B43216C0B43616C0B43A16B36
:1048980043EA0123D360136843F080731360D3683D
:1048A80043F08053D360FDF741FB0446FFF7BDFC9E
:1048B800002882D1FDF73AFB001B0A28F6D955E6F5
:1048C800FDF734FB401B0A28CFD94FE6FDF72EFB36
:1048D8000446FFF7AAFC30B94FF0B042164BD16836
:1048E8000B40D36069E7FDF721FB001B0A28F0D9CC
:1048F8003CE6012B3FF4E1AD4FF0B043D868236BA1
:1049080000F003029A427FF4D8AD626B00F07003A6
:1049180093427FF4D2ADA26B00F4FE43B3EB022FB7
:104928007FF4CBAD636C00F06040C01A18BF012063
:10493800AEE500BF8C80C111FCFFFEEE2DE9F04111
:104948000D46044610B90120BDE8F081754E336864
:1049580003F007038B4216D32368980727D54FF037
:10496800B047A268BB6823F0F0031343BB60FDF7B0
:10497800DDFA0646BB68D90319D4FDF7D7FA831BBD
:10498800022BF7D911E0336823F007030B43336098
:10499800FDF7CCFA0746336803F00703AB42DBD0D8
:1049A800FDF7C4FAC01B0228F5D90320CCE7236819
:1049B8009A0616D54FF0B0476269D7F8083123F048
:1049C800F0031343C7F80831FDF7B0FA0646D7F8E5
:1049D80008319B0305D4FDF7A9FA831B022BF6D9EE
:1049E800E3E72368580617D54FF0B047A269D7F810
:1049F800083123F00F0343EA1213C7F80831FDF713
:104A080095FA0646D7F80831D90305D4FDF78EFA8A
:104A1800831B022BF6D9C8E723685A0713D54FF032
:104A2800B047E268BB6823F4E0631343BB60FDF75B
:104A38007DFA0646BB689B0305D4FDF777FA831B0E
:104A4800022BF7D9B1E72368180714D54FF0B04700
:104A58002269BB6823F4605343EAC203BB60FDF7D5
:104A680065FA0646BB68590305D4FDF75FFA831B50
:104A7800022BF7D999E72368DA070FD4294C236862
:104A880003F00703AB4239D8FFF7AEFC264B18609A
:104A9800264BBDE8F0411868FDF746BA6268022A5D
:104AA8001DD1FFF7ADFB00283FF44DAF4FF0B046E6
:104AB80041F28838B36823F003031343B360FDF76A
:104AC80035FA0746B368626803F00C03B3EB820F4C
:104AD800D4D0FDF72BFAC01B4045F3D965E7032A6C
:104AE80002D1FFF7A2FBDEE712B9FFF78FFBDAE787
:104AF8004FF0B0431B685B05D8D424E7236823F044
:104B080007032B432360FDF711FA0646236803F0D9
:104B18000703AB42B8D0FDF709FA801B0228F5D984
:104B280043E700BF004000587400002078000020D0
:104B380008B5FFF759FC4FF0B043044A9B68C3F32C
:104B4800022352F82330D84008BD00BFE8F9000816
:104B580008B5FFF749FC4FF0B043044A9B68C3F31C
:104B6800C22352F82330D84008BD00BFE8F9000836
:104B78004FF0B043D3F89000C0F3400070474FF0B7
:104B8800B0410209D1F8883002F47F22000123EAFB
:104B9800020300F47F200343C1F8883070474FF0C8
:104BA800B041020CD1F88830120423EA020343EA28
:104BB8000040C1F8880070470368DA0370B50446FE
:104BC80039D5FFF7A9FAFDF7B1F9614E0546336803
:104BD800DB0532D54FF0B043616BD3F8902002F477
:104BE800407291421DD0D3F89010D3F8902042F42F
:104BF8008032C3F89020D3F8902021F4407022F43A
:104C080080328D07C3F89020C3F8900009D5FDF7CE
:104C18008DF941F288360546FFF7AAFF012840F0D2
:104C280090804FF0B042616BD2F8903023F440731B
:104C38000B43C2F89030002605E0FDF777F9401BDA
:104C48000228C4D903262568E8070AD54FF0B041E1
:104C58006268D1F8883023EA124392B21343C1F84C
:104C68008830A9070AD54FF0B041A268D1F888303A
:104C780023EA124392B21343C1F88830AA0609D531
:104C88004FF0B0422169D2F8883023F440630B43D7
:104C9800C2F88830AB0502D5206AFFF780FF6805A7
:104CA80002D5606AFFF77BFF290502D5A06AFFF7E6
:104CB80076FF6A0602D56069FFF761FF2B0602D509
:104CC800A069FFF75CFFE80502D5E069FFF757FF29
:104CD800E90610D54FF0B042E168D2F8883023F4E5
:104CE80040730B43C2F88830B1F5807F02BFD368A8
:104CF80043F08073D3602A040ED54FF0B042216B85
:104D0800D2F8883023F040430B43C2F8883019B9F1
:104D1800D36843F08073D3606B0410D54FF0B04272
:104D2800E16AD2F8883023F040530B43B1F1005FB9
:104D3800C2F8883003D1D36843F48033D360304657
:104D480070BDFDF7F3F8401BB0427FF665AF79E719
:104D58000004005830B590F82C30012B02464FF073
:104D6800020022D0174B82F82D00CA24012582F8B0
:104D78002C505C6253245C62B1F5807F146B996996
:104D880014D121F488519961596C24F0010421F05F
:104D9800004159641463DD650A4BFF215962002004
:104DA800012382F82D3082F82C0030BD21F40851FF
:104DB8009961D96C24F0020421F00041D96414638C
:104DC800D865E9E70028004070B50B4E036B756D98
:104DD8001D40EA07044603D50123F365FDF703FAEE
:104DE800AB0704D50223F365204600F0C9F9012377
:104DF80084F82D3070BD00BF0028004038B50A4C3B
:104E0800E36823F02003E360FDF790F80546E368C4
:104E18009B0601D5002038BDFDF788F8401BB0F58A
:104E28007A7FF4D90320F6E700280040F8B5114D41
:104E3800EC6814F0400406461AD1EB6843F080038E
:104E4800EB60FDF773F823460746EC6814F040045E
:104E580001D1032B01D11846F8BDFDF767F8C01B37
:104E6800B0F57A7F234684BF032386F82D30ECE71C
:104E78000023F0E70028004038B50F4CE36823F022
:104E88008003E360A3699B06054606D4FFF7B6FFD7
:104E980010B1032085F82D0038BDA36923F0200345
:104EA800A361FFF7ABFF10B1032085F82D00A369BC
:104EB80043F02003A361EFE70028004038B504461B
:104EC80000284BD090F82D3003F0FF021BB980F872
:104ED8002C20FCF787FD0223214D84F82D30EB6848
:104EE800DB0636D4CA236B6253236B622046FFF776
:104EF8009DFF10B1FF236B6238BDAB6923F08E6351
:104F080023F04003AB6121696368AA690B4313432B
:104F1800A2691343AB61D4E9022343EA02432B613C
:104F2800D4E90931EA680B4322F4F8521343EB60E1
:104F38002046FFF7A1FF0028DCD1D4E90713AA69AE
:104F48000B4322F06042134362691343AB61FF23B2
:104F58006B62012384F82D300020CDE70120CBE7D8
:104F6800002800400023092803D840EA0310C0B2F3
:104F780070470A380133C0B2F5E700002DE9F04761
:104F880090F82C30012B05464FF0020069D0012320
:104F980085F82C304E4B85F82D00DE6806F44076F7
:104FA800B6F5807F78D04C69087891F8019091F82F
:104FB80002A091F82470002A55D19B6913F0400390
:104FC80008BFCB70FFF7CEFF80464846FFF7CAFF01
:104FD80002465046FFF7C6FF81463846FFF7C2FF34
:104FE8000B6ACF78234343EA875343EA090343EA2A
:104FF800084343EA022343EA0063354ACA20506261
:10500800532050628C6A8869B4F5807F946945D1D1
:1050180024F4885494610124D465B6F5807F09BFCF
:10502800CB6913640343536418BF5064284B4A6820
:105038001A672A6B42F001022A639A6942F488527D
:105048009A61244AD2F8803043F40033C2F88030A1
:105058001F4BFF225A620020012385F82D3085F866
:105068002C00BDE8F087B4F1803F07D0B4F5000FFD
:1050780004D09B6913F0400308BFCB700B6ACA7851
:105088001C4344EA0A0444EA004343EA092343EA86
:10509800825343EA0763B0E70023AEE724F40854D9
:1050A80094610224D465B6F5807F09BFCB69936407
:1050B8000343D36418BFD064054B4A685A672A6B08
:1050C80042F002022A639A6942F40852B8E700BF24
:1050D800002800400008005890F82C20012A0346B8
:1050E8004FF0020012D00A4A83F82D00CA215162FB
:1050F80053215162916941F020019161FF21516270
:105108000020012283F82D2083F82C00704700BF6F
:105118000028004090F82C20012A03464FF0020096
:1051280019D00D4A83F82D00CA21516253215162CA
:1051380091690A4841F080019161D0F8801041F4EA
:105148008021C0F88010FF2151620020012283F8DD
:105158002D2083F82C0070470028004000080058D4
:10516800064B5A6D520610B5044603D54022DA653F
:10517800FDF73CF8012384F82D3010BD00280040CD
:105188007047890001F1804101F531410A6070479B
:10519800890001F1804101F531410868704700003C
:1051A800034AD2F8903043F40043C2F89030704775
:1051B80000040058034AD2F8903023F40043C2F8A0
:1051C8009030704700040058074B1A6822F04002DC
:1051D8001A6040F441704FF4B85218605A601A6867
:1051E80042F040021A6070470000015837B5054682
:1051F80000284ED0837903F0FF046BB1032C0BD049
:10520800254B4FF400629A612868FFF7DDFF002400
:1052180001232B71AC602FE000236B712846FCF74B
:105228009BFD1E4AD2F8903043F48053C2F8903068
:10523800002CE5D102234FF0B042AB71D2F8943084
:1052480023F40043C2F89430154B1B681C214B43D0
:10525800DB0C64214B430193019B93B90124AC609F
:10526800FFF79EFF0C4B9A6842F400629A604FF475
:1052780000629A61002CC7D00123AB71204603B0AD
:1052880030BD019B013B0193D2F894305B04E3D419
:10529800E6E70124F2E700BF0004005800080058C0
:1052A8007400002037B5174D2B6802461C20434375
:1052B800DB0C6420434314480193019B93B90120FC
:1052C8009060114C21732B681C214B43DB0C64212B
:1052D8004B430193019B6BB9012090600A4BDB683B
:1052E80003B030BD019B013B019383689C07E4D563
:1052F8000020E6E7019B013B0193A368DB07E9D5A2
:10530800ECE700BF740000200000015837B5184DC5
:105318002B6802461C204343DB0C6420434315489A
:105328000193019BA3B901209060124CFF232373C2
:105338002B681C256B43DB0C64256B430193019B95
:1053480073B9012090600B4BDB680B7003B030BD64
:10535800019B013B019383689C07E2D50020E4E7A9
:10536800019B013B0193A368DB07E8D5EBE700BF8E
:1053780074000020000001580E4B0F491B681822CA
:10538800534382B01B0D6422534301934B69019A26
:10539800C3F3800322B902238360012002B070475F
:1053A800019A013A01924A69920701D5002BEDD181
:1053B8000020F3E7740000200004005807B50379C3
:1053C800012B0FD10A4B1B68182253431B0C019366
:1053D800FFF7F0FE019B013B0193019B002BF9D1E4
:1053E800FFF7DEFE03B05DF804EBFFF7C5BF00BFB3
:1053F80074000020F8B51E468379012B1546044633
:105408000F46DAB22DD14379012B2AD002234271FB
:105418008371FFF7D3FF0D212046FFF7CBFEFFF77F
:1054280041FF390A2046FFF73DFFF9B22046FFF752
:1054380039FF2E44B5420ED12046FFF7B1FEFFF7E3
:105448009BFFA06801230038A3714FF0000318BF29
:1054580001206371F8BD15F8011B2046FFF722FFF4
:10546800E8E70220F6E7F8B51E468379012B1546D2
:1054780004460F46DAB22FD14379012B2CD0427162
:10548800FFF79CFF1D212046FFF794FEFFF70AFF58
:10549800390A2046FFF706FFF9B22046FFF702FF58
:1054A80000212046FFF7FEFE2E44B5420ED12046CD
:1054B800FFF776FEFFF760FFA06801230038A371AD
:1054C8004FF0000318BF01206371F8BD294620463C
:1054D800FFF71CFF0135E8E70220F6E7F8B51F469D
:1054E8008379012B154604460E46DAB22CD143794E
:1054F800012B29D04271FFF761FF06F0EF03A3F1FA
:10550800840253425341237131462046FFF752FE2D
:10551800FFF7C8FE2F44AF4210D1FFF741FE842E9B
:1055280002D02046FFF728FFA06801230038A371A6
:105538004FF0000318BF01206371F8BD15F8011B77
:105548002046FFF7AFFEE6E70220F6E7F8B51E466D
:105558008379012B154604460F46DAB227D14379E1
:10556800012B24D04271FFF729FF39462046FFF767
:1055780021FEFFF797FE00212046FFF793FE2E44F9
:10558800B5420ED12046FFF70BFEFFF7F5FEA068E7
:1055980001230038A3714FF0000318BF0120637185
:1055A800F8BD29462046FFF7B1FE0135E8E702209D
:1055B800F6E737B50023ADF8043001AA022312211B
:1055C8000546FFF7C3FFBDF80440022364BA01AAE9
:1055D800A4B219462846FFF781FFE20702D52846FC
:1055E80008F0DEFFA30702D5284608F0DFFF6007B2
:1055F80002D5284609F004F8210702D5284609F003
:1056080005F8E20602D5284609F006F8A30602D5F1
:10561800284608F0EFFF600602D5284608F0CCFFC0
:10562800210606D514F4807118BF0121284608F018
:10563800C9FFA20502D5284608F0D4FF630402D5A5
:10564800284608F0EFFF03B030BDF8B51E46837951
:10565800012B154604460F46DAB227D14379012BB0
:1056680024D04271FFF7AAFE0E212046FFF7A2FDC3
:10567800FFF718FE39462046FFF714FE2E44B542C0
:105688000ED12046FFF78CFDFFF776FEA0680123B8
:105698000038A3714FF0000318BF01206371F8BDF3
:1056A80015F8011B2046FFF7FDFDE8E70220F6E7A5
:1056B800F8B51E468379012B154604460F46DAB223
:1056C8002BD14379012B28D04271FFF777FE1E2199
:1056D8002046FFF76FFDFFF7E5FD39462046FFF747
:1056E800E1FD00212046FFF7DDFD2E44B5420ED135
:1056F8002046FFF755FDFFF73FFEA068012300385D
:10570800A3714FF0000318BF01206371F8BD29464B
:105718002046FFF7FBFD0135E8E70220F6E70268BF
:1057280052E8003F23F0C00342E800310268002934
:10573800F5D102F1080353E8003F23F4000302F116
:10574800080C4CE800310029F3D12023C0F8883038
:105758007047000010B5026852E8003F23F49073C8
:1057680042E8003102680029F5D10F4C02F1080324
:1057780053E8003F234002F1080C4CE800310029AF
:10578800F4D1C36E012B07D152E8003F23F0100378
:1057980042E800310029F7D12023C0F88C300023DB
:1057A800C366436710BD00BFFEFFFFEFF8B50446B0
:1057B8001346D4F88850202D32D1F1B1EAB1E06F08
:1057C800A4F85620A4F8542000262122C4F890609A
:1057D8002165C4F88820226888B1124FC762124F29
:1057E8000763124F2832C0E90D76FEF749F930B148
:1057F8001023C4F89030C4F888500120F8BD2368FD
:1058080040221A62226802F1080353E8003F43F07D
:10581800800302F1080141E800300028F3D1EDE7E8
:105828000220EBE739580008815800088D58000815
:1058380008B50346806A1B681B6813F0200317D15C
:10584800A0F85630026802F1080353E8003F23F03D
:105858008003083242E8003102680029F2D152E898
:10586800003F43F0400342E800310029F7D108BD6A
:10587800FCF7FAFDFBE7704708B5806AFFF7FBFF06
:1058880008BD7047806A38B50468D0F88830D0F809
:105898008C50A268120606D5212B04D10023A0F84B
:1058A8005630FFF73CFFA3685B0606D5222D04D1CE
:1058B8000023A0F85E30FFF74DFFD0F8903043F09A
:1058C8001003C0F89030FFF7DCFF38BD08B5806AD8
:1058D8000023A0F85E30A0F85630FFF7D2FF08BDCD
:1058E800704700000368D9691A682DE9F04140F64D
:1058F8000F0631429D68044610D18E0640F197800C
:1059080002F0200605F080573E4300F09080436F78
:10591800002B00F08580BDE8F0411847AB4EAC483D
:105928002E401040304300F08280CF0709D5D005C3
:1059380007D501201862D4F8900040F00100C4F89F
:1059480090008F0709D5E80707D502201862D4F818
:10595800900040F00400C4F890004F0709D5E8070C
:1059680007D504201862D4F8900040F00200C4F86B
:1059780090000F070BD502F02000304307D0082015
:105988001862D4F8900040F00800C4F890000E05A2
:105998000AD5500108D54FF400601862D4F8903049
:1059A80043F02003C4F89030D4F89030002B37D05F
:1059B8008B0609D502F0200205F080552A4303D052
:1059C800636F0BB1204698472668D4F89020B368D7
:1059D80002F0280203F0400353EA0205204621D0D2
:1059E800FFF7B8FEB3685F0617D5226802F108030F
:1059F80053E8003F23F04003083242E80031002911
:105A0800F3D1D4F8800040B1724B8363FEF7B1F84C
:105A180030B1D4F88000836B7DE72046FFF731FF73
:105A2800BDE8F081FFF72DFFC4F89050F8E7E06E6D
:105A3800012840F08980CE0640F18680D00640F1EA
:105A4800838010221A629A6851064BD5D4F88020B8
:105A580011684A6892B2002AE2D0B4F85C00904219
:105A6800DED9A4F85E200A6892062FD453E8002FE6
:105A780022F4807243E800210029F7D103F10802DB
:105A880052E8002F22F0010203F1080040E800214B
:105A98000029F3D103F1080252E8002F22F0400256
:105AA80003F1080040E800210029F3D12022C4F8BE
:105AB8008C20E16653E8002F22F0100243E8002111
:105AC8000029F7D1D4F88000FEF71EF802232367D7
:105AD800B4F85E30B4F85C10C91A89B22046FFF7F2
:105AE800FFFE9DE7B4F85E20B4F85E00B4F85C10E1
:105AF80080B292B2002893D0891A89B200298FD037
:105B080053E8002F22F4907243E800200028F7D1D0
:105B1800314D03F1080252E8002F2A4003F108062C
:105B280046E800200028F4D12022C4F88C206067C1
:105B3800E06653E8002F22F0100243E80020002816
:105B4800F7D102232367C9E7CF0209D56E0207D52B
:105B58004FF4801220461A62BDE8F04100F0A0BD63
:105B680008060BD502F0800005F40005284305D08F
:105B7800A36F002B3FF454AF2046CCE64F0611D557
:105B880056060FD553E8002F22F0400243E80021C3
:105B98000029F7D12023C4F88830A1672046FCF7F4
:105BA80063FC3DE70D0206D5500004D52046BDE84C
:105BB800F04100F077BDCB017FF532AF002ABFF688
:105BC8002FAF2046BDE8F04100F06BBD010000108A
:105BD80020010004D5580008FEFFFFEFD0F88C2004
:105BE800B0F86010222A08B5036855D15B6A826D47
:105BF8000B401370836D01338365B0F85E30013B51
:105C08009BB2A0F85E30B0F85E309BB2002B42D158
:105C1800026852E8003F23F4907342E800310368B9
:105C28000029F5D103F1080252E8002F22F0010201
:105C380003F1080C4CE800210029F3D12022C0F818
:105C48008C20184A41679342016705D1C26E012A28
:105C58000ED0FCF717FC1EE05A681102F6D553E87F
:105C6800002F22F0806243E800210029F7D1EDE7F8
:105C78000022C26653E8002F22F0100243E80021F8
:105C88000029F7D1DA69B0F85C10D20644BF1022B7
:105C98001A62FFF725FE08BD9A6942F008029A6168
:105CA800F9E700BF00800040D0F88C20B0F8601001
:105CB800222A08B5036852D15A6A1140826D22F827
:105CC800021B8265B0F85E20013A92B2A0F85E200D
:105CD800B0F85E2092B2002A40D153E8002F22F497
:105CE800907243E800210029F7D103F1080252E835
:105CF800002F22F0010203F1080C4CE800210029D2
:105D0800F3D12022C0F88C20174A416793420167DB
:105D180005D1C26E012A0ED0FCF7B4FB1EE05A680A
:105D28001102F6D553E8002F22F0806243E80021E3
:105D38000029F7D1EDE70022C26653E8002F22F0D0
:105D4800100243E800210029F7D1DA69B0F85C10A5
:105D5800D20644BF10221A62FFF7C2FD08BD9A6935
:105D680042F008029A61F9E7008000402DE9F84FF7
:105D78000368B0F86060D3F81CB01F689D68D0F85D
:105D88008C20222A044640F0B980B0F8683043B12C
:105D9800DFF87491DFF874A14FF000081BF0200FB2
:105DA80020D1B4F85E309BB2D3B1B4F868209A42DF
:105DB80016D9226802F1080353E8003F23F0805304
:105DC800083242E8003122680029F2D1504B63675B
:105DD80052E8003F43F0200342E800310029F7D1A0
:105DE800BDE8F88F2368A26D5B6A33401370A36D1A
:105DF8000133A365B4F85E30013B9BB2A4F85E3072
:105E08002368D3F81CB01BF0070F2ED01BF0010F2E
:105E180009D0F90507D501221A62D4F8902042F07A
:105E28000102C4F890201BF0020F09D0EA0707D539
:105E380002221A62D4F8902042F00402C4F890209A
:105E48001BF0040F09D0E80707D504221A62D4F81A
:105E5800903043F00203C4F89030D4F8903023B166
:105E68002046FFF70EFDC4F89080B4F85E309BB270
:105E7800002B93D1226852E8003F23F4807342E854
:105E8800003123680029F5D103F1080252E8002FF8
:105E980002EA090203F1080040E800210029F3D1D1
:105EA80020225345C4F88C20616721670AD05A68BC
:105EB800110207D553E8002F22F0806243E8002141
:105EC8000029F7D1E26E012A14D10022E26653E8D4
:105ED800002F22F0100243E800210029F7D1DA69E7
:105EE800B4F85C10D20644BF10221A622046FFF7AD
:105EF800F7FC53E72046FCF7C5FA4FE79A6942F0EA
:105F080008029A616CE700BFFEFFFFEF00800040C7
:105F1800E55B00082DE9F84F0368B0F86060D3F836
:105F28001CB01F689D68D0F88C20222A044640F0D7
:105F3800B780B0F8683043B1DFF87091DFF870A12E
:105F48004FF000081BF0200F20D1B4F85E309BB250
:105F5800D3B1B4F868209A4216D9226802F108032E
:105F680053E8003F23F08053083242E800312268AA
:105F78000029F2D14F4B636752E8003F43F02003FA
:105F880042E800310029F7D1BDE8F88F2368A26DF7
:105F9800596A314022F8021BA265B4F85E20013A22
:105FA80092B2A4F85E20D3F81CB01BF0070F2ED0D5
:105FB8001BF0010F09D0F90507D501221A62D4F8A0
:105FC800902042F00102C4F890201BF0020F09D083
:105FD800EA0707D502221A62D4F8902042F0040298
:105FE800C4F890201BF0040F09D0E80707D5042255
:105FF8001A62D4F8903043F00203C4F89030D4F811
:10600800903023B12046FFF73CFCC4F89080B4F8E8
:106018005E309BB2002B95D1226852E8003F23F4F2
:10602800807342E8003123680029F5D103F10802A2
:1060380052E8002F02EA090203F1080040E80021B3
:106048000029F3D120225345C4F88C2061672167C9
:106058000AD05A68110207D553E8002F22F080624F
:1060680043E800210029F7D1E26E012A14D1002269
:10607800E26653E8002F22F0100243E800210029CD
:10608800F7D1DA69B4F85C10D20644BF10221A625C
:106098002046FFF725FC55E72046FCF7F3F951E7C2
:1060A8009A6942F008029A616EE700BFFEFFFFEFAF
:1060B80000800040B15C000838B5044603682169D7
:1060C800A2681D68C0690A4361690A4377490243A7
:1060D80029400A431A605A68E16822F440520A4388
:1060E8005A60734AA16993421CBF226A11439A6895
:1060F80022F06E4222F430620A439A60DA6A616AD8
:1061080022F00F020A43DA626A4A934219D14FF029
:10611800B043694AD3F8883003F0030343F44033AB
:10612800934200F0B480B3F1031F24D0013A9342A4
:1061380040F0B580B0F5004F40F08F80FEF7E6F8EC
:106148006EE05E4A93421CD14FF0B0435C49D3F8ED
:10615800883003F00C0343F440228A4200F0978011
:1061680006D8002B7CD0574B9A42E3D0012026E07A
:10617800B2F10C1FFAD1B0F5004F53D04FF40040E4
:1061880075E04B4A9342F1D14FF0B043D3F88830D1
:1061980003F44063B3F5006F18D006D85BB1B3F5CC
:1061A800806FE3D1FEF7B2F807E0B3F5406FDDD1B9
:1061B8004FF400400BE0FEF7BBFC40B900204FF065
:1061C8000113A3660023C4E91D3338BD3E48656842
:1061D8003E4B626A05EB450133F81220B0FBF2F33F
:1061E8009942C3D8B3EB053FC0D800231946FAF744
:1061F800E9FE090241EA10616B080002C0182A464C
:106208004FF0000341F10001FAF7DCFE304BA0F536
:1062180040729A42AAD82368D860CFE7FEF788FC74
:106228000028CBD06168294B626A33F81220B0FB92
:10623800F2F24B0803EB42034FF6EF72B3FBF1F3B4
:10624800A3F11001914291D823F00F02216892B274
:10625800C3F342031343CB60B0E7FEF757F804E0FB
:10626800B0F5004FDAD0FEF763FC0028A6D06368CB
:10627800616A164A32F81120B0FBF2F000EB5300C5
:10628800B0FBF3F04FF6EF73A0F11002C1E7B0F5E1
:10629800004F0D48EBD1C5E7FEF75AFCC0E7B0F553
:1062A800004FF9D0FEF754FCDFE700BFF369FFCFDA
:1062B8000080004000380140020003000044004014
:1062C80008000C0004000C000024F40048FA000840
:1062D800FFFC0F00836ADA0710B506D50168C46AA7
:1062E8004A6822F4003222434A609C0706D50168B6
:1062F800046B4A6822F4803222434A60590706D563
:106308000168446B4A6822F4802222434A601A07D3
:1063180006D50168846B4A6822F4004222434A6029
:10632800DC0606D50168C46B8A6822F480522243D1
:106338008A60990606D50168046C8A6822F40052BE
:1063480022438A605A060FD50168446C4A6822F4D1
:1063580080122243B4F5801F4A6005D14A68846CD4
:1063680022F4C00222434A601B0606D50268C16CAB
:10637800536823F400230B43536010BD2DE9F84301
:10638800DDF8209005460F46164698462A68D369D8
:1063980037EA03030CBF01230023B34201D00020D6
:1063A80029E0B9F1FF3FF2D0FBF7C0FDA0EB0800F0
:1063B80048452C6802D8B9F1000F1ED154E8003FB7
:1063C80023F4D07344E80032002AF7D104F108031B
:1063D80053E8003F23F0010304F1080141E80032CB
:1063E800002AF3D12023C5F88830C5F88C30002363
:1063F80085F884300320BDE8F88323685A07C5D59B
:10640800E3691B05C2D54FF40063236254E8003FDB
:1064180023F4D07344E80032002AF7D104F10803CA
:1064280053E8003F23F0010304F1080141E800327A
:10643800002AF3D12023C5F88830C5F88C30C5F878
:106448009030D4E773B504460026C0F89060FBF797
:106458006DFD23681B681A07054619D423681B6855
:106468005B070AD56FF07E43009300222B464FF45A
:1064780080012046FFF782FFB0B900202023C4F82E
:10648800883084F88400C4F88C30E06620670CE01B
:106498006FF07E430093324603464FF400112046C6
:1064A800FFF76CFF0028D9D0032002B070BD10B5EB
:1064B800044650B3D0F888301BB980F88430FBF715
:1064C800D7FE22682423C4F88830136823F0010318
:1064D80013602046FFF7F0FD012816D0A36A13B118
:1064E8002046FFF7F7FE23685A6822F490425A6064
:1064F8009A6822F02A029A601A6842F0010220463D
:106508001A60BDE81040FFF79DBF012010BD0000D4
:1065180030B581658168A0F85C200023B1F5805F03
:10652800A0F85E20436735D10369002B40F2FF13C2
:1065380018BFFF23A0F860300023C0F89030222352
:10654800C0F88C30016801F1080353E8003F43F0BC
:106558000103083141E800340368002CF2D1456E8C
:1065680084680169B5F1005F32D1B0F8685095428E
:106578002ED8B4F5805F244A03D1244C002908BFE3
:1065880022464267B1B153E8002F42F4807243E8D3
:106598000021F7E729B90369002B14BF7F23FF23E4
:1065A800C8E7B1F1805FC5D10369002B14BF3F2351
:1065B8007F23BFE703F1080252E8002F42F0805220
:1065C80003F1080040E800210029F3D1002030BD84
:1065D800B4F5805F0E4A03D10E4C002908BF22464D
:1065E800426741B153E8002F42F4907243E800211A
:1065F8000029F7D1EAE753E8002F42F0200243E8E8
:1066080000210029F7D1E1E7755D00081D5F00084A
:10661800E55B0008B15C0008D0F88C30202B30B462
:1066280015D1B9B1B2B100230468C3660A4B9C42C4
:106638000AD063681B0207D554E8003F43F0806323
:1066480044E80035002DF7D130BCFFF761BF0220C8
:1066580030BC70470120FBE700800040436E30B536
:106668002BB90123A0F86A30A0F8683030BD036860
:10667800094D9A689968094C490FC2F342626B5CEC
:10668800615CDB00B3FBF1F3A0F86A30AB5CA25CA1
:10669800DB00B3FBF2F3E7E768FA000860FA0008EA
:1066A8007047704770471FB504AB03E9060090F8C0
:1066B8008430012B04463AD0012380F88430242307
:1066C800C0F8883003681A6822F001021A609A68D4
:1066D80022F440120A439A6071B95A68BDF80C0056
:1066E8009DF80E1022F0100202435A605A6822F0F8
:1066F8007F4242EA01625A601A6842F001021A6057
:10670800FBF714FC6FF07E42034600924FF48001C1
:1067180000222046FFF732FE38B92023C4F888301B
:10672800002384F8843004B010BD0320F8E7022069
:10673800F9E790F88430012B0FD0012380F88430DA
:10674800016851E8002F42F0020241E80023002BC3
:10675800F6D180F88430184670470220704710B58B
:1067680090F88430012B044617D02423C0F88830D1
:1067780003681A68196821F00101196042F0005293
:106788004FF0005141661A60FFF768FF2023C0F8F8
:106798008830002084F8840010BD0220FCE770B522
:1067A80090F88430012B044617D005682423C0F8DC
:1067B80088302E682B6823F001032B60AB6823F028
:1067C80060431943A960FFF749FF20232E60C0F8F2
:1067D8008830002084F8840070BD0220FCE770B582
:1067E80090F88430012B044617D005682423C0F89C
:1067F80088302E682B6823F001032B60AB6823F0E8
:1068080060631943A960FFF729FF20232E60C0F8B1
:106818008830002084F8840070BD0220FCE7000066
:1068280038B5084D052455F8043B2BB9013C14F044
:10683800FF04F8D1204638BDDB6898470028F5D01A
:10684800F9E700BFBC050020034BD870034B1B6859
:106858001B6C03B118477047A4050020A005002051
:10686800034B1874034B1B685B6C03B118477047E4
:10687800A4050020A0050020F0B5314D314B95F955
:106888000420314E91B00C46012795F905108DF87A
:10689800047002288DF809208DF80A1010D18DF89F
:1068A8000800D8711C7202F063FD337803B114B18B
:1068B80001A803F0C1F9254B059A1A6011B0F0BD83
:1068C80059714FF480711A71D9801C7233788DF820
:1068D800087053BB1F2306A88DF81C208DF81830AC
:1068E80002F024FF20238DF8183006A82B798DF8A4
:1068F8001C3002F01BFF22238DF8183006A86B7994
:106908008DF81C3002F012FF21238DF8183006A8EC
:106918006B798DF81C3002F009FF29238DF81830A7
:1069280006A80B4B079302F001FF02F021FD01239B
:1069380006A88DF818308DF81C3002F0F7FEB4E781
:10694800A4050020AC00002080040020740500206D
:10695800000400017FB5092301A88DF8043003F075
:106968006BF90038044B059A1A6018BF01204042A1
:1069780007B05DF804FB00BF7405002070B504463D
:106988000B46144962784A700020A2780A7208708F
:106998001A884A729A788A72DB780B746368CB60BB
:1069A8000D4B1B68DA6A2AB1237803F0FB030A2B24
:1069B80000D09047094E002556F8043B1BB15B6A8E
:1069C8000BB1204698470135EBB2052B6DB2F3D1D8
:1069D80070BD00BF7C000020A0050020BC05002081
:1069E80070B5044611480123037063784370A37897
:1069F8008372E368C360E378037623694376237977
:106A080043720B4B1B689B6A03B19847094E0025DC
:106A180056F8043B1BB19B690BB1204698470135DA
:106A2800EBB2052B6DB2F3D170BD00BF9000002012
:106A3800A0050020BC050020014B1868704700BF66
:106A48007405002000B58BB0012368468DF800302E
:106A580002F046FD38B99DF80400003818BF01203F
:106A68000BB05DF804FB0020FAE7000008B501F060
:106A780037FE40B9FFF7E6FF012806D0054B197A23
:106A8800D879FFF7F9FE012008BDBDE80840FFF7F7
:106A9800C7BE00BFAC0000202DE9F04186B0054616
:106AA8000E46174601F01CFE002873D101F030FE97
:106AB800044640B9FFF7C6FF01280AD03D4B197AB2
:106AC800D879FFF7D9FE6FF00204204606B0BDE87A
:106AD800F081DFF8E48088F80860003E18BF0126DE
:106AE8008DF80460354E687833798DF81230694630
:106AF80002F094FC00283FD08DF804400394ADF8D0
:106B080010406FF0060495E803002D4B83E803005E
:106B1800337988F80A30394601A803F091F9294BEE
:106B2800059A1A6011283FD801A353F820F000BF36
:106B3800A36B00089D6B0008B16B0008B16B0008DF
:106B4800B16B0008B16B0008B16B0008CF6A000890
:106B5800B16B0008B16B0008B16B0008976B0008B7
:106B6800B16B0008B16B00089D6B00089D6B0008B5
:106B78009D6B0008B76B00082B788DF808306B7890
:106B8800ADF810306B6803934FF0FF34BBE76FF03C
:106B980005049AE76FF0010497E70B4B00221A707F
:106BA800E31D18BF144690E74FF0FF348DE76FF0F0
:106BB80004048AE7AC00002090000020A40500200F
:106BC800A0000020740500207305002037B501F0EF
:106BD800A9FD134D052455F8043B4BB11A693AB188
:106BE8009B682BB1984718B155F8043C1B69984726
:106BF800013C14F0FF04EED1FFF712FE68B9094D0D
:106C08002B7853B1084BADF80040D978019422464F
:106C18006846FFF741FF00B92C7003B030BD00BFD4
:106C2800BC05002073050020A405002030B58BB0FA
:106C3800044601F055FD0546002835D1FFF702FF4F
:106C4800012834D168468DF8005002F049FC40BB59
:106C58009DF80430A34204D0012C22D0022C12D07B
:106C680014B100200BB030BD002BFAD068468DF867
:106C7800044002F05BFDA0B90E4B1B681B6B002B98
:106C8800EFD09847EDE763B968468DF8044002F005
:106C98004DFD30B9074B1B681B6B002BE1D020461C
:106CA800EFE74FF0FF30DDE76FF00100DAE76FF054
:106CB8000200D7E7A005002010B504468AB018B92D
:106CC8004FF0FF300AB010BD002368468DF8003041
:106CD80002F006FC0028F3D19DF804302370F1E798
:106CE8007FB500220B4620498DF8072001220A7043
:106CF80042784A700446002A33D102790A721A8807
:106D08004A729A788A72DB780B740369CB60C3780D
:106D1800164D8DF80830037B8DF80930836803938E
:106D28002B68DB6A0BB102A898472B689B6B13B1E1
:106D3800227E02B198470E4E052556F8043B1BB13A
:106D4800DB690BB120469847013D15F0FF05F4D1EA
:106D58000DF10700FFF7B0FF637913B1054B01226E
:106D68001A7004B070BD00BF7C000020A005002090
:106D7800BC0500207305002010B504468AB018B978
:106D88004FF0FF300AB010BD202368468DF8003060
:106D980002F0A6FB0028F3D1024A9DF904302370C3
:106DA8001371EFE7A405002000B58BB023230190F1
:106DB80068468DF8003002F0B9FC003818BF012091
:106DC80040420BB05DF804FB70B5654C01468EB0CF
:106DD8001822204606F08CF8624B00221A70FBF746
:106DE800B7FF23784068012202FA03F1014004D179
:106DF8005D4B084607F03AFDFEE75C495C481A46D9
:106E080002F0F8F818B14FF0FF300EB070BD27232C
:106E180004A88DF8103002F089FC564E564D002813
:106E280070D1012333702B68DB690BB100209847C0
:106E3800272304A88DF8103002F052FB059B93F825
:106E48004820227093F8182193F81A316270A370C1
:106E5800464BD3E9020105F03BFF05460028D2D195
:106E6800464E062304A88DF8103002F039FB059B26
:106E7800736104A802F05AFC022304A88DF81030AC
:106E8800059602F02DFB0836032304A88DF8103070
:106E9800059602F025FB0F2605F0E0FF012304A864
:106EA8008DF814308DF8106002F040FC10230DEBC3
:106EB80003008DF810308DF8145002F037FC0423CD
:106EC8008DF8103004A8A3788DF8143002F02EFC49
:106ED8003A238DF8103004A86369059302F026FC64
:106EE80002A920788DF8086004F09CF8003818BFD3
:106EF8000120E0711420FFF757FFE07903F062F9F1
:106F0800284682E728238DF810302B681B6943B187
:106F180004A802F0E5FA2B6805981B6940F2C451F1
:106F28009847272304A88DF8103002F0FFFB50B9CA
:106F3800012304A88DF8103002F0D2FA9DF814301D
:106F4800002B7FF46EAF3378002B7FF46CAF0522F3
:106F580004A88DF81020059302F0E8FB78E700BF3D
:106F6800A40500207305002070FA000878050020A9
:106F78009005002080040020A0050020E0050020E6
:106F880037B500230D4601930446D0B900F0A8FB9D
:106F98000190019BD3B10F4A42F824300E4A9A62FD
:106FA8000E4A1268916B1963916C596392690C4986
:106FB800D9625A6128465B680A49F222984700203C
:106FC80006E001A900F092FB0028E2D04FF0FF3064
:106FD80003B030BDBC05002081680008A005002072
:106FE8005D69000881040020194B07B51860194B2A
:106FF800194A1A60194A5A60194A9A60194ADA6095
:10700800194B02681A6042685A6082689A60C268BE
:10701800DA60164A1A6182695A61154BC26B5A6066
:10702800144A019119609A601946134ADA600020DF
:10703800FFF7A6FF48B901A800F056FB003818BFB3
:107048000120404203B05DF804FB4FF0FF30F9E740
:10705800A005002090050020E9690008E96C0008F7
:10706800FD7000088569000878050020DDAF00087C
:10707800D0050020516800086968000849B118B1B6
:10708800012804D000207047034B0B60FAE7034B3C
:10709800FBE74FF0FF3070470004000101000102D8
:1070A80008B503F0ABF8002814BF6FF0010000200A
:1070B80008BD08B502F084F9002814BF6FF001007C
:1070C800002008BD10B504468AB018B94FF0FF304B
:1070D8000AB010BD212368468DF8003002F000FA8E
:1070E8000028F3D1024A9DF9043023705371EFE769
:1070F800A40500202DE9F0412F4D304F00232B70BF
:1071080043786B703B689B6A8AB004460BB128468B
:107118009847DFF8AC80002658F8043B1BB11B6A7F
:107128000BB1204698470136F3B2052B76B2F3D15E
:107138002378052B2FD00B2B35D0012B25D1214CB3
:10714800062368468DF8003002F0CAF90199E07903
:1071580005F004FE10B91C4B019A5A611B48FFF751
:107168000BFE1B48FFF7AEFF6B788BB9A371194B69
:107178005878FFF75BFD3B685B6A0BB1114898478D
:107188006B7813B9E07905F07BFE0AB0BDE8F081B1
:10719800FF23A371EFE7104B01225A74227A9A74E5
:1071A800627ADA74F1E76378002BEED00AB0BDE8B2
:1071B800F041FFF7CFBB00BF90000020A0050020E2
:1071C800BC050020AC000020E0050020B000002035
:1071D800B1000020A40500207C00002030B58BB051
:1071E800FFF767FF0446F0B903F0FCFE831C1DD0CF
:1071F800F8B9134D2B685B69DBB1272368468DF816
:10720800003002F06DF92B6801985B694FF4B961A1
:10721800984703F0F9FE78B92CB9094B1B68DB696C
:107228000BB10120984720460BB030BD6FF0070422
:10723800EFE74FF0FF34ECE74FF0FF34F3E700BF20
:10724800A0050020014B1878704700BF14060020E5
:10725800014B5878704700BF1406002070470000A3
:10726800044B9A7A0AB101225A70034B5B6903B145
:107278001847704714060020B800002073B5224C48
:107288006378002B33D007F0D9FD66680546FFF711
:10729800D3FB0644AE4214D2A37A93B1E0228DF810
:1072A80000208DF80130217AE368019301226846B5
:1072B800FFF7F2FB08B1073010D100236370A37207
:1072C800656094F83430EBB1002384F834300F4B08
:1072D8005B6BBBB102B0BDE87040184740F2DC51AF
:1072E8000B4807F077FE0A4807F03AFEE8E794F8FB
:1072F8003520002AE5D094F8360084F83530FFF7B9
:1073080095FCDEE702B070BD14060020B80000202E
:10731800F805002037B5104D104CC8B1C1B16272E4
:10732800012300222860E16023700D480D4B009274
:107338004FF0FF3107F068FD00250B482582202219
:10734800294605F0E9FD6570A574A58603B030BD32
:1073580000232B602370EFE710060020140600209E
:10736800F805002069720008280600202DE9F0477A
:107378008E4C23788CB0002B56D0C2780AB9837B08
:1073880013B1238A01332382437B002B4CD0E02A9C
:107398004AD10023A372876897F80080B8F1220FBA
:1073A80027D8B8F1220F30D8DFE818F04100FB00E9
:1073B80052005A0061006E0075008E009D00B400F6
:1073C800C7002F002F002F002F002F002F002F00A5
:1073D8002F002F002F002F002F002F002F002F002D
:1073E8002F002F002F002F002F002F00C900D000E2
:1073F800D400B8F17E0F00F0CC80B8F17F0F00F018
:10740800DF80B8F17D0F00F0AB80A57A002D00F089
:107418005B81674C637A3BB94FF47A71204607F079
:10742800D9FD204607F09CFD0CB0BDE8F087E36865
:1074380001220021A2721970A37AE1689818A0723B
:107448000620C854A37AE1689818A072CA54DCE7E9
:10745800584B9B6A002BD8D0012102209847D4E7CB
:107468007B7884F83630012384F83530CDE704235F
:107478008DF804307B78003B18BF012301A88DF8F4
:10748800083002F053F9C0E77878003818BF0120B7
:1074980002F098FEB9E7484E0FCE01AD0FC50FCEEA
:1074A8000FC596E8070085E807007B780A2BACD85B
:1074B800424A12685268002AA7D00CA901EB83033C
:1074C80053F82C0C9047A0E77878431E012B9CD8E2
:1074D8003A4B01381B6818BF012020729B68002BAB
:1074E80093D0984791E7E26801230821A3721170AD
:1074F800627A057BA17AAA4228BF2A46934284D29F
:1075080085685A1CEB5CE56801334E1CA6726B5407
:10751800D3B2EDE7E3680122A27209221A70A37AB6
:10752800E268218A581CA072D154A27A238AE168A1
:107538001B0A501CA0728B5467E7238265E705235A
:107548008DF8043001A802F077FB5EE7194BDB6A7F
:1075580098475AE7194B78781B686075DB68BEE76F
:10756800037B072B7FF451AF06238DF80430B7F85F
:107578000130ADF808307B793A791B0443EA0223DD
:10758800FA781343642253430393BB798DF8103080
:10759800D8E73B2201A88DF804208DF8083002F0C6
:1075A800C5F8012384F834302FE700BF1406002003
:1075B800F8050020B800002054F400081006002048
:1075C8002A2301A88DF8043001F08AFF94F80A9064
:1075D800E6689DF808009DF809509DF80A709DF826
:1075E8000BC09DF80D309DF80E209DF80F109DF8EA
:1075F8000CE009F1010A84F80AA006F80980354E62
:1076080094F80A903668D4F80C8009F1010A84F8D5
:107618000AA096F803A008F809A094F80A90D4F8EC
:107628000C8009F1010A84F80AA096F802A008F86B
:1076380009A094F80A90D4F80C8009F1010A84F89A
:107648000AA096F801A008F809A094F80A9009F190
:10765800010A84F80AA096F80080E66806F809800E
:1076680094F80A80E66808F1010984F80A9006F897
:1076780008C094F80AC0E6680CF1010884F80A808A
:1076880006F80C70A77AE66807F1010C84F80AC0BE
:10769800F555A57AE6686F1CA7727055A07AE5685B
:1076A800461CA6722954A17AE0684D1CA572425462
:1076B800A27AE168501CA0728B54A37AE268591C24
:1076C800A17202F803E0A0E6034807F0FBFB65702F
:1076D800AAE600BF10060020F80500207047000049
:1076E80000487047B8000020002070474FF0FF3076
:1076F80070470000044B054A93F81831022B18BF55
:10770800062382F89034704700800020F406002099
:10771800034BD3F8483313B15B6903B1184770477B
:10772800F4060020034A137843F004031370FFF7AC
:10773800EFBF00BF600600201FB50A4B8DF8090097
:1077480093F87C208DF80A2093F88C2093F8480051
:107758000D3202A98DF8082003F064FCC0B205B010
:107768005DF804FB0080002008B5074807F0AAFB75
:10777800064B93F81A2412B1012283F81924BDE8A4
:107788000840FFF7C5BF00BFF40A0020F406002038
:1077980010B50C4CD4F8403343F08003C4F84033A0
:1077A80094F81A3413B10020FFF7DEFF94F89134EF
:1077B80023F0120343F0120384F89134BDE810401B
:1077C800FFF798BFF40600202DE9F041DFF8AC8000
:1077D80098F81831022B06460D4602D0284BDB6A72
:1077E800984702F0A6FD044628B1022002F097FD52
:1077F800002002F099FD98F81831012B17D102F0FA
:107808009AFD074630B1002002F08AFD002002F000
:107818008CFD3C4602F091FD48B1002002F081FD4C
:10782800002002F083FDBDE8F041FFF763BF002CA4
:10783800F9D1144C94F8902494F81A34BAB90BB1CD
:1078480084F84164304602F017FFD8F82C0007F09E
:10785800FFFAD4F8B4339842E5D30B4807F032FB6B
:1078680094F8913443F0100384F89134DBE70BB1BA
:1078780084F84154284602F0FFFEF1E7008000201A
:10788800E8010108F40600208C0A0020074A10B518
:10789800137843F002031370FFF73AFFBDE8104076
:1078A800034B01220021022006F0E0BF6006002001
:1078B800B9FA0008074A10B5137843F008031370A3
:1078C800FFF726FFBDE81040034B012200210220EC
:1078D80006F0CCBF60060020C9FA00082DE9F04187
:1078E8000F4616461D46804607F0A8FA0B4A0C4C70
:1078F8001378278123F0110343F01103C4E900082A
:10790800137066812573FFF703FFBDE8F041054B4F
:1079180001220021022006F0A9BF00BF6006002056
:107928004C060020D9FA000813B507F087FA0D4B6A
:107938006C461860204607F0D5F994E803000A4A17
:107948000A4B83E80300137843F020031370FFF712
:10795800DFFE074B01220021022002B0BDE81040E3
:1079680006F084BF5C060020600600202C0A002078
:10797800E6FA00082DE9F04192B0064602F0D9FC7B
:10798800002840F05881AD4D95F81831012B09D0E9
:107998002B6BAB4C93B194F80431BBB1042B6FD073
:1079A800032003E002F0C7FC18B10F2012B0BDE8B5
:1079B800F08102F0C2FC0028EAD0F6E7B5F82031E1
:1079C800D4F81C24013B53432B63E4E79D4803F0A0
:1079D80060FA002840F0128194F80C3123802B6B58
:1079E8000C930DF1180895F839308DF83830404669
:1079F80095F81C318DF83A3007F09AF9D5F8283106
:107A0800009302AF98E80600D5F82431384607F00D
:107A180026F997E803000FAB83E80300EB6A0D93A0
:107A280000238DF844302388ADF8463095F830317E
:107A380001228DF839201BB98DF844208DF8393092
:107A4800814B0093814B95F84800A3F179020CA96A
:107A580003F05DFBC0B10B28A8D1D4F8941499B1F8
:107A6800002EA3D0D4F84033794843F02003C4F85B
:107A7800403307F0AFFA764807F072FA002095E72E
:107A8800704803F03AFAA4E795F8487095F9693018
:107A980095F9392095F87D106E4E384603F044FB71
:107AA800009641B2EB6C95F850203846183603F032
:107AB800DFFA0096EB6C95F8502095F9701095F860
:107AC800480003F0D5FAD4F8C413AB6DD4F8DC231E
:107AD8000B44C4F8B033EB6D1344C4F8B43394F8D2
:107AE8000431042B07D02B6E0B44C4F8B0336B6EF3
:107AF8001344C4F8B4330023089395F83031002BAD
:107B080040D100238DF8133095F839308DF82130A5
:107B180095F838308DF82230D5F880300993D5F8AB
:107B280084300A932388ADF82C3095F8303194F8D6
:107B38001B648DF82E3095F84800474B8DF820606F
:107B48000DF1130208A903F0A7FA012384F84134C0
:107B580095F8393084F842349DF8133084F843346A
:107B6800D4F81C34C4F85064C4F84834C4F8583401
:107B780002F0E5FBC8B1D4F81C0402F0F2FBA0B196
:107B8800102013E708A802F0A7FC60B995F939009E
:107B980094F837629DF82070FFF7CEFD3E44B0425E
:107BA800AFD2082002E7132000E795F81831012B1F
:107BB80001D102F0D8FB02F0C5FB0023059394F82D
:107BC800043195F9395094F81B649BB1042B7FF468
:107BD800E7AE05A802F0B4FE58BB94F8183413B108
:107BE800059B013B0593174B05983246E9B202F015
:107BF8000DFF02E0134802F0DDFE08B11120D5E6C2
:107C0800D4F8403394F80C11218043F00203C4F8EF
:107C1800403394F8183411480133DBB284F818342F
:107C280084F845340E4B00259B6AC4F8985498474D
:107C380024E71220BAE60E20B8E600BF0080002034
:107C4800F4060020FC07002030800020880B00206C
:107C58005C0A0020AC0A0020100B0020F606002069
:107C6800E801010873B5134D134E0096EB6C95F8B7
:107C7800502095F9781095F8480003F0F9F995F82F
:107C88003031337595F8480040F2012306F13C0283
:107C98003146738203F0F8F950B196F83C3086F813
:107CA8008230064B00205B6B9847F37C86F8A8303F
:107CB80002B070BD00800020DC0A0020E801010845
:107CC800F8B5324C94F81831012B05460ED0022B2A
:107CD8004ED0002B57D138B9D4E91B0104F17403F5
:107CE80083E803000020F8BD012806D102F02CFB30
:107CF8000028F8D184F81851F5E7022843D1244E1A
:107D080084F8180106F5747CBCE80F0006F57A774C
:107D18000FC79CE8030094F8E92094F8003187E83D
:107D2800030086F8FB53D2B1022B18D1D4F80431E2
:107D38006367C6F8EC3394F87D3094F8082186F828
:107D4800F83394F88C3084F8782086F8F93396F86C
:107D58001B2486F8E82340F20133A6F8FA330023FF
:107D680086F81A340B4BDB6A9847FFF77BFFB9E7B5
:107D780048B9074B84F81801062283F89024054B6C
:107D8800DB6A9847AEE70320ADE700BF008000201C
:107D9800F4060020E8010108F0B5504C504EB4F844
:107DA800DC202287D4E92D0194F8B12084F86920D9
:107DB80004F16C0282E80300D4E92F0104F1740293
:107DC80082E80300B4F8C420A4F87C2091B0D4F869
:107DD800CC20D4F8C810C4F884200025D4F8D020CA
:107DE800C4F888200123A4F82031C4F8801084F84E
:107DF8003051A56284F81B5184F83A5084F81D511B
:107E080084F81E51C4F83451C6F89854A6F818548A
:107E180086F81A54A4F838518DF8183004F5097307
:107E2800039304F50A7394F84800049303A92D4BAF
:107E380084F84551C4E94F55A4F84651059303F019
:107E4800FFF8E36EC6F8D43394F87D3086F8E03353
:107E580094F88C3086F8E1334FF48073A6F8E23357
:107E680086F8D05394F8303186F8E43306F5747701
:107E78000FCF06F57A740FC497E8030040F2012388
:107E880084E80300A6F8FA33D6F8483386F81B547A
:107E9800CDE901551BB15A685B6901920293124BF7
:107EA8000793A3F148020892A3F1140209920F4A1A
:107EB8000B9229330A93A2F19C030C93A2F1980325
:107EC8000D93131D0E9301A902F14C0307A802F5A7
:107ED80099620F9302F022FA11B0F0BD00800020E1
:107EE800F4060020640600205C0B0020E4800020DB
:107EF800F8B50D4F0D4E0C4606F0E4FF3B6B984766
:107F08000B4A96F84800214603F0BEF850B1094DD7
:107F1800706D95F8243485F86A347B6B9847E37C58
:107F280085F89034F8BD00BFE80101080080002002
:107F3800180B0020F40600200F4890F81B3480F836
:107F4800B8330E4B93F8692080F8BB2393F87D2053
:107F580080F8C82393F88C2080F8C92393F830312F
:107F680080F8CC330022A0F8CA2300F56E7100F522
:107F78006070FFF7BDBF00BFF4060020008000203E
:107F8800114890F89034EBB190F81B3480F8D03356
:107F98000E4BDA6EC0F8D42393F87D2080F8E023E6
:107FA80093F88C2080F8E12393F8303180F8E4339B
:107FB8004FF48072A0F8E22300F5747100F5667042
:107FC800FFF796BF704700BFF4060020008000202E
:107FD80070B5344C2421204604F0A0FF636A98420F
:107FE80018BF60624FF01C012F4814BF01250025FF
:107FF80004F094FF636C984218BF60644FF480717A
:108008002A4818BF45F0020504F088FFD4F8483123
:10801800984218BFC4F848014FF0D401244818BF4B
:1080280045F0040504F07AFFD4F82032984218BFCE
:10803800C4F820024FF000011E4818BF45F008059B
:1080480004F06CFFD4F82432984218BFC4F8240214
:108058004FF46071184818BF45F0100504F05EFF32
:10806800D4F8A835984218BFC4F8A8054FF01401F1
:10807800124818BF45F0200504F050FFD4F8C03569
:1080880098420F4B18BFC4F8C005D3F8483318BF3F
:1080980045F040052BB11B691BB12846BDE870406F
:1080A800184770BD008000202880002048800020EC
:1080B8004C8100202482002028820020AC850020EA
:1080C800F40600202DE9F04F8FB04FF00009012B86
:1080D80006460F4690468DF80D90ADF8109002D8E0
:1080E8004C46BC4202D30FB0BDE8F08F305D02F0C1
:1080F80033FA2044B842F6DC335D651C023BEDB22E
:10810800112BF0D801A252F823F000BF5D810008BE
:108118008781000885820008AD8200082B8300084B
:1081280051830008B7830008DF83000865840008CE
:10813800EF800008EF800008B9840008EF8000088D
:10814800EF8000086185000889850008C18500085E
:10815800F5850008052002F0A7FA70B10521002076
:1081680002F068FA725DBA4BE51C0234E4B283F897
:108178005C24325D83F85D24EDB22C46B1E7002320
:108188008DF80E308DF80F308DF814308DF81830CA
:10819800B9F1000F6DD1AF4C4FF0050994F87C2070
:1081A8008DF831206B1E94F839208DF83320334434
:1081B80094F838200B938DF8342094F81A3194F8F9
:1081C80068208DF83520D4F82C218DF832300A92A9
:1081D80073B37B1C5B1BDBB28DF8303006AB0193AD
:1081E80005AB009394F848000DF10F030DF10E0252
:1081F8000AA902F05DFF8DF80D0000F007000728BE
:1082080013D194F939209DF90E3084F839309A4207
:108218009DF80F3084F83830B8BF01229DF814302B
:10822800B8BF84F81D2184F868304FF0000A09E0CF
:108238000523D1E701220DF10D01032002F0A4F876
:108248000AF1010A5FFA8AF29DF81830B3FBF9F1D6
:108258009142EFD82B44DDB26B1EDBB29F420BD9A3
:10826800F25C032A9AD0AF4288BF1D464FF001093D
:1082780083E70534E5B2F9E71D46F7E7735D75490D
:1082880003F00F03012281F81B31023402FA03F3D1
:10829800A1F82031E4B2002204A9042002F074F805
:1082A80025466AE707238DF80D30735DC3F3021284
:1082B80003F00F038DF82830E31CDBB28DF829207A
:1082C800F25C231DDBB2651DF35C0234E4B21B04CF
:1082D80043EA0223325D5F4C13436422534394F80C
:1082E80048000B930AA902F0F2FE00F00703072BDF
:1082F800EDB28DF80D000CD19DF8283084F870305F
:1083080084F878300B9BE36663679DF8293084F81E
:1083180069308DF81000012204A9052002F034F814
:108328002BE74B4BD3F8483363B11B6853B19847DD
:1083380008F03F038DF810008DF81130022204A9CF
:108348000620EBE7FF20F3E703238DF80D30735D7C
:108358008DF81C300AAB0693E31CDBB2A51DF25C5A
:10836800231DDBB206A9F35C1B0443EA0223A21C0B
:10837800D2B20534B25C134364225343E4B20A9385
:1083880000230B93335D8DF83030324B93F848005F
:1083980002F0A3FEC3B20028EDB28DF80D30FFF64F
:1083A800ECAE8DF81030012204A90720B6E7735D02
:1083B80003F00F03012B4FF47A7238BF01235343A4
:1083C800244A0234936503F57A73D365E4B2002234
:1083D80004A9082062E7735D1E4DC3F340128DF8AF
:1083E800152095F84800C3F3001205A903F00F0300
:1083F8008DF814208DF8163002F075FE0234013025
:10840800E4B23FF44DAFBDF81430134AA5F87C3000
:108418009DF816309DF814A0D05CF8F7E5FB022310
:10842800C5F880000AA995F848008DF828308DF81D
:108438002AA002F0F7FD95F93930069040B298422B
:10844800B8BF184685F83900002204A9092025E795
:10845800F406002000800020F3FA000803238DF8BA
:108468000D30735D8DF82830E31CDBB2651DF25CBE
:10847800231DDBB20234F35CE4B21B0443EA02239B
:10848800325D1343642253430B93644B0AA993F858
:10849800480002F02EFEC3B20028EDB28DF80D3070
:1084A800FFF66BAE8DF81030012204A90A2035E7DB
:1084B800092002F0F9F8DFF868B1002849D009214D
:1084C800002002F0B7F80023ADF81E30A31CDBB281
:1084D800F25CE31CDBB216F803A0735D4FEA0A4AAC
:1084E8004AEA022A4AEA030A231DDBB2A51D05341B
:1084F800F35CE4B24AEA036A335D4FF47A72534399
:108508000AAC1B122046ADF81C3006F0EBFB454BBD
:1085180053440693DBF83C3300930DF1180A9AE8AC
:108528000600DBF8383308A806F099FB099B00938E
:1085380094E80600089B504606F076FB9AE803008C
:1085480006F0A8FB01F00AFF0123EDB28BF83834DE
:1085580013E68BF8380410E60C2002F0A5F8002882
:108568003FF40BAE0C21002002F064F82C4B93F87A
:108578009034043B012B7FF600AE01F0EBFEFCE5E6
:10858800A31CDBB2725DF15CE31CDBB2651DF35C1E
:108598000434E4B21B04305D43EA0123134364212D
:1085A800594300F00F0001F0D6FEEDB28DF810002F
:1085B800012204A91120B1E60D2002F075F8002867
:1085C8003FF4DBAD0D21002002F034F8A31CDBB230
:1085D800154AF05C735D1268251D0334E4B243EA62
:1085E8000020315DEDB201F0B8FEC6E5725DA31C56
:1085F800251D0334DBB2E4B2F15C335D1B0443EAAE
:10860800012313436420584301F0A9FEEDB28DF80D
:108618001000012204A9132080E600BF008000207A
:10862800F4060020803DD5124C0600200E4B93F82E
:108638009124920703D593F88F24012A08D90B496E
:1086480091F81A2122B18A6A501C18BF01328A6235
:108658000022A3F8182483F81A24D3F8402322F020
:108668000202C3F840237047F4060020008000206F
:1086780070B5184C1848194D06F024FCD4F840334E
:10868800D4F89804D5F8906023F02003C4F8403358
:1086980038B106F0DDFB864203D2002385F83A3074
:1086A80070BD0120FFF766F90028F9D00B28F7D034
:1086B80095F8393084F84234092094F8183484F84D
:1086C800453484F8410401F0D7FFBDE87040FFF756
:1086D800ADBF00BFF40600205C0A00200080002027
:1086E800094BD3F84023012A0AD008490978C90759
:1086F80008D43AB993F89204013818BF012070479A
:108708000020704701207047F40600206006002012
:10871800034BD3F84003431E58425841704700BFEB
:10872800F40600202DE9F04FA9B0EFF3108272B6DD
:10873800DFF8F0B20021DBF80030CBF8001082F34C
:108748001088B94C002B00F0E180DAB29B06039246
:1087580064D5B64D95F81831022B02D0B44BDB6ABC
:108768009847EFF3108872B6B24F06F067FB3E6881
:10877800D4F8B013361A3144AF4806F02BFCAE4893
:1087880006F0EEFBD4F8B413AC48314406F022FCF2
:10879800AA4806F0E5FB88F3108894F81A34002BF1
:1087A80000F06B81152312A995F848008DF8483020
:1087B80002F038FCD4F8B4130F900144A04806F036
:1087C80009FC9F4806F0CCFB3B6894F81B24EB623D
:1087D8000DAF38468DF870201D9306F0A9FAD5F82C
:1087E8002831009306AE97E80600D5F824313046C4
:1087F80006F035FA96E803001FAB83E80300D4F8C7
:108808001C341E9395F8303195F84800003B18BF8A
:1088180001231CA98DF8713002F00DFC039BDF06C3
:1088280048D5824DDFF81CA2D5F8E42004929BF8C5
:108838000020BAF90A809AF90C90A4F88C840023D5
:1088480063F300020A9384F84434A4F8223484F8C9
:108858002534C4F82834A4F82C3484F82E34C4F809
:10886800303484F82034C4F8343484F83834C4F804
:108878003C346F4B8BF8002094F89024DB6A84F822
:108888008E9484F88F24DAF80470BAF80860984750
:1088980094F88F3413B9694806F014FB314638460A
:1088A80001F045FD8346002800F0EA80A4F87E84A4
:1088B80084F88094039B19071AD55C4B93F81831F8
:1088C800022B02D05A4BDB6A98470220FEF712FFB0
:1088D80084F8410401F0D0FE94F81A3413B101234E
:1088E80084F8193494F8913443F0100384F89134DF
:1088F800039B5A0703D506210520FEF765FF039B56
:108908009B0703D504210320FEF75EFF01F02DFD30
:1089180094F89124D7065FD5002384F89234D4F8CC
:1089280040331E0644BF23F08203C4F8403312F0DC
:10893800050F00F0FB820B2001F0B6FE002800F0C6
:10894800F58294F89134DD0700F1F082580740F180
:108958000783D4F8403323F00203C4F84033D4F833
:10896800402382BB94F8915415F001011EBF2B4699
:1089780062F3000384F8913494F891345E0744BF9D
:108988006FF3820384F89134012384F8923421B17F
:10899800D4F844332C481B6898476D070BD52B48EF
:1089A80001F08EFE01F0BCFE28B194F8913443F03A
:1089B800040384F8913401F0C6FC94F891346FF301
:1089C800041384F89134012384F8923494F8913490
:1089D80043F0200384F8913494F8913418070AD5A9
:1089E8006FF3C3031A4984F89134D4F84433A1F1DE
:1089F8002400DB68984794F8913499070AD56FF3F7
:108A08004103134984F89134D4F84433A1F16C003C
:108A18005B68984794F89034022B1BD1FFF722F932
:108A280018E000BF60060020F40600200080002047
:108A3800E80101085C060020740A00208C0A002066
:108A4800F40A00204C060020340B0020480B0020BC
:108A5800800B002094F891349A0640F1C4826FF399
:108A6800451384F89134D4F84033002B40F0BB828E
:108A780029B0BDE8F04FFFF7ABBA84F84134A3E65C
:108A880095F81831012B0CD101F055FC804668B1DE
:108A9800584601F045FC584601F047FC042384F889
:108AA8008F347EB9012384F821344FE101F045FC6D
:108AB8000028F6D0404601F034FC404601F036FC70
:108AC8000523ECE73B7805935B09013B062B00F295
:108AD8001782DFE813F007001502950015029200CF
:108AE80015020602102EDDD995F830311297F6B22C
:108AF8008DF84C60002BD5D11CA804F021F912AADE
:108B08001CA9FF2002F09EF89DF85830C3F3030318
:108B180007468DF82C3095F8480095F87D308DF88B
:108B28002D3007220BA902F090FA002F5DD1002802
:108B38005BD09DF853309DF852201599C5F8E41084
:108B48001B0443EA02239DF8512002201343C5F871
:108B5800E03004F003F99DF8583095F8480085F89E
:108B68002E71C3F30212C3F3030385F8703085F83E
:108B780078309DF8593085F86920012B38BF0123DA
:108B88004FF47A725343AB651344EB650DF15A0306
:108B98004FF001081093113E94F81B348DF83C30C7
:108BA8000FA985F868808DF8446002F056FA022310
:108BB800404685F8303101F077FD18B14146384616
:108BC80001F038FD94F88F34012B00F2A78194F856
:108BD8001A34002B40F09A8194F8913443F0100332
:108BE80084F89134FEF786FD64E6012001F05CFD0F
:108BF8000028E7D001210720E2E7012384F8203488
:108C080095F87D308DF82E3094F824348DF82D3079
:108C180095F88C3095F848000D330BA98DF82C3059
:108C280002F000FAA6F10D031BB2099023EAE373E0
:108C380000B283423FF736AF0B2E7FF633AFBA4B05
:108C480025931CA8FF231C978DF874608DF8983025
:108C580002F0C4F8074600287FF424AF95F81831CD
:108C6800012B13D101F067FB002872D0384601F0C0
:108C780057FB384601F059FB04239DF87C101E98D9
:108C880084F88F34C1F3001101F06EFB9DF87C303D
:108C98001E99C4F8341413F00F0203D09DF8900005
:108CA800002862D19DF89800002861D0002A7FF43E
:108CB800F9AE9DF89020002A14BF4FF003084FF03A
:108CC800020800220A92D5F8EC2095F8E9009142B2
:108CD80051D100284FD0D5F80C1195F8EAB00968A1
:108CE8000A9195F81811022902D1032184F88F14EA
:108CF800B8F1030F7FF4D6AE13F0600F7FF4D2AE55
:108D08000492012795F82E31BBF1000F36D0BBF144
:108D1800010F13D1012B33D16FF0090646FA08F67B
:108D280006F00106C6F10206F6B2BDF87E100AAAE0
:108D3800304601F011FE38B3072823D0012384F808
:108D480021340A9BC4F83034C4F86C34FEF720FD93
:108D5800B0E501F0F2FA002898D0384601F0E1FABF
:108D6800384601F0E3FA052387E74FF00008A8E743
:108D78004FF00108A5E74FF0010BC3E70426D4E73D
:108D88000326D2E70823DAE71CAB009304990A9B71
:108D98003246584601F0A2FE20B1022814BF0B2328
:108DA8000A2380E60A9BC4F83034C4F86C349DF872
:108DB8007C3084F82104C3F3401384F82E3484F8FB
:108DC800443494F88F3484F82274012B9EBF012216
:108DD800A86285F81E21012FC4F8280484F82C0401
:108DE80084F8410438D1022284F8202495F83A20E6
:108DF800002A4AD19DF87C20D60646D4012B94F847
:108E080040149DF87C2005D8012901D1900601D590
:108E180001F04CFBB8F1020F94F88F3443D0B8F14D
:108E2800030F0AD09DF87C10B8F1010F4A4601F0F3
:108E38000F0120A83BD0FFF745F99DF8903084F842
:108E48002334259BC4F828349DF8983084F82C34B2
:108E5800012384F82D3430E0059A02F0E002A02ABC
:108E68001BD195F82E11012285F83A2009B92799C6
:108E78006963012B84F8202407D9D5F89020C4F819
:108E88003C24DAF80020C4F8982495F81821002A20
:108E9800B4D1012284F82524B0E7002285F83A20CD
:108EA80084F82024A6E79DF8981025984A46FFF7ED
:108EB80009F99DF8903084F823349DF89020E02A31
:108EC80008D195F81F312BB984F82324C4F8283425
:108ED800A4F82C3494F8913443F0020384F89134C4
:108EE80070E6114D013EB2B2791C284604F000F834
:108EF8000323A4F82034C4F8285484F82C64E9E740
:108F0800012384F82134FEF743FC5BE694F84434EB
:108F1800002B3FF461AE0020FEF726FC94F88F3456
:108F2800022B3FF45FAE57E62C09002094F89134E9
:108F3800590715D5012001F0B7FB60B1012001F0F8
:108F48008BFB08B984F81804D4F8403323F00203E3
:108F5800C4F8403304E0062001F0A6FB0028F3D152
:108F680094F89134DA077FF5FAAC94F840240AB102
:108F7800032A18D11D4A94F8181492F868209142CF
:108F880005D29B0723D594F88F34012B1FD8184896
:108F980005F098FFD4F8403323F02003C4F8403399
:108FA800FFF744FBDBE4012A11D194F81924002AC5
:108FB8003FF4D5AC0D4A94F8181492F86820914201
:108FC800E5D29F0703D594F84434002BDFD194F8F9
:108FD800913400206FF3041384F8913484F8190451
:108FE800FFF746FBBBE429B0BDE8F08F0080002006
:108FF8005C0A00202DE9F04F89468DB0904607465F
:10900800002800F08F81002900F08C810368002B74
:1090180000F088814368002B00F084818368002B6E
:1090280000F08081C368002B00F07C81104601F0BD
:10903800F5FF002800F07881BD4CBE4D384601F0A0
:10904800AFFA40F2C4520021204603F065FF40F217
:109058001C520021284603F05FFFB74BC4F82C319F
:1090680004F50973089304F50A730026404609932A
:1090780008A9B24B84F848800A9384F8186184F8E8
:109088008C608DF82C6001F0DBFF0F2306A994F8A3
:1090980048008DF8183001F0C5FF801B18BF01206B
:1090A8004FF00A0B84F81C0106A994F848008DF8C3
:1090B80018B001F0B7FF4FF0060A84F8DC0006A9E3
:1090C80094F848008DF818A001F0ACFF102384F83C
:1090D800DD0006A994F848008DF8183001F0A2FFC9
:1090E8001123C4F89C0006A994F848008DF818309C
:1090F80001F098FF1223C4F8A00006A994F84800CC
:109108008DF8183001F08EFF1323C4F8A40006A9C7
:1091180094F848008DF8183001F084FF1423C4F83F
:10912800A80006A994F848008DF8183001F07AFFD5
:109138001623C4F8AC0006A994F848008DF8183036
:1091480001F070FF172384F8B10006A994F84800CD
:109158008DF8183001F066FF18230DEB0301C4F8F1
:10916800B400C4F8BC0094F848008DF8183001F039
:1091780059FFC0B21D2384F8B80084F8C00006A9BE
:1091880094F848008DF8183001F04CFF1E2384F83D
:10919800C40006A994F848008DF8183001F042FF81
:1091A8001F2384F8C50006A994F848008DF81830E4
:1091B80001F038FF2023C4F8C80006A994F8480035
:1091C8008DF8183001F02EFF0B23C4F8CC0006A947
:1091D80094F848008DF8183001F024FF0C2306A9F4
:1091E800A4F8D00094F848008DF8183001F01AFF60
:1091F800D4F89C306365D4F8A030A365D4F8A430C3
:10920800E365D4F8A83023664FF00108D4F8AC30F1
:109218000590A4F8D200636684F8B080C4F894B0CE
:1092280084F898A0C4F84CB084F850A084F86880FA
:1092380084F81F81C5F84893FEF7AEFDC5F844735E
:10924800C4E90B663E4B84F8198185F89164C5F82A
:10925800408332464FF0FF31009605F55A7005F00D
:10926800D3FD384B009632464FF0FF3105F560705C
:1092780005F0CAFD344B009632464FF0FF3105F534
:10928800667005F0C1FD02AF304B009632464FF0D4
:10929800FF3105F5806005F0B7FD384605F048FD5B
:1092A80097E8030004F5927383E80300284B294FDD
:1092B8001E60294BC5F84C33284BC5F85433284B4E
:1092C800C5F85C33274BC5F85033274BC5F85833DE
:1092D80005F553703B68984704F5A67003F04CFBFE
:1092E80020B1112630460DB0BDE8F08F204601F0C0
:1092F80003FB0028F5D101F039F8B8B91B4801F093
:109308004DFB06460028ECD17B69984703F0CEFD5B
:10931800BB6D94F819019847FB6A9847012385F8B3
:109328009234DFE70326DDE70926DBE71326D9E7D2
:1093380000800020F40600200004000164060020DC
:1093480079860008417F0008897F00087177000846
:1093580060060020E801010831790008E578000876
:109368002D770008BD78000895780008E88000206F
:1093780008B5034B0020C3F84003FEF7BBF908BD4E
:10938800F406002010B5FFF7ABF90A4C60B90A4B98
:1093980093F81831022B02D1084BDB6A9847012356
:1093A800C4F84033002010BDD4F84003013818BF7A
:1093B8000120F8E7F406002000800020E8010108F9
:1093C80038B5124C204605F07DFD04F1180005F073
:1093D80079FD04F1300005F075FD04F1980005F001
:1093E80071FD00F0AFFF0A4B0025DB6A984744F88F
:1093F800285CFEF7EDFD0749074840F2C45203F028
:1094080077FD012344F8283C284638BD5C0A002033
:10941800E801010800800020C485002070B52E4BAB
:109428008AB0054693F8DD008DF8090093F8DC0052
:109438008DF80A0029489A6A90F8180403920026C1
:109448008DF80B0004960C46002940D00692D3F8FC
:10945800882007921A8F93F81A118DF8151052BAAE
:10946800ADF8202093F87C2093F848308DF824300C
:1094780003AB8DF822008DF8232000930DF10A022A
:109488000DF10B030DF1090105A88DF8146000F02A
:10949800D7FE9DF90900FEF74FF9607004A801F0A6
:1094A8001BF8B0B9049A0F2A0DD863789A420AD8E3
:1094B8001544AB42A3EB02012CBF00200120217010
:1094C800C0000AB070BD002323700820F9E703200C
:1094D800F7E71320F5E700BF00800020F40600201E
:1094E8001FB50446002800F010810378412B00F2D4
:1094F8000781DFE813F0420049004D005100550094
:1095080059005E0005010501050105010501050178
:1095180005010501650069006D0078007F00820083
:1095280085008A0088008C009000930096009900BE
:109538009C009F00AE00B200BA00B600BE00C10099
:10954800C500CE00CA00CC000501D2000501050106
:1095580005010501050105010501050105010501D3
:1095680005010501050105010501DA00DE00E2003B
:10957800E700EB00EF00F300FC00664B93F81831AE
:109588002371002004B010BD624B93F83031F7E727
:10959800406803F08FFBF4E7406803F0D1FBF0E785
:1095A8005C4B93F81A31EBE75A4BD3F8E030636021
:1095B800E7E7584B011D93F8300103F0D9FBE0E7CA
:1095C800544B93F81931DBE7524B93F88C30D7E7BB
:1095D8001C238DF808304F4B02A993F8480001F07E
:1095E80021FD6060CDE74C4B043493E8030084E828
:1095F8000300C6E7494B0434F7E7494B0434F4E762
:10960800484B0434F1E71A23E3E71923E1E7414B18
:1096180093F86830B4E73F4B5B6DC8E73D4B9B6DF3
:10962800C5E73C4BDB6DC2E73A4B1B6EBFE7394BD6
:109638005B6EBCE702238DF80830364B02A993F81D
:109648007C2093F848008DF80A2001F0EBFC20718B
:1096580097E7304B93F8DD3092E72E4B93F839308B
:109668008EE72C4B93F8DC308AE72A4B93F8383096
:1096780086E7284BDB6C9AE7264B93F850307FE758
:10968800244BD3F8843063607BE7224B8FE7264B6B
:109698008DE7204BD3F8CC30F5E71E4BD3F82C31AF
:1096A800436001F04DFDA0606BE71A4BD3F8903092
:1096B8007DE7184B93F81F3162E7164BB3F88830F3
:1096C800A3805EE7134BB3F88A30F9E7114BB3F880
:1096D800D030F5E70F4BB3F8D230F1E70D4B93F8E4
:1096E80048200AB1062A12D1B3F8A035E8E7094B99
:1096F80093F848200AB1062A09D1D3F8A43556E7C9
:1097080004B0BDE8104000F021BE03203AE718205D
:1097180038E700BF008000206C800020B480002063
:1097280074800020BC800020C48500207FB50446DA
:1097380010B9032004B070BDA34DD5F840339A0783
:1097480000F16F820278412A00F26882DFE812F0A5
:109758004200470055005B005F0064006900760026
:10976800810087008D00930099009F00A500AB0041
:10977800B5006602BA00DC00EF00160138012901C5
:1097880042014B014F01530157015B0166025F0122
:10979800710199018701AB01B101B801BD01C20195
:1097A80066022802660266026602660266026602AF
:1097B8006602660266026602660266026602660261
:1097C80066026602340239023E02430248024D0232
:1097D80052025C020079FEF773FA30B1AAE7037906
:1097E800022BA6D0794A82F8303195F8913443F0AB
:1097F800200385F8913400209CE7406803F04CFA78
:109808000028F2D095E7406803F08AFAF8E76F4B32
:10981800027983F81A21E8E76C4B4268C3F8E02024
:10982800E3E76A4E416896F8300103F097FA00289A
:109838007FF47FAF6368C6F8E430D6E74168002953
:109848003FF477AF002001F0DDF90028CDD01120DA
:1098580070E7416800293FF46CAF0120F3E74168E5
:1098680000293FF466AF0820EDE7416800293FF47E
:1098780060AF0920E7E7416800293FF45AAF0C20A0
:10988800E1E7416800293FF454AF0D20DBE7416868
:1098980000293FF44EAF0E20D5E7416800293FF478
:1098A80048AF0F20CFE74A4C484B007983F819019D
:1098B800A36D9847E36A984797E7444B027983F882
:1098C8008C2092E7414E037A8DF8043096F84800D0
:1098D80096F87D308DF80530072201A901F0B5FB17
:1098E80000283FF426AF636896F8480001930022E9
:1098F80001A901F0AAFB00283FF41BAF6C36D4E99C
:10990800010186E8030070E7304E037A8DF80430D1
:1099180096F8480096F87D308DF80530072201A9A1
:1099280001F093FB00283FF404AFB436E7E7274E75
:10993800037A8DF8043096F8480096F87D308DF853
:109948000530072201A901F080FB00283FF4F1AEA1
:10995800D4E9010106F1740383E8030096F818318D
:10996800022B7FF442AF96F83031002B3FF43DAF25
:10997800174BDB6A9847FEF775F936E7134E037AFB
:109988008DF8043096F8480096F87D308DF805304B
:10999800072201A901F059FB00283FF4CAAEBC36E2
:1099A800ADE74368029301238DF80C30074B02A9F9
:1099B80093F8480001F056FB00287FF416AFB8E68C
:1099C800436802930023EFE7F4060020008000209C
:1099D800E801010803795A1E0E2A3FF6AAAE934AF7
:1099E80082F8683001E7914B42685A65FDE68F4B73
:1099F80042689A65F9E68D4B4268DA65F5E68B4B65
:109A080042681A66F1E6894B42685A66EDE6874C69
:109A1800037994F848008DF80430062201A901F072
:109A280014FB00283FF485AE9DF8043084F8DD303F
:109A3800DBE67E4C03798DF8043094F8480094F8FE
:109A48007C308DF80630052201A901F0FEFA0028C5
:109A58003FF46FAE9DF8043084F83930C5E6734C96
:109A6800037994F848008DF804300A2201A901F01E
:109A7800ECFA00283FF45DAE9DF8043084F8DC3041
:109A8800B3E66A4C037994F848008DF8043009224B
:109A980001A901F0DAFA00283FF44BAE9DF8043032
:109AA80084F83830A1E6614B4268C3F89420DA6440
:109AB8009BE65E4B027983F8982083F8502094E661
:109AC8005A4B4268C3F884208FE6584B4268C3F863
:109AD800CC208AE6012B40F0A480554C2421204656
:109AE80003F01CFA636A984201D0172022E61C2171
:109AF80004F1280003F012FA636C9842F5D14FF490
:109B0800807104F1480003F009FAD4F8483198420A
:109B1800EBD1D42104F5A67003F000FAD4F8203272
:109B28009842E2D1002104F5097003F0F7F9D4F85E
:109B380024329842D9D14FF4607104F50A7003F0C9
:109B4800EDF9D4F8A8359842CFD1142104F2AC50DD
:109B580003F0E4F9D4F8C0359842C6D1334E214613
:109B6800304640F2C45203F0C3F9204640F2C452D2
:109B7800002103F0D1F995F81B3485F8E833736FA9
:109B8800C5F8EC3396F87D3085F8F83340F20123B8
:109B9800A5F8FA33274B96F819019B6D984724E6E8
:109BA8008379012B3FF6C5AD204B42684068C3F866
:109BB8002C2100F0BDFE48E61C4B4268C3F89020FB
:109BC80013E61A4B027983F81F210EE6174B828899
:109BD800A3F8882009E6154B8288A3F88A2004E6B2
:109BE800124B8288A3F8D020FFE5104B8288A3F897
:109BF800D220FAE50D4B93F848200AB1062A12D173
:109C0800A288A3F8A025F0E5084B93F848200AB1EC
:109C1800062A08D16268C3F8A425E6E500F098FB97
:109C2800DBE5012086E5182084E500BF00800020E0
:109C3800C4850020E80101082DE9F04387B000231E
:109C4800ADF800300646002800F0EE800361FEF70C
:109C580047FD20B10124204607B0BDE8F08300F09D
:109C680065FD0028F6D100F05BFD014618B96F4884
:109C7800142203F051F96E4D95F89134012243F006
:109C8800040385F8552485F8913433788DF8043029
:109C98000021013B8DF80520ADF806100C2B00F2D1
:109CA800BB80DFE803F007B9B9B97982B9B990B9CF
:109CB800AD9AA900D5F8407317F02007CAD196F8D5
:109CC8000480B8F1020F46D1DFF868815A4CFEF7DC
:109CD80063F896F9051098F848003A4601F00FFA2B
:109CE80088F83900B37988F83830384607238DF872
:109CF8000530FDF7E5FFFF2304F58670A5F80C3164
:109D0800C5F8084185F8047103F01AF804F58A705B
:109D180002F0D0FF3846FDF72DFE0446002839D062
:109D280096F9051098F84800012201F0E8F988F83A
:109D38003900D5F894343361002C71D000F0F0FC70
:109D4800002888D195F8913485F81A0460F38203C5
:109D580085F891347FE7B8F1010F4FF00204E8D19C
:109D6800DFF8D0908DF8144099F8480089F81D71F3
:109D780002A901F065F9337989F830318DF8057059
:109D88008DF80680FDF7C4FC95F8913443F0100374
:109D980085F891340024CCE700226946022000F0BF
:109DA800F3FA0028F6D01324C3E7244BB288DB6B00
:109DB80096F90C10B0689847D5F8403343F0020381
:109DC800C5F84033E6E702A90D2000F053FB002850
:109DD800E0D0002269460D20E1E7164B93F81831D0
:109DE800D3B9347904F0070000F0ABFA8DF80040DD
:109DF800012269461020D2E7002269461220CEE7E8
:109E08008DF8072000F08EFA044638B900F087FA7A
:109E1800204600F089FABDE702248AE7012488E792
:109E280001A800F0D1FB16E7032414E7480B002033
:109E3800F406002000800020F6060020E801010852
:109E48002DE9F04F99B08046059118B9032019B053
:109E5800BDE8F08F00230361FEF742FC04460028AA
:109E680040F0A58046460FCE0EAD0FC514225248CD
:109E780098F800A0B8F80C7098F90EB04F4E21462B
:109E880003F04AF84E4B012283F8412496F830211A
:109E9800022A25460BD196F81821022A07D196F8EE
:109EA8001E2122B9BAF1010F38BF4FF0010ABAF1E9
:109EB800010F2BD0BAF1030F2AD0BAF1000F33D11A
:109EC80002229DF83C30DDF84090029362F347157A
:109ED800012496F87C108DF8321002220CA996F80D
:109EE80048008DF8302001F09DF896F81A3196F860
:109EF80030C196F81D1140B2002B63D0BCF1010FA0
:109F080057D1002955D1002C61D153E00422D8E75C
:109F18000023DDF83C90BDF840709DF942B00293F3
:109F280065F01F050124D4E74FF0000BD946CDF8A2
:109F380008B0CEE74FF0010084F81A04D2E005F229
:109F48009A420BA900F0D4FA002800F015811320DA
:109F5800049B33871A4B002283F81A2423E105F265
:109F68009A452A460BA900F0C3FA0028EFD10B9BAB
:109F780084F82801C4F82C5184F83031FCE0B9F198
:109F8800000F00F0F980002A00F0F6804946E01C36
:109F980002F0AEFF94F8373201332380ECE0122050
:109FA800D6E70220D4E70720D4E71320D2E7012020
:109FB8004DE7FCB90220F6E0340B002000800020B9
:109FC800F4060020002CF5D05845B8BF584696F83E
:109FD8007C308DF82000052296F848008DF8223054
:109FE80008A901F032F800283FF430AF9DF820307E
:109FF80086F839306F4A704BD2F89804D3F89040FD
:10A0080038B104F025FF6C4B84423CBF002283F832
:10A018003A20198F1A8F93F830010491996A09919F
:10A0280052BA0028BFD093F81B0100B9186393F8FF
:10A038001801ADF85820013893F87C2093F81A419C
:10A048001491D0F1000BD3F888108DF85B204BEBFE
:10A05800000B93F8482093F83A0093F868308DF88D
:10A068005A3009AB0093554B03904FF001008DF81F
:10A078004C0015918DF85C20A3F12F01A3F130025B
:10A0880013A88DF84D4000F0DBF8039B4FEA0B1B3B
:10A098004BEA431B00264BEA801B4BEAC413B1452D
:10A0A800444C039308BF37463A46494604F59C702A
:10A0B800CDE90A669B46268084F81A6402F018FFE8
:10A0C800E9B2A570C5F34215FAB2042D3A4E039BC6
:10A0D80084F837223FF42EAF072D3FF450AF022DFE
:10A0E8007FF45FAF364D84F80D110420029984F88F
:10A0F8000401FF2084F80C0184F8281184F8143135
:10A10800D6F8E410C4F8085105F59B730AA8C4F8FA
:10A11800101184F83021C4F82C3100F011FC00280B
:10A128007FF43DAF0A9BA4F844040BA8A4F81631A9
:10A13800C4F84C3400F0D0F900287FF408AF0B9B2A
:10A14800D3B196F93900FDF7F7FA94F83732002BB6
:10A158003FF405AF0B9B0F2B3FF6F1AE05F58B7265
:10A168000BA90F2000F0C4F900287FF4F0AE0B9B78
:10A1780063F3030B84F814B10598FDF7FBFB002883
:10A188007FF4E6AE099B86F83A00B36200F080F9E6
:10A1980000287FF40AAF94F8913484F840A443F07F
:10A1A800010384F89134034BD3F89434C8F8103081
:10A1B8004DE600BFF40600200080002068800020E3
:10A1C800F606002037B50B4D8DF8040004460F2223
:10A1D80095F8480001A900F038FF40B1064A85F813
:10A1E8001C4192F8913443F0200382F8913403B073
:10A1F80030BD00BF00800020F406002010B5FFF736
:10A20800C1F8044688B90A4804F05CFE094804F01D
:10A2180059FE094804F056FE00F094F8FDF7BCFD1D
:10A22800064BDB6A9847204610BD0124FBE700BFB8
:10A238005C0A0020740A00208C0A0020E80101084A
:10A248002DE9F04F8BB047780093149B90F90C8060
:10A2580090F90D6090F80EB08A464168196004467E
:10A268009146002F58D002238DF8103004A9C37BE3
:10A27800007C8DF8123000F0D5FEB4F808C0618972
:10A2880043B26068984545466144B8BF1D4660457D
:10A2980034BF00270127884209D30A218DF81010FE
:10A2A800207C019304A900F0BDFE019B46B2B4F8DE
:10A2B80008C0608961680CEB400E714519D3A1EBA9
:10A2C8000C01B1FBF0FC00FB1C1191B9984503DCB3
:10A2D8002378CBB94FF0010B21238DF81030207C67
:10A2E800E37B8DF8115004A98DF8123000F09AFE26
:10A2F80045B2009B8AF80050384689F8006083F818
:10A3080000B00BB0BDE8F08F0223207C8DF824301C
:10A3180006A900F095FEDDE74546EAE77047704775
:10A32800704770470020704770477047704700209B
:10A3380070470020704700207047002070470020B9
:10A348007047704770477047022070470220704777
:10A358000220704770470020704770477047002000
:10A3680070470020704770477047704710B5054C1C
:10A378004FF403722046002102F0CEFD0020C4E90C
:10A38800000010BD100C00202DE9F84381469046CE
:10A3980000293CD01F4C2023224604F1100012F85B
:10A3A800017F6FBB8242FAD11B4E3368013403B977
:10A3B8003460736803B11C6000252560C4F8088008
:10A3C80074601FFA88F284F80490601D02F090FD12
:10A3D800B9F1110F4FF0000398BF104D6373D6F811
:10A3E800083298BF25FA09F503F1010398BF05F073
:10A3F800010543442573C6F808323846BDE8F8839A
:10A40800013B13F0FF030446C6D10227F5E70127F5
:10A41800F3E700BF170C0020100C002020070200F3
:10A4280010B518B3124A1368984204D10368136030
:10A43800002305E00B46002BFAD019688842F9D1B1
:10A448005168884208BF53600BB101681960D2F89F
:10A4580008328168013B00245B1A04602146C2F877
:10A468000832102202F058FD204610BD0120FCE7FA
:10A47800100C0020054B1B6813B11A798242FAD1DF
:10A48800002B0B600CBF032000207047100C00202D
:10A4980010B5054B186800B910BD037B04680BB9EB
:10A4A800FFF7BEFF2046F6E7100C002038B5084B32
:10A4B800084C186800B938BD03790568112B05D810
:10A4C80024FA03F3DB0701D5FFF7AAFF2846F1E7D3
:10A4D800100C00202007020028B1044BD3F80832E2
:10A4E8000360002070470120704700BF100C002057
:10A4F8002DE9F04107460E46154642B339B3154BD0
:10A508001C6800232CB93046FFF7E6FF0020BDE8A1
:10A51800F081A268F91A0132914215D32279EA54DE
:10A52800581C22895FFA80F8611D55FA80F002F004
:10A53800DFFCA368246898445FFA88F3E2E72046C2
:10A548002568FFF76DFF2C46002CF8D1DBE70120CA
:10A55800DDE700BF100C00200238C0B211289ABFF6
:10A56800014B185C0020704703FB000830B50B4B0B
:10A5780093F820200446084672B100211C33057860
:10A58800A54208D001319842CDB214BF043010382A
:10A59800AA42F4D8002030BD1046FCE71C0E00206B
:10A5A80010B5084C00232060142204F10C00FF2190
:10A5B80084F82030C4E9010002F0AEFC012384F8DD
:10A5C800213010BD1C0E002010B50E4A92F8201044
:10A5D800042915D8936804781C7044785C70C47892
:10A5E800807898700131DC7082F8201002F11C012B
:10A5F8008B4214BF043302F10C039360012010BD99
:10A608000020FCE71C0E0020094B93F8200068B1DD
:10A618005A6803F11C018A4200F1FF3014BF04326A
:10A6280003F10C0283F820005A600120704700BF34
:10A638001C0E002010B5074B93F82020044608464E
:10A6480032B15968FFF792FF10B10123447083704B
:10A6580010BD00BF1C0E002008B5064B93F8202043
:10A668002AB15968FFF782FF08B1407808BD012078
:10A67800FCE700BF1C0E002030B50A4A92F82010F3
:10A68800536882F8210061B1916801241C32DD7899
:10A69800587005B99C70934214BF0433103B99421B
:10A6A800F5D130BD1C0E002008B5044B5968FFF7E2
:10A6B8005DFF003818BF012008BD00BF1C0E002038
:10A6C800F7B50422154E044600210DEB020096F85A
:10A6D800207002F021FC0025EBB29F4201D803B0A4
:10A6E800F0BD7368197821705A786270987838B11B
:10A6F800336820469B689847FFF786FF0135EBE7EC
:10A70800DB788DF804108DF805208DF80730FFF7F9
:10A718007BFF01A8FFF758FFF0E700BF1C0E0020E1
:10A72800014B93F8200070471C0E0020034B93F850
:10A738002000042894BF0020012070471C0E002030
:10A748001FB50024CDE90244C41F8DF800408DF8E0
:10A7580001100C0AADF80420090C120C8DF8031036
:10A768008DF806208DF8073002461B0A012168463D
:10A778008DF802408DF8083002F029FA002818BF39
:10A788000E2004B010BD2DE9F04188B090460D466A
:10A798000F9A0746002847D000240121CDE9044438
:10A7A8008DF810109DF838108DF81510ADF816308A
:10A7B800190CCDE900441B0ECDE902448DF819307F
:10A7C800ADF81A20130C120E07948DF818108DF896
:10A7D8001C308DF81D20E3B21E01002DF6B203DCFB
:10A7E800002008B0BDE8F081013310218DF81F303A
:10A7F80042466B460DEB010002F07FF90346A8B90B
:10A80800102D28463E44A8BF10206946327811F81A
:10A8180001CB013382EA0C02984206F8012BF5DCE1
:10A82800103D2DB20134D6E70920DAE70E20D8E72B
:10A838000138032815D8DFE800F002080C100A4B8D
:10A848001B681B690B6000207047074B1B685B691E
:10A85800F8E7054B1B689B69F4E7034B1B68DB694A
:10A86800F0E70520704700BF400E00202DE9F041B9
:10A87800C4B00C464A9E17461D468046B8B3B1F58B
:10A88800807F36D84FF488720021684602F044FB76
:10A89800492300934FF48073ADF804302B0C8DF8E6
:10A8A8000830330CADF80650ADF80A608DF80C305E
:10A8B80022460023414604A82D0E360E8DF80E3090
:10A8C8008DF809508DF80D608DF80F4002F010FBDF
:10A8D80004F110014B9A3B4689B2684602F0F7F83A
:10A8E80010B1012818BF0E2044B0BDE8F08109203E
:10A8F800FAE70D20F8E7000010B590B10A4C2822BD
:10A908000021206002F008FB2368084A1A60002032
:10A918004FF0FF32C3E90302C3E90522C3E9072266
:10A9280010BD0820FCE700BF400E00200001010117
:10A93800024B1B6818600020704700BF400E0020C3
:10A9480030B1044B1B68DB6801330360002070479B
:10A9580009207047400E002013B500230C460193D0
:10A96800CAB101A9FFF764FF18B9019B591C02D1AC
:10A97800146002B010BD99B2611A002901DD5C189B
:10A98800F6E702D113600720F3E71B0C1B0403F55D
:10A9980080331C44ECE70920EBE7000028B1044BA6
:10A9A8001B681C334362002070470920704700BFB2
:10A9B800400E00201FB5044600B3002303A80393EC
:10A9C80002F05CF9104ABDF80C30126820469380FA
:10A9D800E38200F05EFA98B904F118030093216845
:10A9E8000123132202F068F860B9204600F051FAFA
:10A9F800003818BF0120000104B010BD0920FBE792
:10AA08001020F9E70E20F7E7400E0020F0B50546C4
:10AA180087B01C4613B9092007B0F0BD2E4E336825
:10AA2800DB68834255D894F82020002A0CBF0822FE
:10AA38000922834205D3204600F05FFA68B110204E
:10AA4800EAE7002301900093A36894F82810606A4D
:10AA5800FFF799FE0028EED0DEE723792168B4F8E5
:10AA680008C0A768043B9AB20029D4D0B2F5807F09
:10AA78002DD8ADF80EC08DF817304FEA174C04F1F9
:10AA88002C033F0E8DF8117000932F0C08234FF004
:10AA9800490EADF80C008DF814708DF816002F0EC5
:10AAA8000DEB0300CDF808E08DF810C0ADF812509A
:10AAB8008DF8157002F000F808B10E20ACE72046BA
:10AAC80000F01BFA0028BAD13368DD60A4E70D2036
:10AAD800A2E70620A0E700BF400E00202DE9FF41B5
:10AAE8000A9D80460F4616461C46002D5AD0002364
:10AAF80003A910460393FFF79BFE18B1062004B084
:10AB0800BDE8F081039B9C4201D80133F6D1284669
:10AB180000F064F9002847D1264B1A78424503D043
:10AB28001A79424542D10120AA68BA4240D103EBC2
:10AB38008002EB6A92F801802979CDE90043043953
:10AB4800927828683B4689B2FFF790FE0028D6D154
:10AB580095F820300194002B4FF00103009314BFA7
:10AB68004246082295F82810686A3B46FFF70BFE14
:10AB78000028C4D1013E032EC1D8DFE806F0020741
:10AB88000B0F0D4B1B681C611C62B8E70A4B1B6856
:10AB98005C61F9E7084B1B689C61F5E7064B1B688D
:10ABA800DC61ACE70920AAE70F20A8E70B20A6E79D
:10ABB8000220A4E7F0000020400E00201FB50B295A
:10ABC8004FF00003CDE90033CDE902330A4607D040
:10ABD8000C2914D00A2910D00A2005B05DF804FB0E
:10ABE800012802D120238DF800300021684601F0A9
:10ABF800EEFF002818BF0E20EFE73023F3E70B2104
:10AC0800F4E7000038B5054601F0DCFF044610B152
:10AC18000E24204638BD002DFBD1094B1B680B21A3
:10AC28009878FFF7CBFF0028F2D10C21FFF7C6FF79
:10AC38000028EDD10A21FFF7C1FF0028E9D0E7E796
:10AC4800400E00202DE9F04380468FB00C46174691
:10AC5800002A6BD0002969D0002529461D2206A8A4
:10AC6800059504F035FB8DF81350344D2B680DF124
:10AC780014099E88CDF804900DF1130302933B79D3
:10AC880000933B6832462146404601F0BCFF00284D
:10AC98004ED138683A79494602F02AF9384600F028
:10ACA8004FF8002846D13C7AFA79BB79240444EA63
:10ACB80002241C432B689A6894423DD99C609DF8F5
:10ACC80013000B21FFF77AFF034658BB0C21FFF74F
:10ACD80075FF034630BB0A21FFF770FF034608BB28
:10ACE8007B7ABA7AFF7A3F0447EA02271F433A463B
:10ACF800334621460920FFF723FD034690B9334622
:10AD08003A4621460820FFF71BFD034650B92A683A
:10AD18009DF8131091700021D1604FF0FF31C2E906
:10AD28000411916118460FB0BDE8F0830923F9E7D3
:10AD38000E23F7E70F23F5E70323F3E7400E002080
:10AD480010B50446002845D00168002942D011F802
:10AD5800013B43710322063002F0CAF82046032261
:10AD680050F8091B043102F0C3F82168CB79E3607D
:10AD78000A7A43EA0223E3604A7A43EA0243E36039
:10AD88008A7A43EA0263E360CB7A23740B7B6374A9
:10AD98002379212B1AD110220D3104F1120002F06F
:10ADA800A7F81D222168501C8B5C6362085C43EA8B
:10ADB8000023901C6362085C033243EA0043636229
:10ADC8008A5C43EA02636362002010BD112B03DC36
:10ADD8000D22E7E70220F8E70120F6E710B5044660
:10ADE800002854D00168002951D00B7843714B7862
:10ADF80083608A7843EA02238360CA7843EA02437D
:10AE080083600A7943EA026383604B7903738B7921
:10AE1800C381CA7943EA0223027BC38102F00F028D
:10AE28000831103002F064F8237B002203F00F038E
:10AE380084F8202084F82820227903F10800111AC8
:10AE480004290DDD21680933043AD21A085C84F814
:10AE58002000D2B2606A84F82820194402F048F829
:10AE6800237922681A44002012F8043CE36212F89D
:10AE7800031C43EA0123E36212F8021C43EA01437C
:10AE8800E36212F8012C43EA0263E36210BD022078
:10AE9800FCE710B5044660B3036853B30279162A79
:10AEA80029D942791A700146082251F8060B013057
:10AEB80002F028F82146082251F80E0B093002F05A
:10AEC80021F82368E28A5A74E38A22681B0A937479
:10AED8002368A269DA74A36922681B0A13752368B8
:10AEE800628B5A752368E27E9A75172323710020B6
:10AEF80010BD0120FCE70220FAE738B50446002817
:10AF080063D00168002960D0037B90F8282003F003
:10AF18000F03002A57D1083320790432134498428A
:10AF280055D363790B702368A2685A70A3682268A6
:10AF38001B0A937023686289DA702368E27A1A71AF
:10AF48002368227B5A712368E2899A71E38922680F
:10AF58001B0A2146D371227B51F8100B02F00F0215
:10AF6800083001F0C5FF237B94F8282003F00F0375
:10AF780003F108052AB1226894F82010515503F10D
:10AF88000905206894F82820616A284401F0B0FF78
:10AF980094F828302268E16A2B44D1545A1CE16A9B
:10AFA800206892B2090A81549A1C2168E08D92B2F5
:10AFB8008854DA1C216894F82F0092B2043388541C
:10AFC8002371002038BD0933A6E70120FAE70220E3
:10AFD800F8E70000024B1A8810431880704700BF3A
:10AFE800440E002008B5074B1B883BB1FEF7CAF991
:10AFF800002814BF6FF00200002008BD6FF00100A8
:10B00800FBE700BF440E002010B5034B00241C8052
:10B01800FEF7AEF9204610BD440E0020B0FA80F0CD
:10B028004009704782B018B9084602B000F0CAB8A3
:10B03800002002B0704710B9084600F079B970478F
:10B0480010B9084600F090B9704703460846114603
:10B058000BB900F0DDB90020704710B9084600F0C0
:10B0680039BD704710B9084600F0FEB90020704796
:10B0780010B40446084611461A46019B14B910BC80
:10B0880000F00CBA10BC70470346084611460BB9CD
:10B0980000F036BA0020704710B40446084611463E
:10B0A8001A4614B910BC00F0A3BA002010BC7047AF
:10B0B80030B40546084611461A46DDE902341DB982
:10B0C800029430BC00F022BB002030BC704710B99D
:10B0D800084600F0D3BB0020704710B9084600F0BE
:10B0E80037BD0020704710B9084600F0E2BB0020C9
:10B0F800704710B9084600F0DFBB002070470346D0
:10B10800084611460BB900F0F9BB0020704710B48F
:10B118000446084611461A46019B14B910BC00F0B3
:10B12800EFBB092010BC704710B40446084611460E
:10B138001A4614B910BC00F02DBDC8B210BC704737
:10B148000048704701000102064B10B51B6A04460F
:10B15800984730B10448054B204498428CBF0020E2
:10B16800012010BDE8010108403576C9405DC600E0
:10B17800F0B5114B85B00C4610491F56054601F035
:10B1880017F80F4BE4B25E6A072D4FF00103CDE9C3
:10B19800024301460AD105220023CDE900234FF4DA
:10B1A8007A727A431846B04705B0F0BD08220020ED
:10B1B800CDE900203A46F5E7D0FB0008B0FB0008CF
:10B1C800E80101081FB5002300930378013B372BE2
:10B1D80021D8DFE803F01C242020201E2020202076
:10B1E8004143454E2055585B5E6164206C1E6E736A
:10B1F800787A7D207F832620202020202020202070
:10B208002020202085878C2020858C208E92C37852
:10B218000BB102230093009805B05DF804FB837816
:10B22800F6E743788DF8043007238DF805308378E6
:10B23800003B18BF01235B008DF8063010238DF802
:10B248000730314B1B6801A803F55872CDE902237A
:10B2580000F08EFF0090DEE74023DBE72023D9E7EC
:10B26800827890F9013012B9284AD35CD2E7284A8B
:10B27800FBE7827890F90130002AF8D1254AF4E7F3
:10B2880040F6B833C6E74FF47A73C3E74FF4FA636E
:10B29800C0E741F28833BDE741F27073BAE71E4850
:10B2A8004FF47A7101F008FE00F5FA60D2E71B4B03
:10B2B800B0E7154B1B6803F55873ABE7124B1B68D7
:10B2C80003F55B73A6E71023A4E70F4B1B68A1E700
:10B2D80001239FE74FF0834300939CE7104BFBE764
:10B2E800104B97E740F21113ADF8003093E70323B2
:10B2F80090E790F901300C4AB7E70C4990F9010042
:10B3080000F056FFA6E700BF4C0E0020A5FB000882
:10B3180095FB00089DFB000818FCFFFF00EA0637B4
:10B328009A99094040F70937D0FB0008B0FB00089C
:10B3380037B50B4B02781B680C2101FB02335B7A93
:10B3480003EB4304074B1D6803690093C368427805
:10B35800816805EBC40000F0A7FC03B030BD00BF56
:10B368004C0E0020480E002030B587B0027B6423C5
:10B37800ADF80030012A4FF00003CDE90133CDE9E3
:10B3880003338DF802308DF8143028D0022A2FD0DC
:10B398001ABB03680BB34368FBB11A4C806823607F
:10B3A800194B18226946186001F0A2FD174B246852
:10B3B80093E807000C3384E8070093E8070004F1DA
:10B3C8000C05032385E80700A4F86C33012204F573
:10B3D8005B7104F5587000F058FC07B030BD09499E
:10B3E80008684360036100F55B7100F55870F2E787
:10B3F800044B1B68B3F86023B3F86C130A43A3F833
:10B408006023EAE74C0E0020480E002080F4000874
:10B4180008B503460A2924D8DFE801F006232323C8
:10B42800230B161B23212100BDE808400068FFF705
:10B438008BBE90F900009978072271B900F0E5FBFE
:10B44800003818BF012008BD052293F9000000212B
:10B45800F4E790F900005978EEE70221EEE70722B9
:10B46800F3E70020EFE7000008B502791AB1012AD6
:10B478000BD0002008BD084B01681B68012203F5AA
:10B48800587000F002FC0120F4E7034B01681B68C8
:10B4980003F55B70F5E700BF4C0E0020F7B50728F1
:10B4A800144D1C46A8BF072058700E46294617465B
:10B4B80000F07EFE94F90130A070072B13D13220E2
:10B4C80000F076FD0C4BDB6D0546984704F10C0245
:10B4D80008340346019200943A463146284600F063
:10B4E8006CFD03B0F0BD054A55F82310D05C00F0A0
:10B4F80057FDE7E7B0FB0008E8010108D0FB0008AA
:10B508002DE9F04F344F90F901607B68D0F8049032
:10B518008BB00446884698470546002859D1E37CF5
:10B5280073B92E4A2378126803EB4303990002EBA0
:10B538008303D3F80490B9F1000F01D152F80190B8
:10B54800274B484613F906B0FB689847A37C228925
:10B55800D7F818A00993072E28D100230121CDE997
:10B568000223204A0693CDE90431CDE907330521AA
:10B57800CDE900214FF47A7202FB0BF24CF2503104
:10B588001846D047637C13B3174B995D7B6D0D311B
:10B59800C9B228469847E07C3246494600F01AFE70
:10B5A80088F8006001200BB0BDE8F08F002101256C
:10B5B8000823CDE90013CDE90715CDE90511CDE93B
:10B5C80003110292A1782B465A462846D9E7074B21
:10B5D800DBE70020E7E700BFE80101084C0E002088
:10B5E800D0FB0008854501009DFB0008A5FB00086D
:10B5F8002DE9F04F8DB090F90130DFF8FCA0DFF8AD
:10B60800FC90CDE90A123E4A12F903B00278DAF842
:10B6180000300C2505FB02333A4A5B7A126803EBCB
:10B62800430302EBC303044693F9021090F90200A6
:10B6380000F0B9FD3449064694F9010000F0B8FD60
:10B64800A26861688046304600F0DFFC2178DAF8AD
:10B658000020D9F80C306943074650589847D9F864
:10B668001C309C4694F901300025072B4FF47A636F
:10B67800CDE90753CDE905552DD10123CDE9035374
:10B688000523CDE901534FF47A7303FB0BF30093C1
:10B698003946434646F2A81228466746B8472378F3
:10B6A800DAF800200C214B4394F90110D05800F02F
:10B6B800B3FDA18994F90100FFF75AFD0B9B217B8B
:10B6C8001860D9F85430284698470A9B01201E7004
:10B6D8000DB0BDE8F08F01200823CDE90350CDE976
:10B6E80001032A46CDF800B0654643463946A847C7
:10B6F80001200546D3E700BF4C0E0020E8010108F1
:10B70800D0FB0008480E0020B0FB00082DE9F04FE0
:10B718008FB0002405468A46914698460494ADF8B1
:10B728001440ADF8024007264FF0010B2B7AA342D4
:10B7380006D9686804A9204400F0CAFB00285DD136
:10B7480002238DF8083002A86B7A8DF80A30FFF7CB
:10B7580039FDAB7A8DF81D309DF811308DF81E300B
:10B768009DF812308DF81F309DF810308DF820307C
:10B77800EB7A8DF821302B7B8DF822306B7B8DF89E
:10B78800233010238DF81C608DF824303A4E8DF844
:10B798002C000DF102030A93072332688DF82D302F
:10B7A800ADF834302B680C9206930DF1120204ABFD
:10B7B8000DF1110106A800F0A5FB072805460BD1DD
:10B7C80030680C22002100F5587001F0A5FB3368A1
:10B7D800BDF80220A3F860239DF811308AF80030E4
:10B7E8009DF8123089F800309DF8103088F8003044
:10B7F800189B28461C700FB0BDE8F08F9DF81330D9
:10B80800BDF81470ADF802702044C4B2F3B917B390
:10B81800194A00201168072602464FF00C0C062B27
:10B828001BD10CFB00FE51F80EE0BEF1000F04D056
:10B838000BFA00F23A4397B2012201301028EED1F8
:10B84800002A3FF473AFADF802706FE75A1E042A5E
:10B8580001D9062BDCD0062668E747FA00FE1EF061
:10B86800010FEAD00CFB00FE51F80EE0BEF1000F0C
:10B8780008BF0626E1E700BF4C0E002038B5054694
:10B888004068FFF761FC0722841D002195F900003C
:10B89800E4B200F0BAF908B904F0FD0495F9010022
:10B8A8000722002100F0B1F908B904F0FB04204692
:10B8B80038BD00207047000010B503780F2B0446F0
:10B8C80018D84068FFF740FC22780B4902EB420287
:10B8D8000968831C01EB820051F82220DBB21AB9F7
:10B8E80003F0FD0358B210BD032B06BF6268426027
:10B8F8000223F7E70020F6E74C0E002002207047ED
:10B908002DE9F0413A4D0446286896B00E46904617
:10B9180000211F460122032300F55870CDE90411C8
:10B92800CDE906118DF80C108DF80D10ADF80E301C
:10B9380000F08DF930B92A68B2F8603343F0030398
:10B94800A2F860332A68637A8DF8203002F55871BE
:10B95800CDE90912274A94F9083012680B9210228F
:10B96800ADF830200DF10E020D9222680E92626839
:10B978000F92D4E90301A27A8DF8402001228DF8B4
:10B98800412011AA82E80300227DE18A8DF8213046
:10B9980018468DF84C20FFF7EBFB08AB15930DF11B
:10B9A8000D0314900093CDF8048003AB04AA394624
:10B9B8000EA800F099FB044678B99DF80C100139DF
:10B9C80001F07AFA00F158030DEB030010F8483C37
:10B9D8003370204616B0BDE8F0810C2801BF2A68F4
:10B9E800B2F8603343F00303A2F86033F1E700BF15
:10B9F8004C0E0020480E0020F8B50679012E0546A9
:10BA080048D90F2E48D80368187A40F30300072254
:10BA1800002140B200F0F9F82B680446187A40F388
:10BA280003100722002140B200F0EFF8B8B1B4FAD1
:10BA380084F4640929680B7A086843F3030243F322
:10BA480003135BB252B29A42C8BF0124FFF77CFBD2
:10BA580080F00103DBB224B10533D8B2F8BD01246C
:10BA6800E8E7DBB90E4F29683B6806EB460003EBB5
:10BA780080000C2201F03CFA3A680C2303FB0623F1
:10BA880020465C72B2F860130123B3400B43A2F85E
:10BA98006033E3E70620E1E70320DFE70420DDE782
:10BAA8004C0E002010B4017801290ED9084B1868F3
:10BAB8000C234B43C4180022C250C4E9012200F5EC
:10BAC800587010BC102200F0A9B8002010BC7047B4
:10BAD8004C0E00202DE9F04186B050238DF814302B
:10BAE800037A102B074630D14368DD7B6DBB0224F7
:10BAF800A8466426062C14D87A68535D03932A4412
:10BB0800517843EA01230393927843EA024373434B
:10BB1800CDE9033863B968468DF80040FFF7C2FFE6
:10BB28000DE0CDF80C808DF81480CDF81080F2E788
:10BB380003AB01A801938DF80840FFF75DFF0134BE
:10BB4800E4B2102C05F10305D4D106B0BDE8F081AC
:10BB58001FB502680379116849B901A88DF8043046
:10BB6800FFF7A0FF78B1032005B05DF804FB02A839
:10BB780002928DF80C30FFF73FFF042805D0052806
:10BB880005D00028EFD00020EEE70220ECE70120E6
:10BB9800EAE70000C90020B9034B0B449856C0B22D
:10BBA8007047024BF9E700BF55FB000815FB00087A
:10BBB800F0B59A42069D03DB9DF914309A4220DDC8
:10BBC8000020F0BD03EB430331F814C005EB8303F9
:10BBD80000264CFA06F7FF0707D51F7A07F00F0E65
:10BBE800964502DCB2EB171F0DDD0136102E03F16E
:10BBF8000C03EED10134E4B22301DBB29842E1D860
:10BC0800DEE70024F8E70120DBE7884204DB904206
:10BC1800CCBF0020012070470020704710B51409E0
:10BC2800B4EB111F03464FEA11100ED391420CD208
:10BC380002B201F00F0133F81240012000FA01F1BD
:10BC480024EA010123F8121010BD0020FCE7F0B52A
:10BC580028B100EB410501270020914200D3F0BD37
:10BC6800002435F802CB234607FA04F636EA0C0618
:10BC780008BF013304F1010408BFDBB2102CF3D173
:10BC880018440131C0B2C9B2E7E710B500B149B9EB
:10BC980010BD31F8134020F813400133DCB2A24242
:10BCA800F7D8F5E70023F9E782B030B504880493A4
:10BCB800D2B9B3F5616F15D349F6AF2542F21072C8
:10BCC800AB4298BF4FF47A72944238BF144661432E
:10BCD800BDE83040C3688B428CBF5B1A0023C36049
:10BCE80002B070476422EFE7012C38BF0124EEE769
:10BCF8002DE9F04F8FB01546199F03939DF86030DA
:10BD080007930C46804603F099F86A4A0590A7F510
:10BD1800F633303BB3FBF2F3534303F5F63B04939E
:10BD2800182313FB05430BF1300B069300254FF046
:10BD3800FF3A069B9C4207D1002D14BF50464FF096
:10BD4800FF300FB0BDE8F08FBDF96830ADF8243092
:10BD5800099919973846089703F000F82688B8F12A
:10BD6800000F5FD1B7F5616F5AD349F6AF2242F29F
:10BD78001073974298BF4FF47A739E4238BF1E469D
:10BD8800642E59D1DFF83091A060A1680CA803F0A7
:10BD980007F80D9B0093DDE908120C9B0AA802F036
:10BDA8005EFF039A0A9B0AB9079A2AB122694A4593
:10BDB80002D1424A93420ED9414BC4F80C909F429B
:10BDC80009D90023ADF82C300B99CDF828B0584686
:10BDD80002F0C4FFA060606808B9C4F80C90C4F809
:10BDE8001090B8F1000F04D003F032F8E368034470
:10BDF800E360D4E903329342059B88BFE260636045
:10BE08001B9BE1687343994204D20398E8B9B8F1DF
:10BE1800000F1AD001231D442375EDB2183488E7AA
:10BE28006423AAE7039B0BB9234BE360012EDFF8D9
:10BE3800889038BF0126CEE7B6F57A7F0ABFDFF8CB
:10BE48008490DFF88490A0609FE7002093422075DB
:10BE580006D85B1A9A4505F1010528BF9A46EDB246
:10BE6800B8F1000FDAD1642E184AADF82C801DD035
:10BE780049F6B023B6F57A7F18BF1346974281BFBB
:10BE8800049A02F5A83202F5C0729B180A931A9B0D
:10BE980000930AAE96E80600199B304602F0DFFED2
:10BEA80096E8030002F05AFF8246B7E74FF4616351
:10BEB800E4E700BF8051010040771B007F5101007B
:10BEC8002FEC010080A81201002E930230EC010033
:10BED8000378032B14D1437803F00F021B098A70EF
:10BEE8004B7083788B80C27843EA02238B80037976
:10BEF800C3F3021203F00F03CA700B7005207047DA
:10BF0800002070472DE9F3479A464379057990F95F
:10BF180007609146044690F906208846D3B190F907
:10BF28000870002D37D00F2A1BD194F909200F2E45
:10BF380027D194F90A00072D02D1002F08BF012745
:10BF480088F8002089F8000028468AF8007002B0B6
:10BF5800BDE8F08790F90B7090F9092090F90A6014
:10BF6800DFE7A369019394F91530009394F914302D
:10BF78002169207BFFF71CFE0028D8D105F0FD05BC
:10BF8800D5E794F91D00B042D5DC94F91C30B342D2
:10BF980003DA05F0FB053046D2E73046CBE7000070
:10BFA800024B03FA00F0B0FBF1F0704740420F007B
:10BFB8004FF4FA53B3FBF0F0704730B54FF47A758D
:10BFC8000C1F6A4300FB042252001EBF00F1FF341D
:10BFD8001219B2FBF0F2914238BF1146039A116070
:10BFE800820048431CBF013040084FF47A71121A8E
:10BFF80001FB1323002BCABF03F2E73393FBF1F1D4
:10C00800B3FBF1F1049B196030BD38B5400014460C
:10C018000D46F4F7E9FD01462846F4F733FD2146BD
:10C02800F4F730FDF4F710FA03F07EF9F4F7FEFCAC
:10C0380040B238BD2DE9F74F019300239C469E4638
:10C04800048A1E01F6B2B44246D906EB46054FEA09
:10C058004309AD000024476837F809702741FF07F6
:10C0680029D5876807EB050A7F5927B3077837B9B9
:10C07800476927B137F809702741FF071BD59AF898
:10C08800087090F901B047F303084FFA88F8D845CB
:10C0980011DC47F303177FB25F450CDB9AF8097090
:10C0A80007EB4708C76807EBC8073F7D5FB90CF186
:10C0B800010C5FFA8CFC0134102C05F10C05CAD177
:10C0C8000133DBB2BCE70EF1010706EB040801F807
:10C0D8000E805FFA87FEEEE7019B82F800E083F8A6
:10C0E80000C003B0BDE8F08F2DE9FF470446406863
:10C0F800DDE90C671D468A46914602F0A9FE2368D1
:10C108001B1A3B604FF000080123337085F800804C
:10C11800636813B12368834224D8D4F81CC0CAF8D2
:10C128000080A3699CF800E00393D4E9030101AB04
:10C1380083E80300237D0093DCF80C10237A627AED
:10C148007046FFF7D5FD334638602A46E069494610
:10C15800FFF770FF2B782BB1C7F80080002004B0E0
:10C16800BDE8F0873378002B0CBF0C200B20F6E7D6
:10C1780037B590F9002090F90250954204460FD047
:10C18800013A52B295420BD0A368019394F9013059
:10C1980000936168E0782B46FFF70AFD0028EFD08E
:10C1A800104603B030BD8842B8BF0846704700004B
:10C1B80051F82000054B984205D0054BC31A584248
:10C1C8005841400070470120704700BF90D00300DD
:10C1D80020A1070005281FB50ED80C4B53F82030B6
:10C1E8000093CDE901120A4B01220021022002F03E
:10C1F8003DFB05B05DF804FBCDE90012054B0122BB
:10C208000021022002F032FBF3E700BF40FC0008E7
:10C21800D8FB0008F7FB000807B5054BCDE900017E
:10C2280001220021022002F021FB03B05DF804FB8B
:10C2380013FC000810B5102204460021F13000F06C
:10C248006BFE0021C4F814112046F022BDE810400E
:10C2580000F062BE02460846102100F0A5B92DE99B
:10C26800F0430446D0F8140185B00E46154604F292
:10C27800011988B3C0F110089045474628BF1746F2
:10C28800BAB2484400F034FED4F814313B440F2BC2
:10C29800C4F814312DD9A8452BD204F1F00304F5C4
:10C2A800807113F8012F187C8B4282EA00021A7001
:10C2B800F7D104F1F10810224146684600F018FE53
:10C2C80022466946684600F0F1F910226946404660
:10C2D80000F00EFE3E44ED1B04F5807804F1F107F2
:10C2E800102D09D8AAB23146484600F001FEC4F81C
:10C2F800145105B0BDE8F08304F1F003711E13F882
:10C30800012F11F8010F434582EA00021A70F6D195
:10C3180010223946684600F0EBFD22466946684619
:10C3280000F0C4F910226946384600F0E1FD1036E5
:10C33800103DD5E7F0B589B00C461022002105461E
:10C34800684600F0E9FD22466946684600F0AEF905
:10C358009DF90030002B6A464FF0000143DA13784C
:10C3680012F8010F01315B0043EAD0130F2902F8DC
:10C37800013CF4D19DF80F305B0083F08703D4F8BB
:10C388001401DBB210288DF80F303BD104F580730F
:10C39800694604F5887013F8016F11F8012B98426B
:10C3A80082EA06021A70F6D104F1F00304F58071EE
:10C3B80013F8012F187C8B4282EA00021A70F7D119
:10C3C80010220DEB020004F1F10100F091FD22466C
:10C3D800294604A800F06AF910220021684600F0F6
:10C3E8009BFD09B0F0BD137812F8010F01315B0015
:10C3F80043EAD0130F2902F8013CF4D19DF80F301D
:10C408005B00BCE79DF90030002B6A464FF0000145
:10C4180037DA137812F8016F01315B0043EAD6135B
:10C428000F2902F8013CF4D19DF80F305B0083F02E
:10C438008703471CDBB28DF80F30102F04EB000385
:10C44800C0F10F064FF0800288BF002600F581700A
:10C4580083F801210021324620443E4402F038FF8F
:10C46800C4F8146104F58073694604F5887013F8FC
:10C47800016F11F8012B984282EA06021A70F6D170
:10C4880092E7137812F8016F01315B0043EAD61383
:10C498000F2902F8013CF4D19DF80F305B00C8E782
:10C4A8000A780378534003704A78437853404370BE
:10C4B8008A78837853408370CA78C3785340C370AE
:10C4C8000A790379534003714A7943795340437198
:10C4D8008A79837953408371CA79C3795340C37188
:10C4E8000A7A037A534003724A7A437A5340437272
:10C4F8008A7A837A53408372CA7AC37A5340C37262
:10C508000A7B037B534003734A7B437B534043734B
:10C518008A7B837B53408373CA7BC37B5340C3733B
:10C52800704710B50B7814786340037054784B78D3
:10C538006340437094788B7863408370D478CB7869
:10C548006340C37014790B796340037154794B7954
:10C558006340437194798B7963408371D479CB7943
:10C568006340C371147A0B7A63400372547A4B7A2E
:10C57800634043728B7A947A63408372D47ACB7A1D
:10C588006340C372147B0B7B63400373547B4B7B08
:10C5980063404373947B8B7B63408373CB7BD27BF9
:10C5A8005340C37310BD0000A1F11003DBB2102B80
:10C5B8002DE9F047044604D83A4820FA03F3DB078C
:10C5C80005D4002382F8F030FF20BDE8F087561E1E
:10C5D800254615F8013B06F8013F631B0B4413F091
:10C5E800FF00F6D101F11C039B005FFA83FCC3F343
:10C5F8000313013BDFF8B09082F8F03088465318F7
:10C608004FF0010EB8FBF1FA01FB1A8A1AF0FF0A83
:10C6180013F8047C13F8036C13F8025C13F8014C4C
:10C6280030D119F806A019F8056019F8045019F85E
:10C6380007404FEADE1707EB47078EEA0A0A07EBBF
:10C64800C7074FEA4E0EFFB25FFA8EFE87EA0E0E5C
:10C65800574692F800A087EA0A071F7057787E406D
:10C668005E70967875409D70D57808F104085FFA79
:10C6780088F86C40C445DC7002F1040203F104033D
:10C68800C0D8A2E71829E4D9BAF1100FE1D1DFF830
:10C6980018A01AF807701AF806601AF805501AF860
:10C6A8000440D6E70101010058FE00082DE9F04FCB
:10C6B800A3B092F8F0301D911B920193002B00F06B
:10C6C800538101461EA8FFF72CFF1B9BA74CA84DC2
:10C6D800A84E10330293002303939DF87C00049026
:10C6E8009DF886000590205C06909DF87B000790D9
:10C6F800205C089004989DF881C0205C099014F88B
:10C708000C000A909DF880000B909DF885009DF81C
:10C7180078809DF87DE09DF882A09DF887900C9028
:10C728009DF87A00029B1C9314F80A2014F809302B
:10C7380014F8081014F80E700D90205C0E909DF8F7
:10C748007F000F90205C10900B98205C11900C9843
:10C75800205C12909DF8840013909DF87900149045
:10C768009DF87E001590205C16909DF88300179028
:10C77800205C18901398205C19901498205C1A90EB
:10C788000398013003900298DDF804B0103002904D
:10C798009DF80C00834536D88DF878108DF87A20EE
:10C7A80009990E9A8DF87C108DF882201199069AB5
:10C7B8008DF880108DF87E201999169A8DF88410BE
:10C7C8008DF886200A99189A8DF87D108DF88720A3
:10C7D8001299109A8DF87B301B9B8DF881108DF87B
:10C7E80083201A99089A1D988DF885108DF87F2056
:10C7F8001EA903EB0B128DF87970FFF792FE00204B
:10C8080023B0BDE8F08F15F808B082EA03008BEA80
:10C81800000016F80EB080EA0B008DF8780015F8C5
:10C828000E004B40434016F80A0043408DF879301B
:10C8380081EA070315F80A10594016F809305940DB
:10C8480016F808308DF87A107A40534015F8092008
:10C8580053408DF87B30089A069B5340049AAA5C93
:10C86800534016F80C2053408DF87C30DDE908322F
:10C878005A4015F80C305340059AB25C53408DF875
:10C888007D30DDE909325A40059BEB5C5340079A3D
:10C89800B25C53408DF87E30069B0A9A5340049A46
:10C8A800B25C5A40079BEB5C5A408DF87F200E9B88
:10C8B800109A53400B9AAA5C53400C9AB25C5340AE
:10C8C8008DF88030DDE910325A400C9BEB5C534008
:10C8D8000D9AB25C53408DF88130DDE911325A402F
:10C8E8000D9BEB5C53400F9AB25C53408DF882303D
:10C8F800129A0E9B53400B9AB25C5A400F9BEB5C0A
:10C908001C995A408DF88320169B189A5340139A05
:10C91800AA5C5340149AB25C53408DF88430DDE928
:10C9280018325A40149BEB5C5340159AB25C534042
:10C938008DF88530DDE919325A40159BEB5C534080
:10C94800179AB25C53408DF886301A9A169B53405A
:10C95800139AB25C5340179AAA5C1EA853408DF8EC
:10C968008730FFF79DFDB8E6FF2049E758FE00082D
:10C9780058FD000858FC000808B538B1044A0549B4
:10C988001060D82200F0B4FA002008BD0220FCE7AD
:10C99800500E002000E503080A4B1A6870B5002302
:10C9A80002F1180503EB03142E5D864204D11834F6
:10C9B80022440A60002070BD01330B2BF2D1032002
:10C9C800F9E700BF500E00202DE9F041CCB0064633
:10C9D800DDF8488117461C460D4631B3B8F1000F03
:10C9E80023D006A8FFF726FC204601A9FFF7D4FFAD
:10C9F8000446B0B9019906A80131FFF72BFC26B10E
:10CA08001022314606A8FFF72AFC3A46294606A80E
:10CA1800FFF725FC06A902A8FFF78CFC029BC8F8C3
:10CA2800003020464CB0BDE8F0810224F9E7000050
:10CA380030B595B013A90446FFF7AEFF002830D1F2
:10CA48001B4B0C2101FB00F2D5189A5CA2422AD19B
:10CA5800139B1A7C1092DA7B0F929A7B0E925A7B68
:10CA68000D921A7B0C92DA7A0B929A7A0A925A7A77
:10CA780009921A7A0892DA7907929A7906925A797B
:10CA880005921A790492DA7803929A7802925B787E
:10CA980001930022AB6800931146064B022001F077
:10CAA800E5FE15B030BD01300B28CBD1F9E700BF4A
:10CAB800D000010858FF000810B40B2B019C03D8C4
:10CAC800019410BCFFF780BF032010BC704730B53D
:10CAD8000D4685B01446014668B103AA00200092AD
:10CAE8002A460390FFF770FF18B90398001B18BF78
:10CAF800012005B030BD0220FBE72DE9F0430D46CB
:10CB0800BFB014469946804620B31BB311F00F01FD
:10CB180022D1F02201A800F0FFF920466946FFF76C
:10CB28003BFF044648B9009801AA10210130FFF7DD
:10CB38003BFD2E46AF1BFFB21EB920463FB0BDE8F5
:10CB4800F08301AA09EB070108EB0700FFF7AEFD28
:10CB5800103EEFE70224F0E70524EEE7F0B5184EA3
:10CB68003468024685B00846002304F1180103EB37
:10CB780003154F5D97421ED10D2A05F1190513D1F2
:10CB88000023CDE90033CDE902330C2210216B4696
:10CB9800FFF7B3FF0446306810226946284400F0C6
:10CBA800A7F9204605B0F0BD01461022601900F033
:10CBB8009FF90024F5E701330B2BD8D10324F0E7C4
:10CBC800500E002009B1FFF7C9BF022070471FB5FA
:10CBD8001446A0B10C2A01D10B2912D10023CDE9AA
:10CBE8000033CDE902330A466B461021FFF785FF73
:10CBF80018B969462046FFF7B1FF04B010BD0220FE
:10CC0800FBE70320F9E7F8B51E46DDE907479DF87D
:10CC180018505BB354B34FB3212D29D819462A466F
:10CC2800204600F065F90122631C691EB018FFF761
:10CC380064FFF8B9E37ADB093B70EBB96319204666
:10CC480013F8012C13F8021C120642EA014213F8E9
:10CC5800041C0A4313F8031C012342EA0122291F7A
:10CC6800FFF735FF003818BF0120F8BD0220FCE7A8
:10CC78000520FAE70720F8E70420F6E710B5044690
:10CC880028B1044B5B6998472060002010BD022042
:10CC9800FCE700BFE801010808B5014630B1044BC4
:10CCA8000822186800F024F9002008BD0220FCE7DB
:10CCB800500E002008B530B1044B0822196800F066
:10CCC80017F9002008BD0220FCE700BF500E002025
:10CCD8007FB5124E0023044602A801930D46FFF7C4
:10CCE800E9FF33685B6901936CB102AA082312F863
:10CCF800011B41B9013B13F0FF03F8D102A8A0477B
:10CD080002A8FFF7C9FF35B1019B23B901A8A847BD
:10CD18003368019A5A61002004B070BD500E00209B
:10CD280008B5014638B1054B18680822104400F0D0
:10CD3800DFF8002008BD0220FCE700BF500E0020ED
:10CD480008B538B1044B19680822114400F0D0F82E
:10CD5800002008BD0220FCE7500E0020034B1B6892
:10CD680002280CBF1961596100207047500E00203D
:10CD780049B1064B1B68D3E90423022808BF1346B0
:10CD88000B60002070470220704700BF500E002043
:10CD980030B58FB0002405460CA80994FFF78AFF28
:10CDA8009DF8373007939DF8363006939DF8353057
:10CDB80005939DF8343004939DF8333003939DF820
:10CDC800323002939DF8313001939DF83030009352
:10CDD800224621461E4B022001F048FD0AA8FFF713
:10CDE800AFFF9DF82F3007939DF82E3006939DF8DE
:10CDF8002D3005939DF82C3004939DF82B30039328
:10CE08009DF82A3002939DF8293001939DF8283027
:10CE1800009322460F4B2146022001F027FD09A965
:10CE28002846FFF7A5FF9DF8243003939DF8253089
:10CE380002939DF8263001939DF8273000932246EF
:10CE4800054B2146022001F011FD0FB030BD00BF97
:10CE5800B4FF0008F2FF00083000010808B5002000
:10CE6800FFF7E6FD0120FFF7E3FD0920FFF7E0FDEE
:10CE78000820FFF7DDFD0020FFF78AFF002008BD2E
:10CE880010B504460B20FFF7D3FD0C20FFF7D0FDAB
:10CE98000920FFF7CDFD0820FFF7CAFD0A20FFF79C
:10CEA800C7FD2046FFF774FF002010BD014B186036
:10CEB800704700BFF80000200B4A30B514680B4DCE
:10CEC80043F2390305FB04331360091A6FF000427B
:10CED800B3FBF2F2C2EBC27201319B1A93FBF1F27F
:10CEE80001FB1233184430BDF80000206D4EC641D6
:10CEF80001380A44914200D1704711F8013B00F80B
:10CF0800013FF7E710440A44914200D1704711F8F5
:10CF1800013B00F8013DF7E702F0DAB930B530B16E
:10CF28000A4D01444FF0FF33814201D1D84330BD4F
:10CF380010F8012B5340082243F30004013A2C4017
:10CF480092B284EA5303002AF6D1EDE72083B8EDC4
:10CF580001207047054B4FF400529A62044B1B683E
:10CF680013B15B6803B11847704700BF000400485D
:10CF7800E00E0020054B4FF480529A62044B1B6868
:10CF880013B1DB6803B11847704700BF00040048BD
:10CF9800E00E00204FF0FF3070474FF0FF30704731
:10CFA800012070470120704700F0FCBD10B501F06A
:10CFB800DFFA0E21044640F61F1000F0F3FD20466C
:10CFC800012101F0BFFABDE8104000F09DBF00004C
:10CFD80070B50C4E01EB40030D46B3654FF6FF717B
:10CFE800002304461A46084601F024F896F856002D
:10CFF800002101F0A7FA29462046BDE8704000F05C
:10D008005BBF00BF840E002010B5044601F06DFB25
:10D0180001281CD101F071FB34B11248214601F0FE
:10D02800D9FF104801F09CFF0F4C104B00214FF422
:10D038008052A1659A6194F8560001F083FA6378EA
:10D048006BB16FF07F40BDE8104000F019BF0023BE
:10D0580040F262211A46084600F0ECFFDCE7A068BF
:10D068008001F0E7540E0020840E002000040048E0
:10D07800002000F085BE00F0A5BD000008B500F056
:10D088008BFD0438C0B2032896BF024B0020185C01
:10D0980008BD00BFB201010808B501F07EFA0330EF
:10D0A80008BD00F00DBE00F0CDBD08B501F0C4F913
:10D0B80008BD000038B50D46144601F021F8284691
:10D0C80001F056FA0E21054640F61F1000F06AFDE1
:10D0D80028460121074D01F035FA00F015FF4FF4FD
:10D0E8007A716143284601F075FF2846BDE838404B
:10D0F80001F036BF6C0E002001F002B808B5084BED
:10D10800002193F8560001F01DFA00234FF4C07176
:10D118001A46084600F08EFFBDE8084000F0E8BE59
:10D12800840E002010B5044601F0DFFA01281CD156
:10D1380001F0E3FA34B11248214601F04BFF1048E0
:10D1480001F00EFF0F4C104B00214FF48052A165E7
:10D158009A6194F8560001F0F5F963786BB16FF0B5
:10D168007F40BDE8104000F041BE002340F262213C
:10D178001A46084600F05EFFDCE7A0688001F0E789
:10D18800540E0020840E00200004004808B54FF01B
:10D19800040000F0DBFDBDE808400220F4F7CEBE35
:10D1A800F7B500230D4640F201211A460646084607
:10D1B80000F040FF2F4B304C4FF400529A6194F826
:10D1C8005600012101F0BEF92378012B40F68900B1
:10D1D80012D194F85130062B0ED100F0F3FC00F078
:10D1E800FB0140F6890000F0DDFC2378032B29D8E9
:10D1F800DFE803F00F080F3C00F0E4FC40F0040106
:10D20800C9B2EEE7E5771D4801F094F800222946F7
:10D2180015E001F06AFA0128074625D129460DF1E3
:10D228000702304601F066FA0546A0B99DF80730B6
:10D238001248A37501F07EF89DF807102A4630467B
:10D2480000F0CAFD61680E4801F0C4FE0C4801F008
:10D2580087FE002006E00B4B3A460021022001F031
:10D2680005FB032003B0F0BDA575CCE70223A3732B
:10D27800A576C8E700040048840E0020920E00201E
:10D288006C0E00205401010808B500231A461946FF
:10D29800184600F0CFFEBDE8084000F0BDBD000014
:10D2A8001D4B73B51D4D186000241D486C70C5E9F1
:10D2B8000144AC6500F0E8FEAC8100F053FE214665
:10D2C800204601F09BF821460422012000F04CFF83
:10D2D800144E154D4FF6FF7123462246084600F0BE
:10D2E800A9FEFFF753FF2246104B00944FF0FF3181
:10D2F800304601F089FD0E4B009422464FF0FF3175
:10D30800284601F081FD304601F0DCFD284602B0D8
:10D31800BDE8704001F0D6BDE00E0020840E00206C
:10D3280091DB00086C0E0020540E00205DCF000831
:10D338007DCF00080128084805D1084BC17719702E
:10D348000E3000F0F7BF437D012B03D1034B8175ED
:10D358001970F5E7704700BF840E0020FC0000201C
:10D368000D4B10B5044618735873012000F016F8D9
:10D378005CB134214FF4E86000F014FC4421BDE8AE
:10D38800104040F2417000F00DBC14214FF4E860E9
:10D3980000F008FC2421F2E7840E002038B5114D76
:10D3A8000446287001F0AEF9012C0DD0032C17D0DB
:10D3B8002CB1032000F0C2FE00236B7303E020466B
:10D3C80000F0BCFE6C7338BD204600F0B7FE287B29
:10D3D8006B7B8342F7D06873BDE83840FFF7C0BF66
:10D3E8000220E7E7840E00202DE9F04F85B00646BD
:10D3F8000E9DBDF840A09DF844709DF8489001939B
:10D4080088469346494C01F06FF90198A6B1012E60
:10D418004CD0404601F0ACF80E2184F8560040F696
:10D428001F1000F0BFFB94F8560001F062F9169B3C
:10D43800636005B0BDE8F08F0B2384F8443084F8AE
:10D448003860E56301F0F6F8B9F1000F41F604031E
:10D4580063820CBF0123F223E3754FEACA0A012352
:10D4680087F00107237684F84500C4F840B0A67316
:10D47800A4F810A026756775FFF7FAFD3046FFF788
:10D488008DFF04F1380000F0E9FE04F10E0000F011
:10D4980051FF274A1068516802AB03C302A800F085
:10D4A800E1FB40F2FF1000F0B1FBB2E7214A84F83B
:10D4B8003860EBB2125C84F8503070BB0B3D012D24
:10D4C8008CBF00250125053B012B04D8BAF10C0FB0
:10D4D80038BF4FF00C0A9DF83C3084F85230164B98
:10D4E80084F853501B78E37701259DF8543084F86D
:10D4F800512084F82130A573A4F81CA0A77784F8DC
:10D508002090FFF7B5FD2846FFF748FF0B4800F0CD
:10D51800A5FE0B4800F00EFF7BE7012804D1A5F11A
:10D528000C014D424D41CEE70025CCE7840E00208A
:10D5380098F40008E4010108FC000020BC0E00205B
:10D54800920E00202DE9F04F87B0DFF8C4A19DF8B6
:10D5580064B09DF84C8002930F469DF854309DF8B6
:10D568005010BDF8489003918AF801B0BDF84460A6
:10D5780001930546144601F0B7F8BBF1000F18BF38
:10D588004FF00009DFF88CB10399B8F1000F08BF1C
:10D59800FF218BF8001025B1012D50D007B0BDE850
:10D5A800F08F284600F0BAFC0B2138468AF8441060
:10D5B8008AF83850CAF83C4001F03CF8019B9BF8C7
:10D5C80000208AF81620002B0CBF0122F22241F617
:10D5D80004018AF81720F600012288F00108AAF849
:10D5E80012108AF818208AF845008AF80E50AAF80E
:10D5F80010608AF814508AF81580FFF739FD28461C
:10D60800FFF7CCFE0AF1380000F028FE0AF10E0000
:10D6180000F090FE40490868496804AA03C204A8BB
:10D6280000F020FB40F2FF1000F0F0FA4FF4FA523D
:10D6380002FB09F2B2FBF4F2CAF80820AEE70020B8
:10D6480000F06CFC35488AF83850E1B2C05D8AF8C1
:10D658005010002F4DD10B3C012C8CBF002401240D
:10D668000539012902D80C2E38BF0C26029B9BF8DD
:10D6780000208AF852308AF85340019B8AF81F200C
:10D6880001249DF860208AF821208AF820308AF841
:10D6980051008AF80E40AAF81C608AF81E80FFF72D
:10D6A800E7FC2046FFF77AFE1D4800F0D7FD1D482D
:10D6B80000F040FE5FFA89F000F03CFC40F6A30061
:10D6C80000F080FA00EA040140F6A30000F06AFACC
:10D6D8009AF82120A24240F2367013D100F072FA73
:10D6E80000F0FB0140F2367000F05CFA4FF6FF7272
:10D6F800A2E7012F04D1A4F10C035C425C41AFE71F
:10D708000024ADE700F05EFA40F00401C9B2E9E791
:10D71800840E0020FC00002098F40008E4010108B1
:10D72800BC0E0020920E0020F0B58BB00D460446CA
:10D7380017461E46FFF79CFC0020FFF72FFE2046E9
:10D7480000F0DEFC00240123CDE9084303234FF455
:10D75800167229462046CDE90644CDE90444CDE9B0
:10D768000244CDE900532346FFF7ECFE2046FFF7BD
:10D77800D9FCFFF791FCF4F7E1FB01F05FFB0446ED
:10D78800204601F065FBB04205D30124FFF770FC89
:10D7980020460BB0F0BD00F04FFE8742F0DA0024BF
:10D7A800F4E70000F0B5BDF814409DF818709DF836
:10D7B8001CE09DF8205040B1012814D0012200231C
:10D7C80098180138B0FBF2F0F0BD87F00107E300CC
:10D7D80003EBC70318330EEB450503EBC5034FF402
:10D7E8007A714B43ECE7501F012803F1040302D878
:10D7F8000C2C38BF0C24D1B9A2F10B0CBCF1010FD1
:10D808008CBF4FF0000C4FF0010C2801002F00EBEB
:10D81800CE000CBF14250025A0EB8200062A4FEA93
:10D8280082062844A2F102070DD8354610E00129E6
:10D8380006D1A2F10C00D0F1000C4CEB000CE4E78F
:10D848004FF0000CE1E70830BCF1000FEDD0BD004F
:10D858000028ACBF2E182E1C701E90FBF5F003FBA1
:10D868000044094B062A5A5C8CBF0C340E340A2A31
:10D8780009D8A30001334FF47A71BB404B430349E5
:10D8880051F822209CE7FFDEE4010108B8010108F5
:10D8980008B5094B012193F8560000F053FE4FF4E8
:10D8A800D7602D2100F07EF900F033FBBDE8084079
:10D8B800024800F07BBA00BF840E0020FFFF0F0073
:10D8C80073B5A44CB4F854300025202B8DF80350C0
:10D8D800019500F01B8114D8082B0DD87BB1013BB2
:10D8E800072B0CD8DFE813F042005B000B00CD00DB
:10D8F8000B000B000B00FD00102B00F0008102B0A4
:10D9080070BDB3F5807F00F0988011D8402B00F0EF
:10D918001081802BF3D1284600F032FA8E4B1B6819
:10D92800002BECD09B69002BE9D028469847E6E706
:10D93800B3F5007FE3D1894B01222946022000F08C
:10D9480095FF00F029F9042840F08580844B85482C
:10D958004FF400529A6201F0B5FA284600F010FA26
:10D968007D4B1B68002BCAD05B6814E07C4B7D485C
:10D978004FF400529A6201F0A5FA002000F000FA74
:10D9880000F0B5FE012801D100F0BAFE724B1B6809
:10D99800002BB4D01B68002BB1D09847AFE7704B71
:10D9A80071484FF480529A6201F08CFA657895B903
:10D9B800284600F0E5F9294640F6021000F0F2F892
:10D9C80040F6441000F0FEF840F00201C9B240F6FB
:10D9D800441000F0E7F8FF220DF1030163485E4DA3
:10D9E80000F05AFD624800F071FD2B68002B86D0CC
:10D9F8009E68002E83D094F82430012B08D194F926
:10DA0800313094F930209DF803105848B04776E734
:10DA1800E06B01A900F022FE019B9DF8031053481A
:10DA28004FF47A7203F5FA7393FBF2F32A685BB248
:10DA3800956894F92920A84761E7284600F0A0F9DD
:10DA4800454B1B68002B3FF45AAF9B69002B3FF4F2
:10DA580056AF01206AE700F09FF805287FF44FAF22
:10DA68003F4B41484FF480529A6201F02BFA284606
:10DA780000F086F9384B1B68002B3FF440AFDB6899
:10DA880089E700213B4B0122022000F0EFFEA16D47
:10DA980000293FF434AFC1F3074140F6031000F00A
:10DAA80081F894F8591040F6041000F07BF894F8C7
:10DAB800581040F6051000F075F840F6021000F016
:10DAC80081F840F00101C9B240F6021000F06AF88E
:10DAD800002340F262211A460846A36500F0AAFA1C
:10DAE8000DE7254B01220021022000F0BFFE00F0C7
:10DAF800FCFD01287FF403AF00F003FEFFE61F4B97
:10DB080001220021022000F0B1FEF8E6164801F0DB
:10DB1800D9F9607808B900F033F90F4B1B68002B6E
:10DB28003FF4EDAEDB68002B3FF4E9AE9847144BA9
:10DB3800E6E7144B01222946022000F097FE6078A0
:10DB480008B900F01DF9044B1B68002B3FF4D7AE51
:10DB58001B6920E7840E0020E00E002069010108FF
:10DB6800000400486C0E0020540E0020E40E002033
:10DB7800A80E00207D010108860101089001010816
:10DB880099010108A2010108024BA3F85400FFF70C
:10DB980097BE00BF840E0020014B1878704700BF65
:10DBA800F20F002007B501238DF807100DF10702C9
:10DBB80001460348F7F71EFC03B05DF804FB00BFFD
:10DBC800D401002007B5012301460DF107020448DE
:10DBD800F7F749FC9DF8070003B05DF804FB00BFA8
:10DBE800D401002010B50446F5F7BEF801280CD181
:10DBF80040F62310FFF7E6FF00F0F901214340F655
:10DC08002310BDE81040FFF7CDBF10BD10B50C4B79
:10DC18001B7804469BB94FF4D760FFF7D3FFC4F3D2
:10DC2800002100F0FE0001434FF4D760FFF7BAFF70
:10DC3800E1B240F2B960BDE81040FFF7B3BF10BDD4
:10DC4800F10F002010B51346EFF3108472B60A46A0
:10DC580001460348F7F7CEFB84F3108810BD00BFD8
:10DC6800D401002008B5014608224FF4D860FFF718
:10DC7800E9FF002008BD000007B5074B1B7840BA34
:10DC8800ADF804002BB9022201A940F2BC60FFF7ED
:10DC9800D9FF03B05DF804FBF10F002007B5074B6F
:10DCA8001B7840BAADF804002BB9022201A940F252
:10DCB800BE60FFF7C7FF03B05DF804FBF10F00205B
:10DCC80010B51346EFF3108472B60A4601460348AE
:10DCD800F7F7C9FB84F3108810BD00BFD4010020FA
:10DCE80010B51346EFF3108472B60A46014603488E
:10DCF800F7F7ABFC84F3108810BD00BFD4010020F7
:10DD08000A4601460020FFF7EBBF000010B5134696
:10DD1800EFF3108472B60A4601460348F7F7C8FCC9
:10DD280084F3108810BD00BFD401002010B513463D
:10DD3800EFF3108472B60A4601460348F7F7CEFBA4
:10DD480084F3108810BD00BFD401002013B5044629
:10DD58000020F5F703F80220FFF744FF04F007045A
:10DD680001220DF1070184208DF80740FFF7DEFF3F
:10DD7800024B00221A7002B010BD00BFF20F002043
:10DD880007B501228DF807000DF107018020FFF784
:10DD9800CDFF9DF80730002B034B14BF0222012250
:10DDA8001A7003B05DF804FBF20F002007B5094BA9
:10DDB8008DF8060004221A70030C8DF80430032233
:10DDC800030A01A983208DF80530FFF7AFFF03B0E0
:10DDD8005DF804FBF20F002010B51446FFF790FF22
:10DDE8002046BDE81040FFF7E1BF000007B5094B2A
:10DDF8008DF8060005221A70030C8DF804300322F2
:10DE0800030A01A982208DF80530FFF78FFF03B0C0
:10DE18005DF804FBF20F002073B5002640F6E2001F
:10DE28000196FFF7CFFE00F0FE01054640F6E2003E
:10DE3800FFF7B8FE40F6E500FFF7C4FE00F07F01EB
:10DE4800044640F6E500FFF7ADFE6FF07F40FFF7B0
:10DE5800CDFF04220DEB020140F61900FFF730FF59
:10DE68003046FFF78DFF294640F6E200FFF79AFE9D
:10DE7800214640F6E500FFF795FE019802B070BD17
:10DE880013B50C4B04460522972140F6AC001A70D6
:10DE9800FFF788FE230C8DF804300322230A01A91A
:10DEA80082208DF805308DF80640FFF73FFF02B05D
:10DEB80010BD00BFF20F002007B5030C8DF800302D
:10DEC800030A8DF801300B0C49BA8DF80200ADF841
:10DED80004100622694694208DF80330FFF726FFC8
:10DEE800024B06221A7003B05DF804FBF20F002003
:10DEF800002208B51146C520FFF718FF014B07227D
:10DF08001A7008BDF20F002000221146D120FFF739
:10DF18000DBF00221146D220FFF708BF07B5012226
:10DF28008DF807000DF107019F20FFF7FFFE03B0F2
:10DF38005DF804FB07B501228DF807000DF1070114
:10DF4800A020FFF7F3FE9DF807103F2907D901F03D
:10DF5800F8010131C9B240F20670FFF723FE03B0A1
:10DF68005DF804FB07B5F4F7FFFE431E584258411D
:10DF78008DF8070001220DF107019620FFF7D6FE64
:10DF880003B05DF804FB07B500F07F008DF80700CB
:10DF980001220DF107018920FFF7C8FE03B05DF8E3
:10DFA80004FB0000154B984207B51BD8144B984248
:10DFB8001BD8144B98421BD8134B98421BD8134BB1
:10DFC80098428BBF6B2229226F232B238DF80420C4
:10DFD80001A9022298208DF80530FFF7A7FE03B0AB
:10DFE8005DF804FBE122E923F0E7D722DB23EDE724
:10DFF800C122C523EAE775228123E7E700E9A435B2
:10E0080080F8A9328044E52D000B6B1B40FC5419A5
:10E0180007B58DF8062004228DF804008DF8051048
:10E0280095200DEB02018DF80730FFF77FFE03B056
:10E038005DF804FB07B552BAADF8042040BA0822CF
:10E0480049BAADF80000ADF802105BBA694610464F
:10E05800ADF80630FFF76AFE03B05DF804FB07B5BC
:10E068000B0C042200F0070049BA8DF80400ADF843
:10E07800061097200DEB02018DF80530FFF756FECC
:10E0880003B05DF804FB000010B508B1194B186027
:10E09800F3F754FE0220FFF7A5FD0024164B204697
:10E0A8001C70FFF76DFEF4F75DFE012816D14021C4
:10E0B800FFF7D5FF40F611102146FFF773FD4FF02B
:10E0C8007F00FFF760FF0E2140F61F10FFF76AFD83
:10E0D800F4F742FE094B01221A7010BD202140F6C8
:10E0E8001110FFF75FFD202140F61210FFF75AFDCF
:10E0F800E9E700BFE40F0020E80F0020F20F00203E
:10E1080037B50C4D2B7804461BB9FFF74BFF01239D
:10E118002B700023084A6006E109F2F753FF042236
:10E1280000BA01900DEB02018620FFF7FFFD03B056
:10E1380030BD00BFE80F00200048E80107B5094BD3
:10E148008DF807000146187018B940F2AC60FFF767
:10E1580029FD01220DF107018A20FFF7E7FD03B031
:10E168005DF804FBF10F0020012873B50C46164634
:10E1780037D10020F4F7FAFDA042B8BF44B20E2808
:10E1880005461AD101231A4600210420FFF740FF53
:10E198006FF010039C42B8BF1C46182140F6E700F8
:10E1A800FFF700FD022201A98E208DF804408DF8AA
:10E1B8000560FFF7BBFD02B070BD01230A28E4B279
:10E1C8001A464FF0000105D11846FFF721FF033426
:10E1D80064B2DDE70720C5F10E05FFF719FF2C44EF
:10E1E800F6E740F6D800FFF7EDFC40F01E01C9B293
:10E1F80040F6D800FFF7D6FC0120F4F7B7FDA0429F
:10E20800B8BF44B2142805464FF001034FF000028E
:10E218000CD105210320FFF7FBFE023464B26FF036
:10E2280008039C42B8BF1C463821B7E7112805D11E
:10E2380003210220FFF7ECFE0534EFE70E2804D196
:10E2480002210846FFF7E4FEE9E7C5F116050721B4
:10E2580004202544FFF7DCFE6CB2E0E713B5314A31
:10E268000446516810686B4603C32F4B20781B780F
:10E27800834201D0FFF762FF2378032B27D8DFE81A
:10E2880003F00239283C6268284BB3FBF2F31A0CFE
:10E29800A1688DF800208DF802301A0A237B8DF8CA
:10E2A8000330637B8DF801208DF80430204A002369
:10E2B8004806C909F2F786FE030C40BA8DF8053006
:10E2C800ADF80600082269468B20FFF72FFD02B043
:10E2D80010BD2269154BB3FBF2F31A0C8DF8002020
:10E2E8008DF802301A0A237D8DF801208DF803304D
:10E2F8000422E8E7A3690093FAE762680B4BB3FBD3
:10E30800F2F31A0C8DF800208DF802301A0A237BDC
:10E318008DF80330637B8DF801208DF804300522D9
:10E32800D1E700BFA0F40008F10F00200000093D6C
:10E338000048E8011FB52E4A0446D1689068127C4F
:10E3480001AB03C31A702B4B20781B78834201D092
:10E35800FFF7F4FE2378032B26D8DFE803F0023812
:10E368003302637AF12B21D14FF6FF70FFF784FC5B
:10E3780048F20500FFF792FC02236288A188ADF8F5
:10E38800061052BAE188ADF804208DF80B30227AD5
:10E39800A37A8DF80A20ADF808108DF80C30092200
:10E3A80001A98C20FFF7C2FC04B010BDF22BE4D108
:10E3B80041F60F50FFF760FC41F22100FFF76EFCB9
:10E3C8000623DAE7237B8DF804300122E8E7E389A6
:10E3D800094A5BBAADF80430237C13708DF8063017
:10E3E800637C8DF80730638AADF808300622D7E7DA
:10E3F800A0F40008F10F0020F00F002007B502225A
:10E408008DF804008DF805108F2001A9FFF78EFC08
:10E4180003B05DF804FB000010B51346EFF3108459
:10E4280072B60A4601460348F7F790F884F3108855
:10E4380010BD00BFD401002007B5012201A9152095
:10E44800FFF7EAFF9DF804004042401003B05DF872
:10E4580004FB000037B505460C46022201A913202B
:10E46800FFF7DAFF0A4B1B78012B0DD1094B1B78FC
:10E47800012B09D140F20270FFF7A4FB9DF805308B
:10E488002870237003B030BD9DF80400F6E700BF84
:10E49800F10F0020F00F0020F7B50D4606460024C6
:10E4A8000DF10701284617468DF80740FFF7D2FF00
:10E4B8002A78BA4207D89DF807003146FFF726FCAC
:10E4C800204603B0F0BD0120FBE7000013B503228E
:10E4D800044601A91420FFF79FFF184B1A782270F1
:10E4E8004AB1012A17D014220021204600F0CEFAA2
:10E4F8000F2323700DE09DF8043023719DF805303B
:10E50800A2605B425B10A3719DF806305B425B1012
:10E51800637102B010BD9DF804305B425B10237339
:10E528009DF9053002339B1063739DF806305B42FA
:10E538005B10A373024B1B682361EAE7F10F00200D
:10E54800EC0F0020012908B5034608460ED1012B1F
:10E5580007D10420FFF746FB0220BDE80840F4F786
:10E56800FDBB022B14BF08460320F6E70120F4E7A1
:10E5780038B50446F4F7F4FB50B102280CBF022565
:10E588000125284602222146FFF7EEFD284638BD20
:10E59800102CB4BF01250225F3E7012070470000C5
:10E5A800014B01201B681847E40F0020014B022093
:10E5B8001B681847E40F0020014B40201B681847D0
:10E5C800E40F002011B1012904D07047044B1B68E7
:10E5D80080201847024B4FF480701B68F9E700BF92
:10E5E800E40F0020024B4FF400701B68184700BF6F
:10E5F800E40F0020014B20201B681847E40F00207F
:10E60800014B04201B681847E40F0020014B082029
:10E618001B681847E40F0020014B10201B6818479F
:10E62800E40F0020024B4FF480401B68184700BFDE
:10E63800E40F002010B568B1074A002352F83340B0
:10E64800844202EBC30101D9087910BD0133162BAE
:10E65800F4D1FEE71F20F8E77402010873B51D4BDB
:10E668000193044640F607000D46FFF7ABFAC0F3E6
:10E67800C10308336B4413F8042C00F0070301337B
:10E6880002FA03F3144AB2FBF3F2B2FBF4F00728E0
:10E698001ED84000042834BF042302234FF4D66058
:10E6A80002FB03F4FFF78EFA060240F2B160FFF7AF
:10E6B80089FA06F470663043030544BF6FEA0050D8
:10E6C8006FEA105063094343DB112B6002B070BD41
:10E6D8000123E3E704080A0C0048E8014FF0FF3083
:10E6E80070474FF0FF307047704700207047002098
:10E6F800704770474FF0FF3070474FF0FF3070475A
:10E70800704770477047000070B5EFF3108672B617
:10E71800144B5C8A1A8A944213D1C4F5806292B26F
:10E72800904206D3844218D901229A7000221C8094
:10E738005A825A8A0A800244C2F309025A82002085
:10E748000DE006D9C4F58065ADB28542F1D88242A4
:10E75800E9E7121B92B28242EBD84FF0FF3086F302
:10E76800108870BDF4150020EFF3108172B6034ACB
:10E77800D38A0133D38281F310887047F4150020BF
:10E78800EFF3108172B6034AD38A013BD38281F337
:10E7980010887047F415002010B508481822002189
:10E7A80000F074F906484FF48062002100F06EF919
:10E7B800044B05481B68BDE810401847F4150020B5
:10E7C800F311002088F500083DE90008014B586066
:10E7D800704700BFF4150020014B1872704700BF46
:10E7E800F415002073B5EFF3108572B61C4CE08A5F
:10E7F80000282FD1FFF7B8FF218A628A914227D0DB
:10E80800A378012B12D1238820805B1A9BB20221A6
:10E81800A382A17063B9A3702382238A9A428BBF13
:10E82800D21AC3F58063A282A38201E0002BF4D040
:10E83800268A0C4B1E4485F31088F3F76DFB0A4BB0
:10E84800A18ADB680193304602B0BDE870401847E2
:10E85800FFF796FF85F31088002002B070BD00BF57
:10E86800F4150020F311002088F5000808B4F0B56D
:10E8780086B00023ADF800302B4B0B9C1D7A8542E7
:10E888004CD3D86881434CD15B681BB112B169463F
:10E8980002A898470CAB22464FF400712348019315
:10E8A80000F0F4FBFFF760FFBDF8003018440DF1ED
:10E8B800020180B2FFF728FF01302AD00023BDF8FB
:10E8C8000020BDF802601A480DF1080C1F4699B2E5
:10E8D80016FA83F58A42ADB215D817B13244ADF8AD
:10E8E8000220BDF80250019B22464FF400712844D3
:10E8F80000F0CCFBFFF744FFFFF774FF06B0BDE85C
:10E90800F04001B070471CF8011B41550133012745
:10E91800DDE7FFF735FF6FF00200EFE76FF0040067
:10E92800ECE76FF00500E9E7F4150020F30F00208D
:10E93800F311002013B5EFF3108472B6204B9A78C8
:10E94800588A022A1DBF1A8A998A5218002214BFAF
:10E95800C2F309029A7090421A8228D0D98A0129F2
:10E9680025D19978012913D119888A1A022192B2DE
:10E97800997000219A82198062B99A701A821A8A4B
:10E9880090428BBF801AC2F5806298829A8201E019
:10E998000029F4D0188A0B4A104484F310880A4AD4
:10E9A800998AD368019302B0BDE81040184784F3F0
:10E9B8001088F3F7B5FA02B0BDE81040FFF7E0BEE3
:10E9C800F4150020F311002088F50008024A0023FE
:10E9D8001360024A13607047101600200C160020BE
:10E9E80010B5EFF3108472B641B1012903D1064A7C
:10E9F80013680343136084F3108810BD024A136838
:10EA080023EA0003F6E700BF1016002010B5EFF365
:10EA1800108472B641B1012903D1064A1368034331
:10EA2800136084F3108810BD024A136823EA0003B8
:10EA3800F6E700BF0C16002038B5EFF3108572B664
:10EA48000A4B0B4C1B6833B1236898476368984797
:10EA580085F3108838BD074B1B681BB1A36898471E
:10EA6800E368F4E7236998476369F0E71016002024
:10EA7800CCF400080C16002001380A44914200D159
:10EA8800704711F8013B00F8013FF7E700F020BCA0
:10EA980010B5EFF3108472B6064A13680343136087
:10EAA800054A52F83130034342F8313084F3108874
:10EAB80010BD00BF3816002014160020704770479C
:10EAC800B0F5803F3ABF000410230023B0F1807FE7
:10EAD8003EBF08330002DBB2B0F1805F38BF0001EF
:10EAE8004FEA1070054A38BF0433125C38BFDBB2F6
:10EAF800C3F11F03981AC0B2704700BF240301086E
:10EB08002DE9F84F384D394ED5F80080DFF8E0B0E0
:10EB1800DFF8E0A0DFF8E090D6F800C0374FDBF868
:10EB28000010374CDAF80020D9F8003008EA000065
:10EB38002860286800EA020E1EEA0C0F01D019426C
:10EB48001ED04FF0FF333B60FFF7B8FFEFF31084A0
:10EB580072B63368DBF80020DAF800100B40296839
:10EB68000B4205D1D9F80030134201D1F3F762F90D
:10EB780084F31088FFF7A3FFC5F80080BDE8F88F7D
:10EB8800236823680340134062681A4204BF4FF0A9
:10EB9800FF32626060681840FFF792FF6268386071
:10EBA800012303FA00F022EA00026260EFF3108109
:10EBB80072B63A689340326822EA030232602268E9
:10EBC80022EA0303236081F310880E4A3B6852F857
:10EBD80023309847D6F800C0DBF80010DAF8002098
:10EBE800D9F80030A5E700BF000100203816002042
:10EBF8003416002004010020301600202C160020B6
:10EC0800141600201C16002010B51146EFF31084CE
:10EC180072B6FFF755FF034B43F8201084F31088B2
:10EC280010BD00BF1C16002082B082B00DF1080C88
:10EC38000CE90600BDF8042003930B44BDF810103E
:10EC48000A4491B212B2B2F57A7FA2BFA1F57A72E4
:10EC5800013312B20360828002B002B0704782B002
:10EC680082B00DF1080C0CE90600BDF804200393EE
:10EC7800CB1ABDF81010521A91B212B2002ABEBFB8
:10EC880001F57A7203F1FF3312B20360828002B099
:10EC980002B0704730B585B0114D6B4683E803006C
:10ECA80000230293ADF80C3003A82B699847009B0A
:10ECB800BDF804400290181ABDF80C30E41AA3B24B
:10ECC80024B2002CBEBF03F57A731CB200F1FF30EA
:10ECD8002B689847AB682046984705B030BD00BF01
:10ECE80048F5000873B5114E002305460093ADF8AA
:10ECF800043001A833699847F3680090984773680F
:10ED080004469847009B1844BDF8043023449AB23F
:10ED18001BB2B3F57A7FA2BF0130A2F57A731BB29A
:10ED280028602846AB8002B070BD00BF48F50008D7
:10ED380037B500230093ADF80430074B04461B6930
:10ED480001A898476D46009095E8030084E8030001
:10ED5800204603B030BD00BF48F5000837B50F4D59
:10ED680002AB03E90300EB6898476B6804469847D1
:10ED7800BDF80430009A1B1B99B21BB2002BA2EB02
:10ED88000002BEBF01F57A7102F1FF320BB24FF4F7
:10ED98007A7000FB023003B030BD00BF48F50008B0
:10EDA8002DE9F0414FF47A75B1FBF5F5C5EB451344
:10EDB800DFF83C8005EB8303A1EBC3039CB2D8F8D2
:10EDC8000C3006469847D8F8043007469847E319A8
:10EDD80099B21BB2B3F57A7F2844A2BFA1F57A7322
:10EDE80001301BB23060B3803046BDE8F08100BF0F
:10EDF80048F50008024B00221A60024B1B681847AE
:10EE08003C1600205CF50008F8B50446174608468D
:10EE18001E467CB173B1084B00255B6A2560984794
:10EE2800069B60602581A572E6602361E7726561D3
:10EE38002846F8BD0120FCE75CF5000810B5034C36
:10EE4800E3699847A36ABDE8104018475CF50008D5
:10EE580070B5064DEB69064698476B6A044630461E
:10EE68009847AB6A201ABDE8704018475CF500085F
:10EE7800054B1B680BB918467047834201D05B6984
:10EE8800F8E70120704700BF3C1600202DE9F34148
:10EE98000B4E336A044698470123B7692372D4F8A6
:10EEA80000800546B8472844804502D2B847284420
:10EEB8002060B3682068019302B0BDE8F0411847AC
:10EEC8005CF5000870B520B3EFF3108672B6124DEA
:10EED8002B680122827253B10022427298425C6907
:10EEE8000ED102723CB120462C60FFF7CFFF86F3AB
:10EEF8001088002070BD094BDB6898472C60F6E746
:10EF08001A465B69002BF2D09842F9D143695361E4
:10EF1800EDE70120EEE700BF3C1600205CF5000895
:10EF2800084B10B51A685369516911B950614161AC
:10EF380010BD046819688C4202D91A465B69F3E768
:10EF48001946F3E73C160020044A13680BB1002168
:10EF5800197243611060FFF799BF00BF3C1600208B
:10EF68002DE9F041044600282DD0FFF781FF50BB62
:10EF7800657A45BBEFF3108872B6144E6768336A3A
:10EF8800984787422CBF27602060114FA5724FF425
:10EF9800807323813B684BB9336998472046FFF754
:10EFA800D3FF88F310882846BDE8F081B3699847F5
:10EFB800236818443B6820601B6898422046EED3BB
:10EFC800FFF7AEFFEDE70125EDE700BF5CF50008B0
:10EFD8003C16002010B5044608467CB1084B5B6A15
:10EFE800984760602046FFF743FF40B12046FFF78F
:10EFF80069FF2046BDE81040FFF7B2BF012010BDF1
:10F008005CF500082DE9F041EFF3108772B61D4E4C
:10F018001D4D736998473369044698472B684BB967
:10F028004FF000082B688BB9286828BB87F3108835
:10F03800BDE8F081011B241A1A688A428CBF121994
:10F0480000221A605B69002BF6D1E9E71C681CB145
:10F05800B36998478442E7D22C6863692B60A4F8A7
:10F068000880D4E9033098476389B3F5807FD9D104
:10F078002046FFF775FFD5E7037A002BD6D1FFF7B7
:10F0880005FFD3E75CF500083C1600202DE9F04F9A
:10F09800002997B081461E4640F3118104464F1E51
:10F0A8001378A4EB090023B90023237017B0BDE837
:10F0B800F08FB842F8DA252B05D004F8013B9046CA
:10F0C80008F10102ECE792F801E0AEF1300102F13B
:10F0D8000108AEF130034A424A41092B2BD8414678
:10F0E80000250A20884611F8013BA3F1300CBCF139
:10F0F800090F1BD998F80030692B00F09E801DD8A5
:10F10800632B29D0642B00F09880582B5AD0252BDC
:10F118001AD198F80030002B00F0938004F8013BD6
:10F12800A4EB0903BB4280F28A80C9E700FB0533E0
:10F13800A3F13005D6E74FF0FF35DBE7752B7ED01E
:10F14800782B41D0732B1CD0252304F8013BA4EB6A
:10F158000903BB4273DADCE7002D05F1FF3AD8BF9B
:10F168004FF0000A52462046202100F0B1F8A24490
:10F17800002D56F8043B8AF80030D8BF01252C44EE
:10F188009EE7504B56F804BBBBF1000F08BF9B46E7
:10F198005846F0F7EDFF2A1A8542B8BF002282468A
:10F1A80020212046019200F093F8019A002322447E
:10F1B800534502DB02EB0A0482E71BF80310D15423
:10F1C8000133F5E742F040021021DFF8FCB0DFF828
:10F1D800FCA056F804CB12F0400F18BFDA46BEF177
:10F1E800300FCDF808A0A4EB09030CBF4FF0300A8C
:10F1F8004FF0200A9207A7EB03036046CDF80CA056
:10F2080022D5002820DA4042013D4FF02D0C05AAF6
:10F21800019200228246B0FBF1F001FB10AB02988C
:10F2280010F80BB0019800F801BB5145019002F1AC
:10F238000102BAFBF1F0EDD910E042F002020A2116
:10F24800C3E708F1FF386BE7BCF1000F02D04FF0BD
:10F25800000CDCE730228DF814200122BEF1300FBB
:10F26800A5EB020504D02020002D05F1FF350ADCAE
:10F27800BCF1000F05D02D21013B04F8011B3FF420
:10F288001FAF25440AE0013B04F8010BECD117E756
:10F29800039904F8011B013B3FF412AF291B002915
:10F2A800F6DC05A9114423442244A2423FF408AFE6
:10F2B80011F8010D04F8010B9C42F6D100E700207B
:10F2C800F4E600BF34030108600301083B030108AA
:10F2D80002440346934200D1704703F8011BF9E743
:10F2E80070B50D4D0D4C641BA4100026A64209D123
:10F2F8000B4D0C4C00F098F8641BA4100026A64295
:10F3080005D170BD55F8043B98470136EEE755F82E
:10F31800043B98470136F2E790030108900301087F
:10F3280090030108940301082DE9F041C1F30A573D
:10F33800A7F2FF36132E02460B460C4605468046BA
:10F3480035DC002E17DA34A3D3E90023F0F71EFFCB
:10F3580000220023F1F760FB50B1002C57DA24F0AB
:10F3680000442C430025AC422D4C08BF4FF000440C
:10F3780023462A4624E02B4F374101EA070C5CEA72
:10F38800000C1DD024A3D3E90023F0F7FFFE0022D0
:10F398000023F1F741FB0028EAD0002CBEBF4FF450
:10F3A80080133341E41824EA07040025E0E7332EEC
:10F3B8000ADDB6F5806F03D1F0F7E8FE02460B468A
:10F3C80010461946BDE8F081A7F213474FF0FF3CFD
:10F3D8002CFA07F70742F3D00FA3D3E90023F0F77D
:10F3E800D5FE00220023F1F717FB0028C0D0002C1F
:10F3F8000ADA142E01D1013406E0C6F134060123DD
:10F40800B3401D444545F6D325EA0705B0E7002576
:10F418002C46ADE7AFF300809C7500883CE4377E4E
:10F428000000F0BFFFFF0F00F8B500BFF8BC08BC34
:10F438009E467047F8B500BFF8BC08BC9E467047AA
:10F4480000000000010000000200000000000000B1
:10F458008813000010270000204E000030750000BF
:10F46800409C000050C3000060EA0000C0D40100C6
:10F4780080A903000053070000EA063700000000D7
:10F488005000000040F7093700000000500000005D
:10F49800C194C1000000000000000000000000004E
:10F4A8000000000000000000000D0A202D2D2D2D69
:10F4B8002D20537461727420202D2D2D2D2D200D9B
:10F4C8000A0000009B1A0008891A00086D1A000833
:10F4D8008D1A0008691A0008AD1A00080D0A2023C1
:10F4E80023232323202047726F737320576569678E
:10F4F8006874203D25642020203C3C3C3C3C3C205A
:10F508000D0A000D0A20232323232320204E65748F
:10F5180020576569676874203D25642020200D0AFE
:10F52800004E657420576569676874203D2025641E
:10F53800202067200D0A00256473253033643A00C3
:10F54800C520000865210008D520000871210008A1
:10F55800352100087D21000800000000E520000892
:10F568009D20000869200008212000087920000853
:10F578008D2000082D2000083120000845200008B3
:10F58800F52300081D240008A12300088D23000886
:10F5980053776974636820746F20436C61737320B8
:10F5A800256320646F6E650D0A00414243000D0A11
:10F5B800232323232323203D204A4F494E4544201B
:10F5C8003D2000414250203D3D3D3D3D3D3D3D3DBE
:10F5D8003D3D3D3D3D3D3D3D3D3D3D3D3D0D0A00F3
:10F5E8004F544141203D3D3D3D3D3D3D3D3D3D3D2F
:10F5F8003D3D3D3D3D3D3D3D3D3D0D0A000D0A2350
:10F608002323232323203D204A4F494E20464149A6
:10F618004C45440D0A0023232323232320552F4C34
:10F62800204652414D453A4A4F494E207C2044528B
:10F638003A2564207C205057523A25640D0A004C24
:10F648006D48616E646C65722053746F70206F6EC4
:10F6580020676F696E67202E2E2E0D0A004C6D48AC
:10F66800616E646C65722053746F707065640D0A06
:10F67800004C6D48616E646C6572207377697463C1
:10F688006820746F20414250206D6F64650D0A0038
:10F698005765696774205363616C65203A20256457
:10F6A8000D0A00564444413A2025640D0A00746549
:10F6B8006D703A2025640D0A0053454E442052458A
:10F6C80051554553540D0A004E65787420547820DE
:10F6D800696E20203A207E2564207365636F6E640E
:10F6E8002873290D0A000D0A2323232323232042EC
:10F6F8004541434F4E204C4F53540D0A000D0A23E9
:10F70800232323232320424541434F4E2052454380
:10F718004549564544207C2044523A2564207C20A3
:10F72800525353493A2564207C20534E523A25645B
:10F73800207C2046513A2564207C2054494D453A86
:10F748002564207C20444553433A2564207C204985
:10F758004E464F3A303258253032582530325820EC
:10F768002530325825303258253032580D0A000DD0
:10F778000A23232323232320424541434F4E204E6F
:10F788004F542052454345495645440D0A004E56AC
:10F798004D20444154412053544F5245440D0A00D2
:10F7A8004E564D204441544120524553544F5245E2
:10F7B800440D0A004E41434B000D0A232323232303
:10F7C80023203D3D3D3D3D3D3D3D3D3D204D43508C
:10F7D800532D436F6E6669726D203D3D3D3D3D3D45
:10F7E8003D3D3D3D3D3D3D0D0A002323232323237D
:10F7F80020552F4C204652414D453A25303464203F
:10F808007C20504F52543A2564207C2044523A259B
:10F8180064207C205057523A256400207C204D53A8
:10F828004720545950453A00434F4E4649524D459A
:10F8380044205B25735D0D0A00554E434F4E4649E3
:10F84800524D45440D0A004C4544204F46460D0A8A
:10F85800004C4544204F4E0D0A0023232323232325
:10F8680020442F4C204652414D453A2530346420DF
:10F878007C20504F52543A2564207C2044523A252B
:10F8880064207C20534C4F543A2573207C205253DB
:10F8980053493A2564207C20534E523A25640D0A78
:10F8A800004E564D204441544120555020544F207D
:10F8B800444154450D0A004E564D204441544120C0
:10F8C80053544F5245204641494C45440D0A004186
:10F8D80050504C49434154494F4E5F564552534945
:10F8E8004F4E3A205625582E25582E25580D0A00D9
:10F8F8004D575F4C4F524157414E5F564552534901
:10F908004F4E3A20205625582E25582E25580D0A98
:10F91800004D575F524144494F5F56455253494F36
:10F928004E3A202020205625582E25582E25580D91
:10F938000A004C325F535045435F56455253494F76
:10F948004E3A20202020205625582E25582E25585E
:10F958000D0A0052505F535045435F564552534974
:10F968004F4E3A20202020205625582D25582E2548
:10F97800582E25580D0A0031003200435F4D4300D0
:10F98800505F4D43000000007FF9000881F900082E
:10F99800B4F5000883F900083DFC000888F9000860
:10F9A800A0860100400D0300801A060000350C00F7
:10F9B80040420F0080841E0000093D0000127A00BA
:10F9C8000024F40000366E010048E801006CDC02F7
:10F9D800000000000000000000000000000000001F
:10F9E800000000000000000000000000000000000F
:10F9F80001000000020000000300000004000000F5
:10FA080001000000030000000500000001000000E4
:10FA180001000000060000000A00000020000000AD
:10FA280002000000040000000800000010000000B0
:10FA380040000000800000000001000000020000FB
:10FA4800010002000400060008000A000C00100073
:10FA580020004000800000010804020408010101A0
:10FA680001010103070100006572726F723A2052AA
:10FA78006567696F6E206973206E6F7420646566B0
:10FA8800696E656420696E20746865204D573A2058
:10FA9800736574206C6F726177616E5F636F6E66F9
:10FAA8002E68206163636F7264696E676C790D0AF2
:10FAB800004D414320727854696D654F75740D0A85
:10FAC800004D414320747854696D654F75740D0A73
:10FAD800004D4143207278446F6E650D0A004D4118
:10FAE80043207478446F6E650D0A00080A0C0D0EE9
:10FAF80010121415181A1B1D1E21240305020501D6
:10FB080006020205000006000001050404020202C4
:10FB180002020202020202020202020203020202BC
:10FB280002020203040302020202020405040302A1
:10FB3800020202050605040302020206070605047E
:10FB4800030202070707060504030207070000006F
:10FB58000000000102010000000000020302010091
:10FB6800000000030403020100000004050403026E
:10FB78000100000506050403020100060706050446
:10FB88000302010707070605040302070700000B25
:10FB9800357DF2F2F233337373DEDEDEDE33337338
:10FBA80073F2F2F2F200000048E8010048E80100B0
:10FBB80048E8010048E8010048E8010048E8010079
:10FBC80090D00300000000000C0B0A090807073258
:10FBD80052585F2573206F6E206672657120256408
:10FBE80020487A2061742044522025640D0A00526E
:10FBF80058206F6E206672657120256420487A202F
:10FC080061742044522025640D0A005458206F6EF8
:10FC1800206672657120256420487A20617420442A
:10FC2800522025640D0A004D756C74695F43004DC0
:10FC3800756C74695F5000007FF9000881F900084D
:10FC4800B4F500082FFC00083DFC000837FC00084C
:10FC5800A584998D0DBDB1545003A97D1962E69A0A
:10FC6800459D408715EBC90BEC67FDEABFF7965B2E
:10FC7800C21CAE6A5A41024F5CF434089373533F76
:10FC88000C52655E28A10FB509369B3D2669CD9FAC
:10FC98001B9E742E2DB2EEFBF64D61CE7B3E719706
:10FCA800F568002C601FC8EDBE46D94BDED4E84A83
:10FCB8006B2AE516C5D75594CF100681F044BAE3F0
:10FCC800F3FEC08AADBC4804DFC17563301A0E6DFF
:10FCD8004C14352FE1A2CC3957F28247ACE72B956B
:10FCE800A098D17F667EAB83CA29D33C79E21D7682
:10FCF8003B564E1EDB0A6CE45D6EEFA6A8A4378B5C
:10FD0800324359B78C64D2E0B4FA0725AF8EE918AC
:10FD1800D5886F7224F1C751237C9C21DDDC868550
:10FD28009042C4AAD8050112A35FF9D0915827B907
:10FD38003813B333BB7089A7B622922049FF787A6B
:10FD48008FF88017DA31C6B8C3B07711CBFCD63A32
:10FD5800C6F8EEF6FFD6DE916002CE56E7B54DEC5A
:10FD68008F1F89FAEFB28EFB41B35F452353E49BA3
:10FD780075E13D4C6C7EF5836851D1F9E2AB622A9E
:10FD88000895469D30370A2F0E241BDFCD4E7FEA9B
:10FD9800121D583436DCB45BA476B77D52DD5E1391
:10FDA800A6B900C140E379B6D48D67729498B0853E
:10FDB800BBC54FED869A66118AE904FEA078254BEB
:10FDC800A25D80053F2170F16377AF4220E5FDBF5A
:10FDD800811826C3BE35882E9355FC7AC8BA32E6F8
:10FDE800C0199EA344543B0B8CC76B28A7BC16AD07
:10FDF800DB647414920C48B89FBD43C43931D3F204
:10FE0800D58B6EDA01B19C49D8ACF3CFCAF4471050
:10FE18006FF04A5C38577397CBA1E83E96610D0F97
:10FE2800E07C71CC9006F71CC26AAE6917993A2734
:10FE3800D9EB2B22D2A907332D3C15C987AA50A587
:10FE48000359091A65D784D082295A1E7BA86D2CBC
:10FE5800637C777BF26B6FC53001672BFED7AB767F
:10FE6800CA82C97DFA5947F0ADD4A2AF9CA472C02A
:10FE7800B7FD9326363FF7CC34A5E5F171D8311597
:10FE880004C723C31896059A071280E2EB27B275B8
:10FE980009832C1A1B6E5AA0523BD6B329E32F8430
:10FEA80053D100ED20FCB15B6ACBBE394A4C58CF28
:10FEB800D0EFAAFB434D338545F9027F503C9FA8FC
:10FEC80051A3408F929D38F5BCB6DA2110FFF3D2CA
:10FED800CD0C13EC5F974417C4A77E3D645D19737E
:10FEE80060814FDC222A908846EEB814DE5E0BDB78
:10FEF800E0323A0A4906245CC2D3AC629195E479AF
:10FF0800E7C8376D8DD54EA96C56F4EA657AAE0808
:10FF1800BA78252E1CA6B4C6E8DD741F4BBD8B8AA3
:10FF2800703EB5664803F60E613557B986C11D9E09
:10FF3800E1F8981169D98E949B1E87E9CE5528DF80
:10FF48008CA1890DBFE6426841992D0FB054BB16AC
:10FF580023232323232320257320253032583A25B1
:10FF68003032583A253032583A253032583A25300E
:10FF780032583A253032583A253032583A253032FC
:10FF8800583A253032583A253032583A25303258C6
:10FF98003A253032583A253032583A253032583AD4
:10FFA800253032583A253032580D0A0023232323AE
:10FFB8002323204465764555493A202020202020D7
:10FFC800253032583A253032583A253032583A25B9
:10FFD8003032583A253032583A253032583A25309E
:10FFE80032583A253032580D0A002323232323237D
:08FFF800204170704555493AA3
:020000040801F1
:10000000202020202020253032583A253032583AFE
:10001000253032583A253032583A253032583A2570
:100020003032583A253032583A253032580D0A00CD
:1000300023232323232320446576416464723A20DA
:1000400020202020253032583A253032583A2530A9
:1000500032583A253032580D0A004170704B65799C
:100060003A2020202020004E776B4B65793A2020E3
:10007000202020004E776B534B65793A20202020BA
:1000800000417070534B65793A2020202000444293
:10009000496E744B65793A202020004D43526F6FB2
:1000A000744B65793A2020004D434B454B65793AB6
:1000B00020202020004D43417070534B65795F3004
:1000C0003A004D434E776B534B65795F303A0000F1
:1000D000000000004150505F5A000108010000007C
:1000E0004E574B5F67000108080000004E574B5306
:1000F00074000108090000004150505381000108BC
:100100000A0000004442495F8E0001080B00000015
:100110004D4352549B0001080C0000004D434B45D9
:10012000A80001080D0000004D434B30B500010848
:100130000E0000004D415330B50001080F000000D3
:100140004D4E5330C2000108100000005A45524F76
:1001500028F50008526164696F53656E64204F761C
:10016000657273697A650D0A004952515F52585F92
:1001700054585F54494D454F55540D0A005052454F
:10018000204F4B0D0A0053594E43204F4B0D0A0090
:10019000484452204F4B0D0A00484452204B4F0D0B
:1001A0000A004952515F4352435F4552524F520D2C
:1001B0000A00020100030000841E0000093D000047
:1001C000127A000024F4000048E8010090D00300F7
:1001D00020A1070000000000B128000061510000CC
:1001E000C3A2000004050600A9D2000885D00008BB
:1001F000A5D3000801D1000831D7000891D200082A
:100200004DD50008F1D3000859CF0008ADD700083C
:10021000A9D1000895D1000879D000082DD1000897
:1002200005D10008BDD00008B3D00008B1CF000848
:100230007FD00008AFD00008ABD000083DD3000845
:1002400069D30008A1D00008C9D8000811D000085F
:10025000D9CF000899D80008B5CF00089DCF000875
:10026000A3CF0008E5E60008EBE60008A9CF0008E8
:10027000ADCF0008C01200001F000000A81600004B
:1002800017000000841C00000F000000E42500009F
:100290001E000000B42D0000160000000839000008
:1002A0000E0000002C4C00001D000000685B0000E8
:1002B00015000000747200000D0000005898000046
:1002C0001C00000034B7000014000000E8E4000047
:1002D0000C000000783101001B000000686E010076
:1002E0001300000034CA01000B0000002862020065
:1002F0001A00000040DB0200120000003C930300E3
:100300000A000000C0C204001900000060B305002C
:1003100011000000382007000900000020A107009C
:1003200000000000040302020101010100000000BE
:10033000000000003C4E554C4C3E0030313233340E
:1003400035363738396162636465666768696A6B38
:100350006C6D6E6F707172737475767778797A00E0
:1003600030313233343536373839414243444546EB
:100370004748494A4B4C4D4E4F5051525354555695
:080380005758595A0000000013
:08038800F0FDFE7F0100000002
:080390005D01000800000000FF
:0803980039010008000000001B
:1003A00000000000350300201027000000000100BD
:1003B0000000000000000000000000000400000039
:1003C000401F0000411E0008711E0008891E000821
:1003D000F51E00084D2600082D2B000835250008C5
:1003E0004D290008000000006D2500089D29000827
:1003F000512A0008F9240008D1280008DF24000849
:100400003D250008E1240008ED24000869290008C2
:100410000200000000093D00100000000000000084
:10042000E00500200000000000000000FF000000C8
:1004300000000000E00500200000000000000000B7
:10044000000000000000000000000000E0050020A7
:100450000000FF0000000000E00000001D73000825
:100460004D720008597200088572000800000000F3
:10047000000000007573000865720008E57600084A
:10048000000000000000000000000000000000006C
:10049000000E0F0D0109081101000000FF0000000F
:0804A000FFFFFFFFFFFFFFFF5C
:020000040803EF
:10E50000000000000000000000000000000000000B
:10E510000000000000000000002B7E151628AED27F
:10E52000A6ABF7158809CF4F3C012B7E151628AEF8
:10E53000D2A6ABF7158809CF4F3C082B7E151628BD
:10E54000AED2A6ABF7158809CF4F3C092B7E151626
:10E5500028AED2A6ABF7158809CF4F3C0A000000C1
:10E56000000000000000000000000000000B0000A0
:10E5700000000000000000000000000000000C008F
:10E580000000000000000000000000000000000D7E
:10E59000000000000000000000000000000000007B
:10E5A0000E0000000000000000000000000000005D
:10E5B000000F00000000000000000000000000004C
:10E5C000000010000000000000000000000000003B
:08E5D000000000000000000043
:0400000508002D7949
:00000001FF
